:100000000C9476250C944F9E0C94249E0C94F99D90
:100010000C94CE9D0C94A39D0C94789D0C944D9DB6
:100020000C94229D0C94A7250C94A7250C94A7252D
:100030000C94A7250C94F1A40C94A7250C94A72547
:100040000C94A7250C94B2B70C94A7250C94A72563
:100050000C94A7250C94A7250C940EE60C94DC9F19
:100060000C94A7250C9411790C94AB790C94A725CA
:100070000C94A7250C94A7250C94A7250C94A725D0
:100080000C94A7250C94A7250C94A7250C94A725C0
:100090000C94A7250C94A7250C94A7250C94A725B0
:1000A0000C94A7250C94A7250C94A7250C94A725A0
:1000B0000C94A7250C94A7250C94A7250C94A72590
:1000C0000C94A7250C94A7250C94A7250C94A72580
:1000D0000C94A7250C94A7250C94A7250C94A72570
:1000E0000C94A72544794A795B7966796E7983798E
:1000F0007279837976797A798379807989998C99FB
:100100007B997F998599C399909994999A999E9989
:10011000A299A899AC99B099C399B699BA99BE9980
:10012000F89EFD9E029F0C9F169F8F9F209F289FE9
:10013000309F3A9F449F4E9F5D9F679F8F9F719F07
:100140007B9F859FD7EDD7EDDEEDDEEDDEEDE5EDB6
:10015000E5EDE5EDF2EDECEDECEDECED084AD73B2D
:100160003BCE016E84BCBFFDC12F3D6C74319ABD86
:1001700056833DDA3D00C77F11BED9E4BB4C3E91AA
:100180006BAAAABE000000803F05A84CCDB2D44E99
:10019000B93836A9020C50B9918688083CA6AAAA9B
:1001A0002ABE000000803F004E414E494E4954593E
:1001B000494E46CDCCCC3D0AD7233C17B7D1387732
:1001C000CC2B329595E6241FB14F0A000020410048
:1001D00000C84200401C4620BCBE4CCA1B0E5AAE92
:1001E000C59D74434F4D4D554E49434154494F4E63
:1001F0000044525952554E004552524F52530049F5
:100200004E464F004543484F00556E6B6E6F776EFC
:1002100020636F6D6D616E643A20220041637469E2
:1002200076652045787472756465723A20004E6F69
:100230002063617365206C696768740A00000000C0
:100240000000000000000000004F666673657473D4
:10025000206170706C696564004572723A20546F59
:100260006F206661722100546F6F20666172206694
:10027000726F6D207265666572656E636520706F62
:10028000696E740A00FFFFFF4B64200023646566FB
:10029000696E65202044454641554C545F004B69CA
:1002A000200023646566696E6520204445464155FB
:1002B0004C545F004B70200023646566696E6520B6
:1002C0002044454641554C545F00504944204175F7
:1002D000746F74756E652066696E697368656421F4
:1002E0002050757420746865206C617374204B70A5
:1002F0002C204B6920616E64204B6420636F6E7309
:1003000074616E74732066726F6D2062656C6F77B6
:1003100020696E746F20436F6E66696775726174D1
:10032000696F6E2E680A00504944204175746F74DD
:10033000756E65206661696C6564212074696D6500
:100340006F75740A00544845524D414C2052554E29
:100350004157415900546865726D616C2052756E49
:10036000617761790048656174696E6720666169CB
:100370006C65640048656174696E67206661696CCC
:10038000656400504944204175746F74756E652032
:100390006661696C6564212054656D706572617475
:1003A00075726520746F6F20686967680A00204B5A
:1003B000643A2000204B693A2000204B703A20001C
:1003C0000A20436C617373696320504944200A001A
:1003D0002054753A2000204B753A2000206D61783A
:1003E0003A2000206D696E3A200020643A200020F7
:1003F000626961733A200043290A0061626C656496
:1004000020286D696E2074656D702000436F6C64E8
:1004100020657874727564657320617265200020B0
:10042000643A0020693A0020703A0020643A0020C3
:10043000693A0020703A00205A00205900580020E4
:10044000204D61783A2000205A00205900580020A1
:10045000204D696E3A20004F6E20004F66660053B3
:100460006F667420656E6473746F70733A20007ADF
:100470005F6D696E3A2000795F6D696E3A20007891
:100480005F6D696E3A20005265706F7274696E67B5
:1004900020656E6473746F70207374617475730A71
:1004A000002F2F2000454D455247454E43595F5080
:1004B000415253455200434153455F4C49474854CC
:1004C0005F4252494748544E45535300544F4747A3
:1004D0004C455F4C494748545300534F465457418D
:1004E00052455F504F574552004255494C445F506A
:1004F000455243454E54004C4556454C494E475F86
:1005000044415441005A5F50524F424500415554B6
:100510004F4C4556454C005052494E545F4A4F424D
:100520000050524F4752455353004155544F524586
:10053000504F52545F54454D5000564F4C554D4509
:100540005452494300454550524F4D00534552497E
:10055000414C5F584F4E5F584F4646004649524DFA
:10056000574152455F4E414D453A4D61726C696E3F
:1005700020204649524D574152455F5645525349F6
:100580004F4E3A312E312E382E36322045585452A5
:10059000554445525F545950453A53696E676C65EE
:1005A000457874727564657220534F555243455FA8
:1005B000434F44455F55524C3A68747470733A2FF8
:1005C0002F636F64652E616C6570686F626A656326
:1005D00074732E636F6D2F646966667573696F6ED1
:1005E0002F4D41524C494E2050524F544F434F4C87
:1005F0005F56455253494F4E3A312E30204D4143BC
:1006000048494E455F545950453A4C756C7A426F93
:10061000742054415A20352045585452554445526F
:100620005F434F554E543A3120555549443A633350
:100630003235356339362D343039372D3438383446
:100640002D386564302D6465643266663962616593
:1006500036310A004C756C7A426F742054415A202E
:1006600035204F66662E002F2F616374696F6E3AD6
:1006700070617573650A0042656420646F6E652E53
:100680000020573A004265642068656174696E67AE
:100690002E0042656420636F6F6C696E672E006F79
:1006A0006B000402FF01F801F101E3016F666600CF
:1006B00044454255473A0045787472756465722026
:1006C000257300000125301D0CFF24311C0BFF2376
:1006D0002F1B0AFFFF040308060202222B1A4142C5
:1006E000033809FF3628294527444350726F746543
:1006F000637465642050696E0A002569730025697A
:100700006D20256973002569682025696D2025699C
:100710007300256964202569682025696D20256995
:100720007300256979202569642025696820256979
:100730006D20256973005072696E742074696D654F
:100740003A200046696C652064656C657465643A9E
:100750000044656C6574696F6E206661696C6564E0
:100760002C2046696C653A20006F70656E206661CA
:10077000696C65642C2046696C653A20004D313205
:100780003500456E642066696C65206C6973740A77
:1007900000426567696E2066696C65206C697374D8
:1007A0000A00526573756D696E67207072696E74A8
:1007B000004C756C7A426F742054415A2035207277
:1007C000656164792E00436C69636B20746F2072DD
:1007D0006573756D652E2E2E00536C6565702E2E1B
:1007E0002E0047322F4733206261642070617261AE
:1007F0006D65746572730A0020746F6F206C6F6E84
:100800006720657874727573696F6E207072657693
:10081000656E7465640A0020636F6C64206578748B
:10082000727573696F6E2070726576656E7465643B
:100830000A0045313A200045303A20005A3A20005B
:10084000593A2000583A20004D53312C4D53322054
:1008500050696E730A004572726F72207772697404
:10086000696E6720746F20454550524F4D210A0034
:100870001FFFFFFFFFFFFF600000000001FF4000BF
:1008800000000000FF8000000000007F83CF000018
:100890000C303F87FF80000C301F867980000C00F1
:1008A0000F8C30C7838C30E78C30CFC7CC31F38CC2
:1008B00030DCECEC33B98C30D86C6C33198C30D024
:1008C0006C0C33198C30D86C0C33198C30DC6C0EFA
:1008D0003B198C30CF7C079F198C30C77C038F1954
:1008E00040000000000002600000000000061FFF42
:1008F000FFFFFFFFF82020506C616E6E657242753D
:100900006666657242797465733A200020467265A6
:1009100065204D656D6F72793A2000436F6D706987
:100920006C65643A204A756C2020362032303138AC
:100930000A00207C20417574686F723A2028416C4F
:10094000657068204F626A6563747320496E632E18
:100950002C204C756C7A426F742047697420526564
:10096000706F7369746F7279290A004A756C202060
:1009700036203230313831313A31323A3437002092
:100980004C61737420557064617465643A20003161
:100990002E312E380A004D61726C696E0020536F43
:1009A0006674776172652052657365740A0020571A
:1009B00061746368646F672052657365740A002010
:1009C00042726F776E206F75742052657365740A7A
:1009D000002045787465726E616C20526573657491
:1009E0000A00506F77657255700A007374617274F3
:1009F0000A006572726F722077726974696E67207F
:100A0000746F2066696C650A00456E6473746F705C
:100A10007320256320256320256320256300205A49
:100A20003A0020593A0020583A00656E6473746F9A
:100A30007073206869743A2000446F6E652073619A
:100A400076696E672066696C652E0A004D32390042
:100A500053442063617264206F6B0A006F70656E8F
:100A6000526F6F74206661696C65640A00766F6C02
:100A7000756D652E696E6974206661696C65640ABE
:100A800000534420696E6974206661696C0A0061D4
:100A900075746F25692E67004D3234004D32332056
:100AA00025730057726974696E6720746F206669D8
:100AB0006C653A20006F70656E206661696C6564D4
:100AC0002C2046696C653A20006F70656E20666167
:100AD000696C65642C2046696C653A200046696C37
:100AE000652073656C65637465640A002053697AD8
:100AF000653A200046696C65206F70656E65643AE2
:100B000020006F70656E206661696C65642C2046FC
:100B1000696C653A20002066696C653A2000646F54
:100B2000696E67006672657368004E6F77200045D6
:100B30004E4420535542524F5554494E450A0022C7
:100B400020706F73002220706172656E743A22000B
:100B5000535542524F5554494E452043414C4C2029
:100B60007461726765743A22004B494C4C45442EBF
:100B70002000747279696E6720746F2063616C6CF9
:100B8000207375622D67636F64652066696C657399
:100B9000207769746820746F6F206D616E79206CA6
:100BA0006576656C732E204D4158206C6576656CBA
:100BB0002069733A004572726F723A00486F6D6532
:100BC0002058592066697273740A00486F6D652059
:100BD0005859206669727374004E6F206D6F766588
:100BE0002E005344207072696E74696E67206279BA
:100BF000746520004E6F74205344207072696E74C7
:100C0000696E670A00436F6F6C696E6720646F6E70
:100C1000652E0048656174696E6720646F6E652E8D
:100C20000020573A00457874727564657220257308
:100C3000004D31343520533C696E6465783E206F39
:100C40007574206F662072616E67652028302D31C3
:100C5000290A00205A3A0020593A0020436F756E45
:100C60007420583A0020453A00205A3A0020593A58
:100C700000583A003A004361703A0025753A253031
:100C8000327500253032753A25303275002575648D
:100C900020253032753A253032750000060900FEF5
:100CA000000000000001090008FE00000508080619
:100CB000000040F0C88888987810050808060000F1
:100CC000C0F88888888888F8050505060001203066
:100CD000F830200508080600002070F820202020A9
:100CE000E00509090600FF2070A8A8B888887020D0
:100CF0000509090600FFE080C0B0A82830282805B3
:100D000009090600FFF8A88888888888A8F8050AD5
:100D10000A0600FE205050505088A8A8887003038F
:100D20000306000340A04000060900FE07019203ED
:100D300021207FFF07FF07FF0000000600000107DA
:100D40000706020080808080800080030202060186
:100D500005A0A00507070600005050F850F85050B5
:100D60000507070600002078A07028F02005070777
:100D7000060000C0C81020409818050707060000AC
:100D80006090A040A89068020303060104C0408060
:100D900003070706010020408080804020030707EA
:100DA0000601008040202020408005050506000146
:100DB00020A870A8200505050600012020F82020A5
:100DC0000203030602FFC04080050101060003F88C
:100DD000020202060200C0C0050505060001081057
:100DE0002040800507070600007088888888887082
:100DF00003070706010040C040404040E0050707E8
:100E0000060000708808708080F80507070600005B
:100E1000F81020100808F0050707060000103050F1
:100E200090F81010050707060000F880F008088801
:100E300070050707060000708080F088887005073D
:100E400007060000F80810202020200507070600EC
:100E50000070888870888870050707060000708811
:100E60008878080870020505060200C0C000C0C0EE
:100E70000206060602FFC0C000C040800407070645
:100E8000000010204080402010050303060002F8F7
:100E900000F804070706010080402010204080056C
:100EA00007070600007088081020002005070706C5
:100EB000000070880868A8A8700507070600007081
:100EC0008888F8888888050707060000F08888F079
:100ED0008888F00507070600007088808080887089
:100EE000050707060000F08888888888F00507074E
:100EF000060000F88080F08080F8050707060000F3
:100F0000F88080F0808080050707060000708880E8
:100F1000B8888870050707060000888888F88888E0
:100F20008801070706020080808080808080050796
:100F30000706000038101010109060050707060023
:100F4000008890A0C0A09088050707060000808058
:100F500080808080F805070706000088D8A8888868
:100F600088880507070600008888C8A8988888052B
:100F700007070600007088888888887005070706BC
:100F80000000F08888F08080800507070600007068
:100F9000888888A89068050707060000F08888F010
:100FA000A09088050707060000788080700808F088
:100FB000050707060000F82020202020200507074D
:100FC0000600008888888888887005070706000062
:100FD0008888888888502005070706000088888848
:100FE0008888A85005070706000088885020508888
:100FF00088050707060000888888502020200507FC
:1010000007060000F80810204080F80307070601D3
:1010100000E08080808080E00505050600018040BA
:10102000201008030707060100E02020202020E010
:10103000050303060004205088050101060000F89E
:101040000202020602058040050505060000700840
:101050007888780507070600008080B0C88888F087
:1010600005050506000070808088700507070600EA
:1010700000080868988888780505050600007088CB
:10108000F880700507070600003048E04040404007
:101090000506060600FF70888878087005070706B1
:1010A00000008080B0C88888880107070602008099
:1010B0000080808080800308080601FF2000202037
:1010C0002020A040040707060000808090A0C0A058
:1010D00090030707060100C04040404040E005057E
:1010E00005060000D0A8A8A8A8050505060000B0C0
:1010F000C8888888050505060000708888887005FE
:1011000006060600FFF08888F080800506060600C7
:10111000FF788888780808050505060000B0C880B3
:10112000808005050506000070807008F004070740
:101130000600004040E04040403005050506000044
:1011400088888898680505050600008888885020EA
:101150000505050600008888A8A8500505050600B5
:101160000088502050880506060600FF8888887889
:101170000870050505060000F8102040F803070771
:101180000601002040408040402001070706020081
:1011900080808080808080030707060100804040B7
:1011A0002040408005020206000268900000000610
:1011B00000005A00590058000920000000000000FB
:1011C000000000000000007FFFE0000000000000C1
:1011D0000000000000007000E000000000000000BF
:1011E000000000000061F860000000000000000046
:1011F0000000000041F82000000000000000000096
:1012000000000040F020000000000000000000008E
:10121000000040602000000000000000000000000E
:10122000005801A07F800000000000000041040081
:101230005C63A0FFC0000000000000002082005E90
:10124000F7A0FFC0000000000000002082005EF751
:10125000A0FFC0000000000000004104005C63A08B
:101260007F80000000000000008208005801A07F7D
:101270008000000000000001041000406020FFC05A
:101280000000000000000104100040F020FFC0003A
:1012900000000000000082080041F820FFC00000AC
:1012A000000000000041040061F8603F0000000001
:1012B000000000000000007000E01E0000000000C0
:1012C000000001FFFF807FFFE00C00000000000035
:1012D0000001FFFF8000000000000000000000008F
:1012E000000000007FFFE0000000000000000000A0
:1012F0000000007000E0000000000000000000009E
:101300000000630C6000000000000000000000000E
:1013100000470E2000000000000000000000000058
:101320004F0F200000000000000000000000005FE0
:101330000FA00000000000000000000000005E0799
:10134000A07F8000000000000000410400406020F9
:10135000FFC00000000000000020820040F020FFDD
:10136000C00000000000000020820040F020FFC00C
:10137000000000000000004104004060207F800069
:101380000000000000008208005E07A07F800000CF
:1013900000000000010410005F0FA0FFC00000006B
:1013A000000000010410004F0F20FFC000000000EB
:1013B000000000820800470E20FFC000000000006F
:1013C0000000410400630C603F00000000000000CA
:1013D000000000007000E01E00000000000000019E
:1013E000FFFF807FFFE00C0000000000000001FF15
:1013F000FF8000000053657474696E672054726149
:1014000076656C20416363656C65726174696F6EAB
:101410003A200053657474696E6720526574726176
:10142000637420416363656C65726174696F6E3AC1
:10143000200053657474696E67205072696E742061
:10144000416363656C65726174696F6E3A20005325
:10145000657474696E67205072696E7420616E6481
:101460002054726176656C20416363656C657261BE
:1014700074696F6E3A2000526573656E643A20009D
:101480002042002050006F6B004B494C4C45442ECD
:1014900020004B494C4C2063617573656420627970
:1014A00020746F6F206D75636820696E6163746965
:1014B00076652074696D65202D2063757272656E86
:1014C0007420636F6D6D616E643A200020204E6F52
:1014D0007A7A6C653A2000200068656174206E6F2E
:1014E0007A7A6C652E00507265737320627574741D
:1014F0006F6E20746F005052494E54205041555326
:1015000045440020204E6F7A7A6C653A2000746F53
:1015100020636F6E74696E75652E2E2E00616E6489
:1015200020707265737320627574746F6E00496EFB
:10153000736572742066696C616D656E74005052DB
:10154000494E54205041555345440020204E6F7A57
:101550007A6C653A2000200066696C616D656E7476
:10156000206C6F6164005761697420666F7200506F
:1015700052494E54205041555345440020204E6F4F
:101580007A7A6C653A2000200066696C616D656E40
:10159000742065787472756465005761697420669B
:1015A0006F72005052494E542050415553454400EB
:1015B000746F20726573756D65005761697420667C
:1015C0006F72207072696E74005052494E542050F0
:1015D000415553454400436172642072656D6F76D6
:1015E0006564004361726420696E7365727465643A
:1015F000001000C90210012C0140012201700118E5
:1016000001B0010E01F00104015002FA00B002F035
:10161000003003E600D003DC009004D2007005C85F
:1016200000A006BE000008B400B009AA00D00BA0BC
:1016300000600E960060118C000015820020197861
:1016400000C01D6E00A0226400B0275A00902C50EC
:101650000000314600E0343C0010383200903A2857
:1016600000603C1E00A03D1400803E0A00203F00A8
:10167000007C3C3E5E2B3D3F2F5B5D3B2C2A225C79
:10168000004B494C4C45442E200020746F6F206C59
:101690006F6E6720657874727573696F6E207072F3
:1016A0006576656E7465640A0020636F6C642065FE
:1016B0007874727573696F6E2070726576656E747A
:1016C00065640A0043616E6E6F74206F70656E20F2
:1016D00073756264697220006563686F3A005448EC
:1016E00045524D414C2052554E415741592042459B
:1016F0004400546865726D616C2052756E6177614B
:101700007900544845524D414C2052554E41574165
:101710005920453100544845524D414C2052554EB8
:101720004157415920453000000022002500280083
:101730002B002E00310034000201000005010801D9
:101740000B0100002100240027002A002D0030009A
:10175000330001010000040107010A010505050528
:10176000070508080808020202020A0A0808040419
:101770000404010101010101010103030303030347
:101780000303040707070C0C0C0C0C0C0C0C0202D6
:10179000020206060606060606060B0B0B0B0B0BD3
:1017A0000B0B010210202008081020401020408060
:1017B0000201020108040201010204081020408015
:1017C00080402010080402018004020180402010A3
:1017D00008040201080402010102040810204080EC
:1017E0000102040810204080000020002300260091
:1017F00029002C002F003200000100000301060127
:1018000009010201050800FF060121023520FFFF42
:1018100007FF06FF09005022165680808080008056
:10182000153353A0A0A00257575050F850F850500D
:101830000257572070A07028702013355580A040A3
:10184000A02002475740A0A040A0A05025135380DD
:10185000808012265640808080804012265680402C
:10186000404040800245559060F060900255552000
:1018700020F82020113353604080044151F011338F
:101880005340E040024656101020408080123656E9
:1018900040A0A0A0A04012365640C0404040E00208
:1018A00046566090106080F0024656F0206010901E
:1018B000600246562060A0F02020024656F080E0EC
:1018C0001090600246566080E0909060024656F0AC
:1018D0001020204040024656609060909060024682
:1018E00056609090701060122555C0C000C0C011A5
:1018F000365660600060408012365620408080403E
:1019000020034353F000F0123656804020204080E0
:1019100012365640A020400040015858304898A840
:10192000A8904030024656609090F0909002465643
:10193000E090E09090E002465660908080906002D7
:101940004656E090909090E0024656F080E080800D
:10195000F0024656F080E08080800246566090801B
:10196000B090600246569090F0909090123656E0FB
:1019700040404040E002465670202020A0400246F1
:101980005690A0C0A0A0900246568080808080F033
:1019900002465690F0F090909002465690D0F0B0EB
:1019A000B090024656609090909060024656E0904B
:1019B00090E08080014757609090D0B06010024660
:1019C00056E09090E09090024656609040209060E3
:1019D000123656E04040404040024656909090906B
:1019E00090600246569090909060600246569090AB
:1019F00090F0F0900246569090606090900256569B
:101A0000888850202020024656F010204080F01296
:101A10003656E080808080E002465680804020106C
:101A200010123656E020202020E016325240A0014D
:101A30004151F0162252804002445470909070023E
:101A400046568080E09090E01234546080806002BE
:101A5000465610107090907002445460B0C06002FE
:101A60004656205040E0404001455560907010605F
:101A70000246568080E09090901236564000C0405A
:101A800040E01137572000202020A0400246568019
:101A90008090E09090123656C040404040E00254A2
:101AA00054D0A8A8A8024454E090909002445460F6
:101AB000909060014555E090E08080014555709020
:101AC000701010024454A0D0808012345460C020A2
:101AD000C00246564040E04050200244549090904E
:101AE00070123454A0A0A04002545488A8A85002F8
:101AF000445490606090014555909070906002440D
:101B000054F02040F0024757304020C0204030229F
:101B10001656808080808080024757C02040304029
:101B200020C006425250A0FFFFFFFFFFFFFFFFFF54
:101B3000FFFFFFFFFFFFFFFFFFFFFFFFFFFFFFFFB5
:101B4000FFFFFFFFFFFFFFFF090050221656800036
:101B5000808080800146562070A0A07020024656EA
:101B60002050E04050A002555588705070880256B1
:101B7000568850F820F820221757808080008080F7
:101B8000800247577080E0907010E0173151A0023A
:101B9000565670A8C8C8A87014355560A06000E0FB
:101BA00003435350A050123353E02020143151E02E
:101BB00002565670E8D8E8D870173151E015335303
:101BC00040A04012355540E04000E014355540A09B
:101BD0002040E0143555C020C020C016225240805D
:101BE000014555909090E08002565678E8E86828C4
:101BF0002824115180112252408014355540C04094
:101C000040E014355540A04000E0034353A050A0ED
:101C1000024757808080A060F0200247578080A054
:101C2000D010207002475780408060A0F02012360C
:101C30005640004080A04002475740206090F090FE
:101C40009002475720406090F09090024757609074
:101C50006090F0909002475750A06090F0909002F2
:101C6000475790006090F0909002475760906090C6
:101C7000F0909002465670A0A0F0A0B001475760C7
:101C80009080809060400247574020F080E080F0D4
:101C90000247572040F080E080F00247576090F004
:101CA00080E080F00247579000F080E080F012372B
:101CB000578040E0404040E01237572040E040402D
:101CC00040E012375740A0E0404040E0123757A0B4
:101CD00000E0404040E00256567048E84848700234
:101CE000475750A090D0B090900247574020609046
:101CF0009090600247572040609090906002475754
:101D00006090609090906002475750A060909090D3
:101D10006002475790006090909060123353A0404B
:101D2000A002465670B0B0D0D0E002475740209095
:101D300090909060024757204090909090600247AA
:101D400057609090909090600247579000909090CC
:101D5000906002575710208850202020024656805D
:101D6000E09090E0800246566090A0A090A00247CC
:101D700057402000709090700247572040007090AC
:101D80009070024757205000709090700247575053
:101D9000A0007090907002465650007090907002B3
:101DA000475760906070909070025454F068B0781B
:101DB000113555608080604002475740200060B078
:101DC000C06002475720400060B0C06002475760C3
:101DD000900060B0C060024656500060B0C0601213
:101DE0003757804000C04040E0123757204000C0C5
:101DF0004040E012375740A000C04040E012365645
:101E0000A000C04040E0024757A040A01070906082
:101E100002475750A000E0909090024757402000A2
:101E200060909060024757204000609090600247A9
:101E3000576090006090906002475750A0006090FB
:101E400090600246569000609090601235554000B8
:101E5000E0004002445470B0D0E0024757402000F8
:101E600090909070024757204000909090700247E9
:101E7000576090009090907002465690009090901D
:101E80007001485820400090907090600147578042
:101E900080E090E0808001475790009090709060C3
:101EA00001050700FE0500FB01F220FFFE05FE050F
:101EB000FE0200400215258080800080053242A08D
:101EC000A002556550F850F8500146562070C030B9
:101ED000E0200255659010204048025565608068FA
:101EE0009068051222808002253540808080400263
:101EF00025358040404080043343A040A003334355
:101F000040E0400122324080043141E00211218052
:101F10000255650810204080024555609090906001
:101F2000022535C040404040024555E0106080F039
:101F3000024555E0106010E00245552060A0F020F9
:101F4000024555F080E010E00245556080E0906069
:101F5000024555F010204040024555609060906069
:101F600002455560907010600313238000800214B6
:101F70002480008080023545204080402003334388
:101F8000E000E00235458040204080024555E010E9
:101F90006000400255657088B8A870024555609091
:101FA00090F090024555E090E090E0023545608069
:101FB000808060024555E0909090E0023545E080D9
:101FC000E080E0023545E080E08080024555708089
:101FD000B090700245559090F09090023545E040E9
:101FE0004040E0024555301010906002455590A0E9
:101FF000C0A09002354580808080E002556588D879
:10200000A8888802455590D0B090900245556090C0
:10201000909060024555E09090E0800146566090B7
:1020200090906010024555E09090E0900245557008
:10203000806010E0023545E0404040400245559048
:10204000909090600245559090A0A0400255658800
:10205000A8A8A850024555909060909002455590D0
:1020600090701060023545E0204080E0022535C0C8
:10207000808080C00255658040201008022535C050
:10208000404040C005324240A0024151F00522329A
:1020900080400244547090907002455580E09090CA
:1020A000E00234446080806002455510709090706A
:1020B00002445460B0C0600235452040E04040001A
:1020C000465670909070106002455580E090909058
:1020D0000215258000808080002737400040404066
:1020E00040800245558090A0E090021525808080B8
:1020F0008080025464F0A8A8A8024454E090909014
:1021000002445460909060004656E09090E08080D9
:10211000004656709090701010023444A0C0808029
:1021200002445470C030E002354540E04040200297
:102130004454909090700244549090A04002546493
:10214000A8A85050023444A04040A00046569090A9
:1021500090701060024454F02040F0023545604019
:102160008040600215258080808080023545C04017
:102170002040C005425250A0FFFFFFFFFFFFFFFFBE
:10218000FFFFFFFFFFFFFFFFFFFFFFFFFFFFFFFF5F
:10219000FFFFFFFFFFFFFFFFFF020040FFFFFFFF0A
:1021A000FFFFFFFFFFFFFFFFFFFFFFFFFFFFFFFF3F
:1021B000FFFFFFFFFFFFFFFFFFFFFFFFFFFFFFFF2F
:1021C000FFFFFFFFFFFFFFFFFFFFFFFFFFFFFFFF1F
:1021D000FFFFFFFFFFFFFFFFFFFFFFFFFFFFFFFF0F
:1021E000FFFFFFFFFFFFFFFFFFFFFFFFFFFFFFFFFF
:1021F000FFFFFFFFFFFFFFFFFFFFFF01060D00FED8
:1022000009016602D620FFFE0BFE0AFE0D006022C9
:102210001969808080808080800080183363A0A04E
:10222000A00357675050F850F85050025969207871
:10223000A0A0702828F02002596948A8501020401A
:1022400050A89002586840A0A040A0989068281319
:1022500063808080113B6B20404080808080804084
:102260004020113B6B8040402020202020404080B7
:1022700006556520A870A8200455652020F8202068
:10228000113363604080065161F811336340E040D0
:1022900002596908081010204040808002596920C6
:1022A00050888888888850200259692060A02020A2
:1022B000202020F80259697088880810204080F892
:1022C000025969F8081020700808887002596910CE
:1022D0001030505090F81010025969F88080B0C842
:1022E0000808887002596970888080F08888887032
:1022F000025969F8081010202040404002596970C6
:102300008888887088888870025969708888887879
:102310000808887011386840E040000040E0401133
:10232000386840E040000060408002596908102091
:10233000408040201008045464F80000F8025969F5
:102340008040201008102040800259697088880859
:10235000102020002002596970888898A8A8B080B1
:10236000780259692050888888F8888888025969D5
:10237000F048484870484848F002596970888080A1
:102380008080808870025969F04848484848484829
:10239000F0025969F8808080F0808080F8025969E5
:1023A000F8808080F0808080800259697088808009
:1023B000809888887002596988888888F888888811
:1023C00088123969E040404040404040E00259698D
:1023D000381010101010109060025969888890A071
:1023E000C0A0908888025969808080808080808029
:1023F000F80259698888D8A8A88888888802596905
:1024000088C8C8A8A8989888880259697088888858
:102410008888888870025969F0888888F080808070
:1024200080015A6A70888888888888A8700802594C
:1024300069F0888888F0A09088880259697088803F
:10244000807008088870025969F820202020202018
:10245000202002596988888888888888887002596D
:102460006988888888505050202002596988888857
:1024700088A8A8A8A85002596988885050205050B0
:1024800088880259698888505020202020200259CD
:1024900069F808101020404080F8113B6BE0808004
:1024A00080808080808080E0025969808040402068
:1024B00010100808113B6BE0202020202020202055
:1024C00020E0085363205088015161F82A2262807D
:1024D0004002566670087888986802596980808042
:1024E000F088888888F0025666708880808870023C
:1024F000596908080878888888887802566670883C
:10250000F880887002596930484040F040404040AF
:1025100000586870888888780888700259698080B7
:1025200080B0C8888888881238684000C040404021
:1025300040E0004A6A1000301010101090906002C5
:10254000596980808090A0C0A09088123969C040ED
:10255000404040404040E0025666D0A8A8A8A88865
:10256000025666B0C888888888025666708888884F
:102570008870005868F0888888F0808080005868EB
:102580007888888878080808025666B0C8808080F5
:10259000800256667088601088700258684040F06B
:1025A00040404048300256668888888898680256BD
:1025B000668888885050200256668888A8A8A85047
:1025C000025666885020205088005868888888986D
:1025D00068088870025666F810204080F8015B6B2E
:1025E0001820202020C02020202018221969808057
:1025F00080808080808080015B6BC020202020183C
:1026000020202020C008536348A890FFFFFFFFFF51
:10261000FFFFFFFFFFFFFFFFFFFFFFFFFFFFFFFFCA
:10262000FFFFFFFFFFFFFFFFFFFFFFFF0D00602227
:1026300019698000808080808080800358682070C5
:10264000A8A0A0A8702002596930484040E040404E
:1026500048B003566688705050708802596988885F
:102660005050F820F8202022196980808080008056
:10267000808080124A6A60908060909060109060C4
:102680001A3262A0A00359697088A8D8C8D8A8884F
:1026900070045767700878887800F80356662850E9
:1026A000A0A05028045363F80808163161E00359CC
:1026B000697088E8D8D8E8D888700A5161F817445A
:1026C00064609090600357672020F8202000F8078E
:1026D000356540A02040E007356540A04020C02A75
:1026E000226240800058688888888898E880800244
:1026F000596978E8E8E8E868282828262161C02098
:102700002262408007356540C04040E00457677052
:102710008888887000F8035666A050282850A002C8
:102720005A6A40C04040E00818283808025A6A40F7
:10273000C04040E01028081038025A6A40A04020EB
:10274000A0481828380802596920002020408088B5
:102750008870025A6A40200020508888F8888802D1
:102760005A6A10200020508888F88888025A6A30F7
:10277000480020508888F88888025A6A285000202B
:10278000508888F88888025A6A50500020508888FB
:10279000F88888025A6A20502020508888F8888853
:1027A00002596958A0A0A0B0E0A0A0B8005B6B706F
:1027B00088808080808088702040025A6A40200093
:1027C000F88080F08080F8025A6A102000F880803B
:1027D000F08080F8025A6A304800F88080F08080EB
:1027E000F8025A6A505000F88080F08080F8123A5F
:1027F0006A804000E04040404040E0123A6A204099
:1028000000E04040404040E0124A6A609000E040F2
:1028100040404040E0123A6AA0A000E04040404002
:1028200040E0025969F0484848E8484848F0025AF0
:102830006A2850008888C8A8988888025A6A402068
:102840000070888888888870025A6A102000708812
:102850008888888870025A6A30480070888888881A
:102860008870025A6A2850007088888888887002A8
:102870005A6A505000708888888888700355658827
:1028800050205088015B6B08709898A8A8A8C8C809
:102890007080025A6A402000888888888888700280
:1028A0005A6A10200088888888888870025A6A309E
:1028B000480088888888888870025A6A5050008842
:1028C000888888888870025A6A102000888850207A
:1028D00020202002596980F0888888F0808080025A
:1028E0005969609090A0A0908888B00259694020F2
:1028F000007008788898680259691020007008787C
:102900008898680259693048007008788898680289
:1029100059692850007008788898680259695050A1
:1029200000700878889868025A6A30483000700849
:1029300078889868025666702870A0A85000586879
:10294000708880808870204002596940200070881B
:10295000F88088700259691020007088F8808870AB
:102960000259693048007088F880887002596950AF
:1029700050007088F8808870123969804000C0402B
:10298000404040E0123969204000C040404040E0F3
:10299000124969609000C040404040E0123969A08F
:1029A000A000C040404040E0025A6A5020601070D1
:1029B0008888888870025969285000B0C88888883B
:1029C0008802596940200070888888887002596997
:1029D000102000708888888870025969304800701B
:1029E000888888887002596928500070888888888B
:1029F0007002596950500070888888887003576742
:102A0000202000F8002020015868087098A8A8C865
:102A10007080025969402000888888889868025927
:102A200069102000888888889868025969304800B1
:102A300088888888986802596950500088888888F2
:102A40009868005B6B1020008888889868088870F8
:102A5000005A6A8080B0C88888C8B08080005B6BEC
:102A6000505000888888986808887000000000002E
:102A70000000000000000000000000000000000056
:102A800000000000000000000000000000000C003A
:102A90000000000000000C00000000000000120018
:102AA00000000000000023000000000000002100E2
:102AB0000000000000004C800000000000005E806C
:102AC0000000000000009240000000000000A14053
:102AD00000000000000121200000000000027F90A3
:102AE0000000000000020010000000000007FFF8D6
:102AF00000000000000400080000000000080004BE
:102B000000000000000800060000000000100002A5
:102B10000000000000301E010000000000207F8146
:102B2000000000000041FFE0800000000043FCF0D6
:102B30008000000000873B7840000000018EDBFC35
:102B400060000000010FEBCC20000000021FEDB67A
:102B500010000000021FDEB6100000000439CD7F17
:102B6000080000000436E0FF08000000087EC0BB3B
:102B700084000000187F005D86000000107FC0ED1B
:102B800082000000203CC07301000000203B337F26
:102B900001000000701BE77E03800000C81DEEDE10
:102BA00004C00000880FDEDC04400001240FDF3C7D
:102BB000092000012607DBF8192000027203E7F064
:102BC000139000025101FFE02290000489007F80F1
:102BD0002448000904801E004824000BFE40000029
:102BE000DFF40010004000008002001FFFFFFFFF25
:102BF000FFFE0000000000000000000000000000D8
:102C000000000000000000000000001022103C3C0A
:102C10000E1F00102210042211040010221008229E
:102C2000110400102210083C110400102210102280
:102C300011040010221020221104001E1C1E3C3C16
:102C40000E04000000000000000000000000000072
:102C50000000000000000000000000000000000074
:102C60000000000000000000000000000000000064
:102C70000000000000000000000000000000000054
:102C80000000000000000000000000000000000044
:102C90000000000000000000000000000000000034
:102CA0000000000000000000004573746570732F81
:102CB0006D6D004573746570732F6D6D005A73747C
:102CC0006570732F6D6D005A73746570732F6D6D21
:102CD000005973746570732F6D6D0059737465704E
:102CE000732F6D6D005873746570732F6D6D005880
:102CF00073746570732F6D6D004D6F74696F6E0026
:102D00004F6666004F6E2000456E6473746F7020CE
:102D100061626F72740053746570732F6D6D004A39
:102D200065726B00416363656C65726174696F6E97
:102D30000056656C6F6369747900416476616E63F7
:102D400065642053657474696E67730043616E6EC9
:102D50006F7420656E746572207375626469723A6F
:102D60002000022E2E004D61696E0020204E6F7AE9
:102D70007A6C653A200020004261636B004D696EF9
:102D8000696D756D2054656D702069732031323026
:102D90002E0048656174696E67206661696C6564C0
:102DA0000045787472756465206D6F7265005265B8
:102DB00073756D65207072696E7400524553554D80
:102DC00045204F5054494F4E533A0020204E6F7AC1
:102DD0007A6C653A20006368616E6765006F6620F3
:102DE0007468652066696C616D656E740057616911
:102DF0007420666F72207374617274005052494E71
:102E000054205041555345440020204E6F7A7A6C2F
:102E1000653A2000200066696C616D656E742075EE
:102E20006E6C6F6164005761697420666F72005048
:102E300052494E54205041555345440020204E6F76
:102E40007A7A6C653A20002000506C6561736520C9
:102E5000776169742E2E2E0048656174696E672053
:102E60006E6F7A7A6C65005052494E54205041552D
:102E700053454400506C65617365207265736574D9
:102E8000005052494E5445522048414C544544004C
:102E90005072696E7465722068616C7465642E206E
:102EA0006B696C6C28292063616C6C6564210A0075
:102EB000656E7175657565696E6720220000004852
:102EC000420000484200004040000000005761728C
:102ED0006E696E673A20486F6D696E672042756D46
:102EE000702044697669736F72203C20310A0002B9
:102EF00002040000A0400000A040000000400000CC
:102F0000954300008A4300007A432F2F6163746960
:102F10006F6E3A726573756D650A004D36303020FC
:102F2000486F74656E6420746F6F20636F6C6420EB
:102F3000746F206368616E67652066696C616D659A
:102F40006E740A004578747275646572004D6F7610
:102F500065205A004D6F76652059004D6F766520CB
:102F600058004D6F76656D656E7400436F6F6C64CD
:102F70006F776E0046616E20737065656420310066
:102F800046616E207370656564203100426564009F
:102F9000426564004E6F7A7A6C65004E6F7A7A6C87
:102FA00065004D61696E005654726176206D696EE0
:102FB000005654726176206D696E005654726176C7
:102FC000206D696E00566D696E00566D696E005613
:102FD0006D696E00566D6178204500566D617820F0
:102FE0004500566D6178204500566D6178205A0085
:102FF000566D6178205A00566D6178205A00566DE2
:103000006178205900566D6178205900566D6178BD
:10301000205900566D6178205800566D617820580F
:1030200000566D61782058004D6F74696F6E0041D5
:103030006D6178204500416D6178204500416D61EA
:1030400078205A00416D6178205A00416D617820E6
:103050005900416D6178205900416D617820580018
:10306000416D6178205800412D74726176656C0065
:10307000412D74726176656C00412D7265747261C8
:10308000637400412D7265747261637400416363FF
:10309000656C00416363656C004D6F74696F6E0011
:1030A00056652D6A65726B0056652D6A65726B00F8
:1030B00056652D6A65726B00567A2D6A65726B00D3
:1030C000567A2D6A65726B0056792D6A65726B00AF
:1030D00056792D6A65726B0056792D6A65726B00A0
:1030E00056782D6A65726B0056782D6A65726B0092
:1030F00056782D6A65726B004D6F74696F6E00248F
:10310000F4D43050C38E20C2A24017828B701112AB
:103110007A910D816CD90AA861E108C758660761E8
:103120005143061E4B5D05C145A7041A4111040910
:103130003D9803713931034036DB0265339102D487
:10314000305402802E1D02632CEE01752AC501B099
:1031500028A001102781018F2564012B244B01E059
:10316000223401AC211F018D200D01801FFC008441
:103170001EED00971DDF00B81CD200E61BC6002024
:103180001BBC00641AB200B219A8000A19A0006A98
:10319000189900D117910040178B00B516840031A3
:1031A000167E00B31579003A157300C7146F0058E6
:1031B000146A00EE1366008813630025135E00C7CF
:1031C000125B006C12570015125400C111510070AF
:1031D000114F0021114B00D61049008D10470046B9
:1031E00010440002104200C00F4000800F3E004219
:1031F0000F3C00060F3B00CB0E3800930E37005CEF
:103200000E3500270E3400F30D3200C10D31009051
:103210000D3000600D2E00320D2D00050D2C00D953
:103220000C2B00AE0C2900850C29005C0C27003506
:103230000C27000E0C2600E80B2400C40B2400A071
:103240000B23007D0B23005A0B2100390B210018A2
:103250000B2000F80A1F00D90A1E00BB0A1E009DA1
:103260000A1D00800A1D00630A1C00470A1B002C6F
:103270000A1B00110A1A00F7091A00DD091900C417
:10328000091900AB091900920917007B091800639E
:103290000917004C09160036091600200916000A05
:1032A000091500F5081500E0081400CC081400B852
:1032B000081400A4081400900813007D0812006B85
:1032C00008130058081200460812003408110023A1
:1032D0000811001208110001081100F0071000E0A9
:1032E000071000D0071000C0071000B0070F00A1A2
:1032F00007100091070E0083070F0074070F006589
:10330000070E0057070E0049070E003B070D002E61
:10331000070E0020070D0013070D0006070D00F92A
:10332000060C00ED060D00E0060C00D4060C00C8EB
:10333000060C00BC060C00B0060C00A4060B00999D
:10334000060C008D060B0082060B0077060B006C46
:10335000060B0061060A0057060B004C060A0042E5
:10336000060A0038060A002E060A0024060A001A79
:10337000060A001006090007060A00FD050900F408
:10338000050900EB050900E2050900D9050900D08F
:10339000050900C7050900BE050900B5050800AD0F
:1033A000050800A50509009C050800940508008C87
:1033B000050800840508007C050800740508006CF9
:1033C000050700650508005D050700560508004E65
:1033D00005070047050700400508003805070031CC
:1033E0000507002A050700230507001C050600162F
:1033F0000507000F0507000805060002050700FB8A
:10340000040600F5040700EE040600E8040600E2E6
:10341000040700DB040600D5040600CF040600C93B
:10342000040600C3040600BD040600B7040600B18C
:10343000040500AC040600A6040600A00405009BD9
:1034400004060095040500900406008A0405008522
:10345000040500800406007A040500750405007068
:103460000405006B04050066040500610405005CAA
:1034700004050057040500520405004D04050048EA
:10348000040500430405003E0404003A0405003529
:10349000040500300404002C040500270404002364
:1034A0000405001E0404001A04040016040500119B
:1034B0000404000D040400090405000404040000D1
:1034C000040400FC030400F8030400F4030400F007
:1034D000030400EC030400E8030400E4030400E038
:1034E000030400DC030400D8030400D4030400D068
:1034F000030400CC030400C8030300C50303002435
:10350000F404D9201BC40C5C0E9804C4095F026546
:10351000077101F405F900FB04B30048048700C1FA
:103520000369005803550003034500BE023A0084B6
:1035300002310053022A002902250004022000E47F
:10354000011C00C8011900AF011700980114008484
:10355000011300710110006101100051010E0043C0
:10356000010D0036010B002B010B0020010B001593
:103570000109000C01090003010800FB000800F329
:10358000000800EB000700E4000600DE000600D89B
:10359000000600D2000600CC000500C7000500C2EE
:1035A000000500BD000400B9000400B5000400B12E
:1035B000000400AD000400A9000400A5000300A25F
:1035C0000003009F0004009B000300980003009587
:1035D00000020093000300900003008D0002008BA6
:1035E00000030088000200860002008400030081BE
:1035F0000002007F0002007D0002007B00020079D3
:1036000000020077000100760002007400020072E0
:10361000000100710002006F0002006D0001006CEB
:103620000002006A000100690002006700010066F4
:1036300000010065000100640002006200010061F9
:10364000000100600001005F0002005D0001005CFD
:103650000001005B0001005A000100590001005800
:103660000001005700010056000100550001005400
:1036700000010053000000530001005200010051FE
:10368000000100500001004F0001004E0000004EFC
:103690000001004D0001004C0001004B0000004BF8
:1036A0000001004A000100490001004800000048F4
:1036B00000010047000100460000004600010045EF
:1036C00000000045000100440001004300000043E9
:1036D00000010042000000420001004100000041E2
:1036E000000100400001003F0000003F0001003EDB
:1036F0000000003E0001003D0000003D0001003CD4
:103700000000003C0000003C0001003B0000003BCA
:103710000001003A0000003A0001003900000039C1
:1037200000010038000000380000003800010037B8
:1037300000000037000100360000003600000036AF
:1037400000010035000000350000003500010034A4
:10375000000000340000003400010033000000339A
:10376000000000330001003200000032000000328F
:103770000001003100000031000000310001003084
:1037800000000030000000300001002F0000002F7A
:103790000000002F0000002F0001002E0000002E6E
:1037A0000000002E0001002D0000002D0000002D63
:1037B0000000002D0001002C0000002C0000002C57
:1037C0000000002C0001002B0000002B0000002B4B
:1037D0000000002B0001002A0000002A0000002A3F
:1037E0000000002A00010029000000290000002933
:1037F0000000002900000029000100280000002826
:103800000000002800000028000000280001002718
:10381000000000270000002700000027000000270C
:1038200000010026000000260000002600000026FF
:1038300000000026000100250000002500000025F2
:1038400000000025000000250000002500010024E4
:1038500000000024000000240000002400000024D8
:1038600000010023000000230000002300000023CB
:1038700000000023000000230000002300010022BC
:1038800000000022000000220000002200000022B0
:1038900000000022000100210000002100000021A2
:1038A0000000002100000021000000210000002194
:1038B0000001002000000020000000200000002087
:1038C0000000002000000020000000200000002078
:1038D0000001001F0000001F0000001F0000001F6B
:1038E0000000001F0000001F0000001F0001001E5C
:1038F0000000001E0000001E0000001E0000004D21
:10390000383420582059205A20450000060900FE6E
:1039100006018902FE20FFFE07FE06FE00000006EB
:1039200000070106060602008080808000800303F5
:1039300003060103A0A0A00507070600FF5050F8EA
:1039400050F850500509090600FE2070A8A0702804
:10395000A870200608080600FF40A8481020485418
:10396000080507070600FF609090609890680103C3
:10397000030602038080800207070602FF40808062
:10398000808080400207070602FF804040404040A0
:10399000800505050600008850F8508805050506D5
:1039A00000002020F820200204040602FEC040404F
:1039B00080050101060002F8020202060200C0C0F2
:1039C000040606060100101020408080040606064A
:1039D000010060909090906003060606010040C0D0
:1039E000404040E00406060601006090102040F0D0
:1039F000040606060100F020601010E00506060629
:103A0000000010305090F810040606060100F08007
:103A1000E01010E00406060601006080E09090606F
:103A2000040606060100F0101020404004060606B9
:103A300001006090609090600406060601006090AE
:103A400090701060020505060200C0C000C0C002F0
:103A500007070602FEC0C000C040408005050506FD
:103A600000001860806018050303060001F800F8E4
:103A7000050505060000C0300830C0040707060130
:103A8000006090106040004005060606000070903F
:103A9000A8B08070050606060000205088F88888C7
:103AA000050606060000F088F08888F00406060681
:103AB0000100609080809060040606060100E0909E
:103AC000909090E0040606060100F080E08080F00F
:103AD000040606060100F080E080808004060606E9
:103AE0000100609080B0906004060606010090908E
:103AF000F0909090030606060100E040404040E050
:103B00000506060600003810101090600406060630
:103B1000010090A0C0A090900406060601008080DD
:103B2000808080F005060606000088D8A8A888884E
:103B300004060606010090D0B09090900506060697
:103B40000000708888888870040606060100E090EE
:103B500090E080800407070601FF609090D0B0607D
:103B600010040606060100E09090E090900406061E
:103B7000060100609040209060050606060000F8EF
:103B800020202020200406060601009090909090AE
:103B900060040606060100909090F060600506063D
:103BA0000600008888A8A8D88805060606000088B0
:103BB00050202050880506060600008888502020E6
:103BC00020040606060100F010204080F0030606DF
:103BD000060100E080808080E00406060601008087
:103BE0008040201010030606060100E0202020205F
:103BF000E00503030600032050880501010600FECE
:103C0000F802020206020480400404040601007067
:103C10009090700406060601008080E09090E00419
:103C2000040406010070808070040606060100107E
:103C3000107090907004040406010060B0C070041D
:103C40000606060100205040E0404004060606013A
:103C5000FE6090907010600406060601008080E00F
:103C60009090900306060601004000C04040E0032B
:103C700008080601FE200060202020A0400406065F
:103C80000601008080A0C0A090030606060100C0C7
:103C900040404040E0050404060000D0A8A8880485
:103CA0000404060100E09090900404040601006002
:103CB0009090600406060601FEE09090E08080048B
:103CC00006060601FE7090907010100404040601B0
:103CD00000A0D0808004040406010070C030E0041D
:103CE00006060601004040E040502004040406019E
:103CF00000909090700404040601009090606005AC
:103D0000040406000088A8A85004040406010090DA
:103D10006060900406060601FE909090709060042A
:103D20000404060100F02040F0030707060100200C
:103D30004040804040200107070602FF80808080CD
:103D400080808003070706010080404020404080BB
:103D500004020206010350A0FFFFFFFFFFFFFFFF69
:103D6000FFFFFFFFFFFFFFFFFFFFFFFFFFFFFFFF63
:103D7000FFFFFFFFFFFFFFFFFF000000060007013E
:103D80000606060200800080808080040606060188
:103D9000FF2070A0A070200507070600FF304840F4
:103DA000F04040F8050505060000A8508850A80519
:103DB00006060600008850F820F8200107070602D2
:103DC000FF808080008080800407070601FF7080EC
:103DD00060906010E0030101060105A006070706D8
:103DE0000000788494A4948478030505060101609A
:103DF000A06000E00505050600002850A05028043A
:103E00000303060100F01010040101060102F00690
:103E100007070600007884B4A4A48478040101068E
:103E20000105F00403030601026090600507070620
:103E300000FF2020F8202000F803050506010140BE
:103E4000A02040E0030505060101C0204020C0027B
:103E5000020206020440800405050601FF9090B0AE
:103E6000D08005060606000078E8E86828280101E9
:103E700001060202800202020602FE4080030505DE
:103E800006010140C04040E003050506010140A0D5
:103E90004000E0050505060000A0502850A00508D8
:103EA000080600FF40C04050703078100508080632
:103EB00000FF40C04050680810380508080600FFA1
:103EC000C0204030F03078100407070601002000C1
:103ED0002060809060050707060000402020507099
:103EE0008888050707060000102020507088880584
:103EF0000707060000205020507088880507070635
:103F000000002850205070888805070706000050E0
:103F100000205070888805070706000020502050B8
:103F200070888805060606000078A0F0A0A0B804F6
:103F300008080601FE60908080906020400407071A
:103F40000601004020F080E080F004070706010031
:103F50002040F080E080F00407070601002050F0C8
:103F600080E080F00407070601005000F080E08048
:103F7000F00307070601008040E0404040E00307EF
:103F8000070601002040E0404040E003070706012B
:103F90000040A0E0404040E0030707060100A00009
:103FA000E0404040E00506060600007048E848484A
:103FB0007004070706010050A090D0B0909004074D
:103FC00007060100402060909090600407070601FA
:103FD0000020406090909060040707060100205088
:103FE000609090906004070706010050A0609090D8
:103FF00090600407070601005000609090906005F3
:10400000050506000088502050880408080601FFB6
:104010001070B0B0D0D0E080040707060100402047
:1040200090909090600407070601002040909090C7
:104030009060040707060100205090909090600463
:104040000707060100500090909090600507070652
:104050000000102088502020200406060601008061
:10406000E09090E0800406060601006090A0A09019
:10407000A00407070601004020007090907004071C
:1040800007060100204000709090700407070601A9
:10409000002050007090907004070706010050A0A7
:1040A0000070909070040606060100500070909019
:1040B00070040707060100205020709090700504DE
:1040C0000406000070A8B0780406060601FE7080A1
:1040D0008070204004070706010040200060B0C047
:1040E0007004070706010020400060B0C07004079C
:1040F0000706010020500060B0C0700406060601EB
:1041000000500060B0C07003070706010080400047
:10411000C04040E0030707060100204000C04040C7
:10412000E003070706010040A000C04040E003068E
:1041300006060100A000C04040E004070706010099
:104140003060107090906004070706010050A000D6
:10415000E0909090040707060100402000609090D6
:10416000600407070601002040006090906004078B
:1041700007060100205000609090600407070601C8
:104180000050A000609090600406060601005000F8
:10419000609090600505050600002000F8002004EE
:1041A000040406010070B0D0E004070706010040D7
:1041B00020009090907004070706010020400090B6
:1041C00090907004070706010020500090909070B6
:1041D000040606060100500090909070040909063C
:1041E00001FE204000909090709060040808060145
:1041F000FE8080E09090E080800408080601FE5078
:10420000009090907090604C696E65204E756D6264
:104210006572206973206E6F74204C617374204C3A
:10422000696E65204E756D6265722B312C204C6174
:104230007374204C696E653A200053544F505045BA
:10424000442E20005072696E7465722073746F7012
:104250007065642064756520746F206572726F727A
:10426000732E2046697820746865206572726F72BB
:1042700020616E6420757365204D39393920746F63
:1042800020726573746172742E202854656D706598
:104290007261747572652069732072657365742E1E
:1042A000205365742069742061667465722072659C
:1042B0007374617274696E67290A004E6F204368D7
:1042C00065636B73756D2077697468206C696E65C2
:1042D000206E756D6265722C204C617374204C6980
:1042E0006E653A2000636865636B73756D206D6958
:1042F000736D617463682C204C617374204C696E1B
:10430000653A20004D313130004D333100534420A7
:1043100072656164206572726F720A00446F6E6527
:10432000207072696E74696E672066696C650A0038
:1043300020496E76616C6964206578747275646575
:1043400072200000000000000000000000000000DB
:1043500000954300008A4300007A43486172646319
:104360006F6465642044656661756C742053657480
:1043700074696E6773204C6F616465640A0028235A
:104380000000282300006400000010270000000047
:10439000964300009643000040400000C8410000E2
:1043A000C9420000C9420000C84400804F44204474
:1043B0000020490020204D3330342050002044009C
:1043C00020490020204D33303120500050494420F6
:1043D00073657474696E67733A0A00204600204260
:1043E0000020480020204D3134352053004D6174A9
:1043F000657269616C2068656174757020706172A6
:10440000616D65746572733A0A00205A0020590084
:1044100020204D323036205800486F6D65206F6681
:10442000667365743A0A00204500205A002059003E
:1044300020580020420020540020204D32303520EA
:104440005300416476616E6365643A20533C6D6944
:104450006E5F66656564726174653E20543C6D698B
:104460006E5F74726176656C5F66656564726174B7
:10447000653E20423C6D696E5F7365676D656E7465
:104480005F74696D655F75733E20583C6D61785F40
:1044900078795F6A65726B3E205A3C6D61785F7A0D
:1044A0005F6A65726B3E20453C6D61785F655F6A4F
:1044B00065726B3E0A0020540020520020204D32CD
:1044C0003034205000416363656C65726174696FBC
:1044D0006E2028756E6974732F7332293A20503C10
:1044E0007072696E745F616363656C3E20523C72EA
:1044F0006574726163745F616363656C3E20543CF4
:1045000074726176656C5F616363656C3E0A00205E
:104510004500205A0020590020204D3230312058CB
:10452000004D6178696D756D20416363656C6572DE
:104530006174696F6E2028756E6974732F733229E8
:104540003A0A00204500205A0020590020204D3210
:1045500030332058004D6178696D756D2066656552
:104560006472617465732028756E6974732F732982
:104570003A0A00204500205A0020590020204D39D9
:104580003220580053746570732070657220756E08
:1045900069743A0A0020204D3230302044300A003D
:1045A00020204D3230302044002044697361626C19
:1045B00065640A0046696C616D656E74207365748C
:1045C00074696E67733A0020204D313439204320DE
:1045D0003B20556E69747320696E2043656C736966
:1045E00075730A002020473231202020203B2055BF
:1045F0006E69747320696E206D6D0A00290A0020AF
:1046000062797465733B2063726320005365747430
:10461000696E67732053746F7265642028002028C8
:1046200063616C63756C6174656429210A002021E3
:104630003D2000454550524F4D20435243206D6967
:10464000736D61746368202D202873746F726564C4
:10465000292000290A002062797465733B20637267
:104660006320002073746F726564207365747469CD
:104670006E677320726574726965766564202800C0
:10468000204D61726C696E3D563437290A00284509
:104690004550524F4D3D00454550524F4D20766597
:1046A0007273696F6E206D69736D61746368200049
:1046B0004D6F766520617869730044697361626C3F
:1046C00065207374657070657273004D38340041F5
:1046D00075746F20686F6D6500473238004D6169F1
:1046E0006E004D3530320A4D353030004C6F61640C
:1046F0002073657474696E677300526573746F72AA
:1047000065206661696C736166650053746F7265DC
:104710002073657474696E677300416476616E63BB
:1047200065642053657474696E6773004D61696ECA
:1047300000466C6F7700466C6F770046616E2073A1
:104740007065656420310046616E20737065656434
:1047500020310042656400426564004E6F7A7A6CD5
:1047600065004E6F7A7A6C6500537065656400531E
:1047700070656564004D61696E004D6F7665205807
:10478000004D6F76652059004D6F7665205A0045C3
:1047900078747275646572004D6F766520302E31C5
:1047A0006D6D004D6F766520316D6D004D6F7665D6
:1047B0002031306D6D004D6F766520617869730032
:1047C0004578747275646572004D6F7665205A0085
:1047D0004D6F76652059004D6F76652058006265F3
:1047E000640A002C2073797374656D2073746F7084
:1047F00070656421204865617465725F49443A20A0
:104800000048656174696E67206661696C65642043
:104810004245440048656174696E67206661696C51
:1048200065640048656174696E67206661696C65DE
:10483000640048656174696E67206661696C6564CF
:10484000204530001000AD0330016A0150022B01F9
:1048500070030A019004F500B005E500D006D80009
:10486000F007CE001009C500300ABE00500BB7009B
:10487000700CB100900DAB00B00EA600D00FA200DE
:10488000F0109D0010129900301395005014920002
:1048900070158E0090168B00B0178700D01884001A
:1048A000F0198100101B7E00301C7B00501D790028
:1048B000701E7600901F7300B0207000D0216E0033
:1048C000F0226B001024690030256600502663003A
:1048D0007027610090285E00B0295C00D02A590042
:1048E000F02B5600102D5400302E5100502F4E004A
:1048F00070304B0090314800B0324500D033420058
:10490000F0343E0010363B0030373700503833006B
:1049100070392E00903A2900B03B2300D03C1B0098
:10492000F03D1100103F0100F03F00004572723A67
:10493000204D494E54454D5020424544004D494E6E
:1049400054454D502074726967676572656400450F
:1049500072723A204D494E54454D50204531004524
:1049600072723A204D494E54454D50204530004515
:1049700072723A204D415854454D502042454400F2
:104980004D415854454D5020747269676765726592
:1049900064004572723A204D415854454D502045AF
:1049A00031004572723A204D415854454D502045D2
:1049B0003000202F002042403A0020403A004D367F
:1049C0003030204230005072696E7420706175730F
:1049D0006564004D31323500004D3234005072694B
:1049E0006E742061626F72746564004E6F20534470
:1049F0002063617264005072696E742066726F6D1C
:104A00002053440053746F70207072696E740041BB
:104A1000626F7574204669726D77617265005265C8
:104A200073756D65207072696E7400506175736581
:104A3000207072696E74004368616E6765206669F4
:104A40006C616D656E7400436F6E66696775726147
:104A500074696F6E0054656D70657261747572650E
:104A6000004D6F76656D656E740054756E65004916
:104A70006E666F2073637265656E0000000A0B023C
:104A8000090C0D0E080703040100000000000000DF
:104A90000000000000000000000000000000000016
:104AA00000000000000000121110000000000000D3
:104AB00000000000000000000000000000000000F6
:104AC00000486F6D65202573257325732066697214
:104AD0007374002066697273740A005A0059005892
:104AE00000486F6D65200000DF9139AF11241FBEB3
:104AF000CFEFD1E2DEBFCDBF00E00CBF13E0A0E0FE
:104B0000B2E0E2E3F4EF01E00BBF02C007900D92C8
:104B1000A63FB107D9F725E1A6EFB3E001C01D928A
:104B2000A532B207E1F715E2C5E7D5E200E006C01D
:104B300021970109802FFE010E948AF9C437D1070D
:104B400080E00807A9F70E94014C0C9408FA0C9425
:104B500000002F923F924F925F926F927F928F92BE
:104B60009F92AF92BF92CF92DF92EF92FF920F93FC
:104B70001F93CF93DF93CDB7DEB7C15CD1090FB6DA
:104B8000F894DEBF0FBECDBF8091BA048D3409F416
:104B900043C6843511F40C94D73F873411F00C943C
:104BA00018408091B8049091B9048A31910509F4B4
:104BB000F3C57CF4843091053CF4823091057CF59A
:104BC00097FF26C00C943240049709F49EC50C94BC
:104BD00032408A35910509F416C66CF48B31910583
:104BE00009F4E1C54C9711F00C94324080E00E942A
:104BF0008D5E0C9432408B35910509F408C68C35D6
:104C0000910511F00C9432400E940C5E0C943240DD
:104C10008091200281110C9435400C9432402091F7
:104C20002002222311F40C94324011E0029709F083
:104C300010E00E947BC482E50E946FC4882309F4BF
:104C40005CC10E940DC46B017C014090F91450902E
:104C5000FA146090FB147090FC148091FD149091F4
:104C6000FE14A091FF14B09100152B968CAF9DAF50
:104C7000AEAFBFAF2B972091A3043091A404409115
:104C8000A5045091A6042F962CAF3DAF4EAF5FAF59
:104C90002F978091A7049091A804A091A904B091A6
:104CA000AA0463968CAF9DAFAEAFBFAF639720E011
:104CB00030E0A901C701B6010E9466F2882309F419
:104CC0000AC5A30192012F966CAD7DAD8EAD9FAD4F
:104CD0002F970E9466F2811111C02B962CAD3DAD2D
:104CE0004EAD5FAD2B9763966CAD7DAD8EAD9FAD38
:104CF00063970E9466F2882309F4EDC420E030E057
:104D0000A901C701B6010E9466F2881F8827881F83
:104D100018130BC020E030E040E85FE3A3962CAF0F
:104D20003DAF4EAF5FAFA3970AC080E090E0A0E830
:104D3000BFEBA3968CAF9DAFAEAFBFAFA397A30160
:104D400092012F966CAD7DAD8EAD9FAD2F970E94D9
:104D50009EF66B966CAF7DAF8EAF9FAF6B972B9629
:104D60002CAD3DAD4EAD5FAD2B9763966CAD7DAD7B
:104D70008EAD9FAD63970E949EF66F966CAF7DAF30
:104D80008EAF9FAF6F976B962CAD3DAD4EAD5FADC7
:104D90006B97CA01B9010E94CBF24B015C016F967F
:104DA0002CAD3DAD4EAD5FAD6F97CA01B9010E940C
:104DB000CBF29B01AC01C501B4010E949FF60E9499
:104DC0000AF967966CAF7DAF8EAF9FAF679720E013
:104DD00030E040E05FE30E94CBF24B015C01A701B1
:104DE0009601C701B6010E94CBF26B017C01A501BF
:104DF0009401C501B4010E94CBF29B01AC01C70133
:104E0000B6010E949EF60E940AF99B01AC01A3968E
:104E10006CAD7DAD8EAD9FADA3970E94CBF24B01E3
:104E20005C012F962CAD3DAD4EAD5FAD2F97C3010C
:104E3000B2010E949FF620E030E040E05FE30E9474
:104E4000CBF26B017C016F966CAD7DAD8EAD9FADED
:104E50006F97905867962CAD3DAD4EAD5FAD67979F
:104E60000E947BF79B01AC01C501B4010E94CBF20B
:104E70009B01AC01C701B6010E949FF6A3019201FC
:104E80000E949EF66B017C0163962CAD3DAD4EAD4C
:104E90005FAD63972B966CAD7DAD8EAD9FAD2B97BF
:104EA0000E949FF620E030E040E05FE30E94CBF2FA
:104EB0002B013C0167962CAD3DAD4EAD5FAD6797C4
:104EC0006B966CAD7DAD8EAD9FAD6B970E947BF701
:104ED0009B01AC01C501B4010E94CBF29B01AC0166
:104EE000C301B2010E949FF62B962CAD3DAD4EAD95
:104EF0005FAD2B970E949EF614C089E40E946FC498
:104F0000882329F00E940DC46B017C0103C0C12CD1
:104F1000D12C76018AE40E946FC48823F9F00E94A4
:104F20000DC463966CAF7DAF8EAF9FAF639720E0EB
:104F300030E0A901C701B6010E9466F281111EC0CE
:104F400020E030E0A90163966CAD7DAD8EAD9FADE4
:104F500063970E9466F2811111C0BDC320E030E06A
:104F6000A901C701B6010E9466F2882309F4B3C300
:104F700063961CAE1DAE1EAE1FAE6397A7019601D1
:104F800050582B962CAF3DAF4EAF5FAF2B9763962B
:104F90008CAD9DADAEADBFAD6397B0582F968CAFC5
:104FA0009DAFAEAFBFAF2F97CA01B9010E94CBF240
:104FB0004B015C012F962CAD3DAD4EAD5FAD2F97F3
:104FC000CA01B9010E94CBF29B01AC01C501B40139
:104FD0000E949FF60E940AF9E3966CAF7DAF8EAFF8
:104FE0009FAFE3972091F9143091FA144091FB148C
:104FF0005091FC1467962CAF3DAF4EAF5FAF6797F3
:10500000A701960167966CAD7DAD8EAD9FAD67979C
:105010000E949FF6A3966CAF7DAF8EAF9FAFA39714
:105020008091FD149091FE14A091FF14B091001591
:105030006F968CAF9DAFAEAFBFAF6F9763962CAD41
:105040003DAD4EAD5FAD6397BC01CD010E949FF6B3
:10505000A7966CAF7DAF8EAF9FAFA7972091A304AB
:105060003091A4044091A5045091A604AB962CAFB6
:105070003DAF4EAF5FAFAB97A3962CAD3DAD4EAD00
:105080005FADA397AB966CAD7DAD8EAD9FADAB978D
:105090000E949EF66B017C018091A7049091A80468
:1050A000A091A904B091AA04AF968CAF9DAFAEAF0A
:1050B000BFAFAF97A7962CAD3DAD4EAD5FADA797F7
:1050C000BC01CD010E949EF64B015C0120910115AF
:1050D000309102154091031550910415EB962CAFB9
:1050E0003DAF4EAF5FAFEB976091AB047091AC04F6
:1050F0008091AD049091AE040E949EF66B966CAFC9
:105100007DAF8EAF9FAF6B978091AF049091B0044D
:10511000A091B104B091B204E7968CAF9DAFAEAF51
:10512000BFAFE797209105153091061540910715FF
:1051300050910815EF962CAF3DAF4EAF5FAFEF9794
:10514000A70196012B966CAD7DAD8EAD9FAD2B97D3
:105150000E94CBF22B013C01A50194012F966CAD6E
:105160007DAD8EAD9FAD2F970E94CBF29B01AC0120
:10517000C301B2010E949FF62B013C01A5019401DD
:105180002B966CAD7DAD8EAD9FAD2B970E94CBF273
:105190004B015C01A70196012F966CAD7DAD8EADE4
:1051A0009FAD2F970E94CBF29B01AC01C501B401CA
:1051B0000E949EF6A30192010E9412F76B017C01EE
:1051C00020E030E0A9010E9466F287FF0AC02BEDC3
:1051D0003FE049EC50E4C701B6010E949FF66B0125
:1051E0007C01112351F02BED3FE049EC50E4C70165
:1051F000B6010E949EF66B017C0120E030E0A9011F
:10520000C701B6010E9466F2811128C0AB962CAD91
:105210003DAD4EAD5FADAB9767966CAD7DAD8EADE0
:105220009FAD67970E9466F2811118C0AF962CADB2
:105230003DAD4EAD5FADAF976F966CAD7DAD8EADB4
:105240009FAD6F970E9466F2811108C04BEDC42E8E
:105250004FE0D42E49ECE42E40E4F42EE3962CAD3E
:105260003DAD4EAD5FADE397C701B6010E94CBF2F5
:105270009B01AC010E94CBF24B015C016B962CAD03
:105280003DAD4EAD5FAD6B97CA01B9010E94CBF247
:105290009B01AC01C501B4010E949FF60E940AF96E
:1052A0004B015C012FE632E143E85AE30E9466F2CB
:1052B00087FD0DC2C501B4010E9414F80E94E8F7F1
:1052C0001B01672B19F422242394312CB10180E0B7
:1052D00090E00E946AF24B015C019B01AC01C701A6
:1052E000B6010E947BF767966CAF7DAF8EAF9FAF24
:1052F0006797A50194016B966CAD7DAD8EAD9FADAA
:105300006B970E947BF7E3966CAF7DAF8EAF9FAF3C
:10531000E397EF962CAD3DAD4EAD5FADEF97E796C1
:105320006CAD7DAD8EAD9FADE7970E949EF6A50159
:1053300094010E947BF7E7966CAF7DAF8EAF9FAF75
:10534000E79767962CAD3DAD4EAD5FAD6797CA014F
:10535000B9010E94CBF220E030E040E05FE30E9420
:10536000CBF29B01AC0160E070E080E89FE30E941B
:105370009EF6AB966CAF7DAF8EAF9FAFAB97EB96C3
:105380008CAD9DADAEADBFADEB9789879A87AB87EE
:10539000BC87EF962CAD3DAD4EAD5FADEF972D8741
:1053A0003E874F87588B6091160270911702072E27
:1053B000000C880B990B0E946CF22091180230911E
:1053C000190240911A0250911B020E94CBF22AE06E
:1053D00037ED43E25CE30E94CBF268A379A38AA392
:1053E0009BA30E94D09F9B01AC0128533F4F4F4F7E
:1053F0005F4FAF962CAF3DAF4EAF5FAFAF972896E4
:105400004FAC289729965FAC29972A966FAC2A97BC
:105410002B967FAC2B9741E050E06D965FAF4EAF7F
:105420006D9759E168965FAF68976D96AEADBFAD69
:105430006D97A215B30509F439C10E9474E70E9463
:10544000D09FDC01CB01AF962CAD3DAD4EAD5FAD35
:10545000AF97821B930BA40BB50BB7FD11C00E9435
:10546000D09F9B01AC0128533F4F4F4F5F4FAF96EA
:105470002CAF3DAF4EAF5FAFAF9780E00E94696742
:1054800068963FAD6897315068963FAF6897332371
:1054900009F44BC0AB962CAD3DAD4EAD5FADAB97B7
:1054A0002F966CAD7DAD8EAD9FAD2F970E94CBF248
:1054B0006B017C0167962CAD3DAD4EAD5FAD67973E
:1054C000B201C3010E94CBF2A70196010E949FF690
:1054D0007B018C01AB962CAD3DAD4EAD5FADAB9776
:1054E000B201C3010E94CBF24B015C0167962CAD67
:1054F0003DAD4EAD5FAD67972F966CAD7DAD8EAD7A
:105500009FAD2F970E94CBF29B01AC01C501B40166
:105510000E949EF62B013C01C701D8012F968CAF4B
:105520009DAFAEAFBFAF2F9761C06D964EAD5FAD73
:105530006D97BA0180E090E00E946AF267962CAD08
:105540003DAD4EAD5FAD67970E94CBF24B015C0164
:105550000E9478F76B017C01C501B4010E9400F93B
:105560004B015C01A70196012B966CAD7DAD8EAD14
:105570009FAD2B970E94CBF22B013C01A50194011A
:1055800063966CAD7DAD8EAD9FAD63970E94CBF2FF
:105590009B01AC01C301B2010E949FF62B013C01AB
:1055A000A50194012B966CAD7DAD8EAD9FAD2B9773
:1055B0000E94CBF24B015C01A701960163966CAD92
:1055C0007DAD8EAD9FAD63970E94CBF29B01AC0188
:1055D000C501B4010E949EF62F966CAF7DAF8EAFD1
:1055E0009FAF2F9759E168965FAF68979201A3012B
:1055F000A3966CAD7DAD8EAD9FADA3970E949FF637
:1056000069837A838B839C832F962CAD3DAD4EAD01
:105610005FAD2F97A7966CAD7DAD8EAD9FADA79773
:105620000E949FF66D837E838F839887E3962CADCF
:105630003DAD4EAD5FADE39769857A858B859C85E1
:105640000E949FF669877A878B879C87E7962CADA7
:105650003DAD4EAD5FADE7976D857E858F859889B1
:105660000E949FF66D877E878F87988BCE0101966B
:105670000E944D69E090A1048E01005E1F4F9E01C3
:10568000235F3F4FAE01475F5F4FBE016B5F7F4FB0
:10569000CE0101960E9438C06D968EAD9FAD6D977C
:1056A00001966D969FAF8EAF6D97BFCEE090A1042F
:1056B0008E01005E1F4F2FEA34E04BEA54E067EAA8
:1056C00074E083EA94E00E9438C00E9466C50E949C
:1056D0007FA30C943240E5EBFBE084918F010F5FD8
:1056E0001F4F882321F00E948584F801F6CFE2EE57
:1056F000F7E084918F010F5F1F4F882311F40C9402
:1057000032400E948584F801F4CF80E50E946FC486
:10571000882329F00E94CDC36B017C0103C0C12CFA
:10572000D12C760183E50E946FC4882361F00E942A
:105730000DC420E030E04AE754E40E94CBF20E941E
:10574000E8F76B017C010E94E64B80912B028111EE
:1057500005C060E089ED97E00E941EC60E947FA30D
:1057600080919D0490919E04A0919F04B091A0040B
:10577000C80ED91EEA1EFB1E0E94D09FDC01CB0181
:105780008C199D09AE09BF09B7FD02C00C943240C7
:1057900080E00E946967F0CF81E080932002109240
:1057A000510A0C9432400E94EAEC81110C94324070
:1057B00080E090E0A8ECB2E489839A83AB83BC8359
:1057C00080E090E0A6E9B3E48D839E83AF83B88741
:1057D00080E090E0A0EAB1E489879A87AB87BC8734
:1057E00080E50E946FC4882319F00E94DDC301C0C8
:1057F00060E068A3BE016F5F7F4FCE0180960E947C
:10580000CECA0C9432401092B7040C94324081E01E
:105810008093B7040C9432408091B8049091B904FD
:105820008637910511F40C943A340CF0E4C08B34B3
:10583000910509F4E9C40CF05FC08831910509F4C1
:1058400094C26CF58231910509F4ECC684F497FF9B
:1058500002C00C943240823091050CF4B7C14197DC
:1058600011F00C9432400E94025E0C94324085315B
:10587000910509F470C23CF4449711F00C94324045
:10588000E1E9F7E027C28631910509F468C247973C
:1058900011F00C9432400E94E55C0C9432408E3141
:1058A000910509F4A1C2C4F48A31910509F48AC2B0
:1058B0000CF47AC28B31910509F492C24C9711F025
:1058C0000C94324040E060E080919B0490919C04F5
:1058D0000E94CF520C9432408032910509F492C359
:1058E0000CF498C38A32910509F43AC489349105BD
:1058F00009F47DC40C9432408836910509F490C4B3
:105900000CF044C08235910509F483C634F58D341A
:10591000910509F481C40CF47BC48135910511F023
:105920000C9432400E949DE40E94E64B0E94446920
:105930001092960410929504109298041092970475
:1059400068EE73E080E090E00E94D44960E084E576
:1059500096E00E941EC60C9432408435910509F4ED
:1059600061C60CF45AC68535910509F48EC68C358E
:10597000910511F00C9432404CE3C42E43E0D42E38
:1059800059E0E52E55E1F52E10E09AC68E369105C8
:1059900009F487C49CF48A36910509F47BC50CF49C
:1059A00021C58B36910509F4A1C58D36910511F0FD
:1059B0000C9432400E94A65A0C94324082379105D2
:1059C00009F4FEC634F48F36910509F47DC40C94B5
:1059D00032408337910509F4F9C68537910511F0F6
:1059E0000C94324060E080919B0490919C040E9452
:1059F000BCC80C9432408C32B1E09B0711F40C947B
:105A0000D8360CF069C0883C910509F4E1C75CF513
:105A10008D37910509F482C58CF48837910509F416
:105A2000CCC70CF466C78937910511F00C9432404D
:105A30001092970D1092960D0C9432408139910579
:105A400009F4C2C734F48C38910509F4ADC40C9440
:105A500032408B39910509F4DFC48E3B910509F47E
:105A600002C50C9432408E3C910511F40C946135C2
:105A7000C4F48B3C910509F4AFC74CF4893C910503
:105A800011F00C9432400E94976D0C9432408C3C83
:105A9000910509F4A5C78D3C910509F4A5C70C949F
:105AA00032408C3D910511F40C9438364CF4833D12
:105AB000910511F00C943240E8EDF6E10C94653557
:105AC0008D3D910511F40C944736823E910511F4F9
:105AD0000C9491360C943240843FF1E09F0711F40E
:105AE0000C946D3ED4F58E3531E0930711F40C948F
:105AF000A63FB4F48E3251E0950711F40C941F3890
:105B000014F40C9402378F32B1E09B0711F40C941B
:105B100073388033914011F40C94A1370C943240C7
:105B20008336F1E09F0711F40C94A93F4CF48F35B4
:105B3000914011F00C9432400E94AC6B0C943240B6
:105B4000803941E0940711F40C94843D8C3A9140E3
:105B500011F40C94873D0C9432408835A2E09A07EA
:105B600011F40C948D3EB4F4863FE1E09E0711F4ED
:105B70000C94733E14F40C94703E873F21E092071E
:105B800011F40C94763E8C31924011F40C94823EC8
:105B90000C9432408C3843E0940711F40C94A33FEA
:105BA0004CF48B38934011F00C9432400E94566CA8
:105BB0000C943240803AB3E09B0709F427C2873E39
:105BC000934011F40C94C23F0C943240A0909B047B
:105BD000B0909C0480E50E946FC4882359F00E9415
:105BE000CDC36B017C0111E0672B682B692B31F46D
:105BF00010E004C010E0C12CD12C760183E50E9496
:105C00006FC48823F1F00E940DC420E030E04AE721
:105C100054E40E94CBF20E94E8F76B017C01111161
:105C200012C0672B682B692B71F4A114B10459F0D1
:105C3000D5018C91882339F061E0C5010E94BCC870
:105C400007C0112391F360E086EC97E00E941EC626
:105C500081E080939A040E94E64B0E947FA3C114C6
:105C6000D104E104F104F1F080919D0490919E042F
:105C7000A0919F04B091A004C80ED91EEA1EFB1E7D
:105C80000E94D09FDC01CB018C199D09AE09BF0990
:105C9000B7FF1CC080919A048823C1F080E00E9465
:105CA0006967EECF80919A04882321F080E00E94FA
:105CB0006967F8CF8091960A60E0823019F481EB31
:105CC00097E002C082EA97E00E941EC610929A04F2
:105CD0000C94324084918F010F5F1F4F882321F075
:105CE0000E948584F801F6CF1092510D40E050E0FB
:105CF000BA018DEF9AE00E94DE798BE1EDEFFAE0D8
:105D0000DE01159601900D928A95E1F78091FB0ACC
:105D10009091FC0A9C838B838BE893E09A83898320
:105D200040E050E0BE016F5F7F4F8BEE93E00E943A
:105D3000D996CE0101960E9456AFE2E8F7E0849131
:105D40008F010F5F1F4F882311F40C9432400E9483
:105D50008584F801F4CF0E9414560C9432401092BE
:105D6000A50A1092A60A0C94324019821A821B824C
:105D70001C8218A219A21AA21BA28091990488233E
:105D800041F040E0BE016F5F7F4FCE0180960E94E0
:105D90002DAE8091A60A882319F081E08093A50A90
:105DA0000E9481940C9432401092A50A0E94239480
:105DB0008DE797E09093FA088093F9080E94F5C266
:105DC0000C9432408091A60A882311F40C9432403E
:105DD00083E50E946FC481110C94E6400C9432401C
:105DE0000E94A85C0C9432408091A60A882311F48A
:105DF0000C94324087E99CE00E94687C87E99CE033
:105E00000E941C7E1092A40A1092A30AE0909B04A8
:105E1000F0909C048091A60A882311F40C943240DF
:105E20000E94C4521D8218861C821B828BE893E05C
:105E30009A83898389EF9AE09093190B8093180BCA
:105E4000F70180818F3209F068C06FE270E0C7010E
:105E50000E94CEF98C010F5F1F4F9E012F5F3F4FB5
:105E600049010115110509F45EC06FE270E0C80137
:105E70000E94CEF96C01009709F456C00817190763
:105E800008F052C05C01A01AB10AA501B801CE0108
:105E900080960E94EEF9E0E2F0E0EC0FFD1FEA0DC3
:105EA000FB1D10828E01005E1F4FD8018D918D0168
:105EB000882319F00E948584F8CF8AE00E948584A7
:105EC0006091180B7091190B6115710511F06C5FE1
:105ED0007F4F21E0AE01405E5F4FCE0105960E94EC
:105EE0000D80811112C0BE01605E7F4F89E697E090
:105EF0000E9420A48EE20E9485848AE00E9485840C
:105F0000C4010E9456AF0C9432409092190B8092BB
:105F1000180B86010F5F1F4FA4CF8AE19BE090937F
:105F2000190B8093180B87016091180B7091190B56
:105F30006115710511F06C5F7F4F18A21BA222E062
:105F4000A801CE0180960E940D80811102C0F12C23
:105F500014C0CE0180960E9447968823C1F361E069
:105F6000CE0180960E944C7C009789F325EEFC01BF
:105F700020831BA20E94DFC8F82ECE0180960E94CB
:105F80004DC5FF2009F1E3E4F7E084917F012FEF95
:105F9000E21AF20A882321F00E948584F701F5CFE6
:105FA000D8018D918D01882319F00E948584F8CF46
:105FB0008AE00E9485841092480D1092490D10923B
:105FC0004A0D10924B0D18C0E1E5F7E084917F0176
:105FD000BFEFEB1AFB0A882321F00E948584F701AA
:105FE000F5CFF80181918F01882319F00E948584F3
:105FF000F8CF8EE20E948584CE0101960E9456AFB2
:106000000C9432400E94675C0C9432400E945C5CAD
:106010000C9432400E944D942CE3C22ED12CE12CE2
:10602000F12CA70196010E9441F6762E672ECA0137
:10603000B901A70196010E9441F66B017C01CA01DA
:10604000B90128E130E040E050E00E9441F64B0108
:106050005C01C9016DE671E00E9463F98E010F5F7A
:106060001F4F6115710599F06F927F92DF92CF9269
:106070009F928F929F938F937F936F9382E297E08B
:106080009F938F931F930F930E94FFF112C000976D
:10609000B1F06F927F92DF92CF929F928F929F93F7
:1060A0008F9382E197E09F938F931F930F930E94AA
:1060B000FFF10FB6F894DEBF0FBECDBF36C081141E
:1060C0009104A104B10479F06F927F92DF92CF9294
:1060D0009F928F9286E097E09F938F931F930F93E9
:1060E0000E94FFF1E6CFC114D104E104F10469F08C
:1060F0006F927F92DF92CF928EEF96E09F938F9375
:106100001F930F930E94FFF1D4CF6F927F928AEF7B
:1061100096E09F938F931F930F930E94FFF10F9030
:106120000F900F900F900F900F9060E0C8010E94A9
:10613000BCC8E8EDF6E184917F01BFEFEB1AFB0AE2
:10614000882321F00E948584F701F5CFB80186E30A
:1061500097E00E9420A48AE00E9485840C9432403B
:1061600083E50E946FC4882311F40C9432400E948E
:10617000EDC3E82E80E50E946FC4882311F40C94CF
:10618000324080E50E946FC4882341F00E94DDC345
:106190008B0177FF02C00C94324002C00DE010E08A
:1061A000902FE3ECF6E088E28E0F2491921729F00D
:1061B00031968E13FACF0C94F740E5EBFBE0849117
:1061C0008F010F5F1F4F882321F00E948584F80103
:1061D000F6CFEBEEF6E084918F010F5F1F4F88231F
:1061E00011F40C9432400E948584F801F4CF809120
:1061F000A50A81110C94324080E50E9440C48111AF
:106200000C9414410C9432400E9481940C943240BE
:106210000E9423940C9432400E9438940C94324093
:1062200088E690E00E940DC581110C943240809167
:10623000A20483FF02C00C94324083E50E946FC425
:10624000882311F40C9432400E940DC40E94E3F79D
:1062500070938F0460938E0480E00E9452E40E9449
:106260000DC420919004309191044091920450917A
:1062700093040E94C5F8181614F00C94324084EE72
:1062800092E09F938F9387EB96E09F938F931F925B
:106290000E94BA940F900F900F900F900F900C9453
:1062A00032408EE40E946FC4882311F40C94324073
:1062B0000E94DDC36093EA067093EB068093EC06C0
:1062C0009093ED060C94324083E50E9440C48823ED
:1062D00059F083E50E946FC4882319F00E94EDC332
:1062E00001C080E08093A204E8EDF6E184918F0183
:1062F0000F5F1F4F882321F00E948584F801F6CF9D
:10630000E0EBF6E084918F010F5F1F4F882321F0AF
:106310000E948584F801F6CFC090A204CC2099F1A8
:1063200002EAA02E06E0B02EE12CF12C80E0D12C68
:1063300096010E2C02C0359527950A94E2F720FFAE
:1063400017C099249394980E882319F08CE20E9428
:106350008584F50125913491F901849189010F5FBC
:106360001F4F882321F00E9485849801F5CF892D45
:10637000FFEFEF1AFF0A22E0A20EB11C35E0E31690
:10638000F104B1F60CC0ECEAF6E084918F010F5FE6
:106390001F4F882321F00E948584F801F6CF8AE000
:1063A0000E9485840C9432408091A20483FF02C035
:1063B0000C94324083E50E946FC4882311F40C943E
:1063C00032400E940DC40E94E3F76739710514F052
:1063D00066E970E070938D0460938C040E9407E47A
:1063E0000C94324089E690E00E940DC581110C9416
:1063F000A544EFE9F6E084918F010F5F1F4F8823DA
:1064000021F00E948584F801F6CF0E9484E38AE09F
:106410000E9485840C94A54483E50E946FC4882360
:1064200011F40C9432400E94EDC3182F8D3308F004
:106430001CE310938B040E94D09F6B017C01212FE1
:1064400030E0A8EEB3E00E948FF6C60ED71EE81E1D
:10645000F91EC0928704D0928804E0928904F092D9
:106460008A040C9432408091A20483FF02C00C94F1
:10647000324083E50E946FC460968FAF60978111B0
:106480000C941F4182E50E946FC481110C941F413E
:106490000C94324080E50E946FC4882341F00E9432
:1064A000EDC3182F823010F00C94324001C010E080
:1064B00083E50E946FC4882329F00E94DDC3362F34
:1064C000272F02C03FEF20E0E12FF0E0EE0FFF1F8B
:1064D000EB56FB4F832F922F8F3F910519F010F051
:1064E0008FEF90E0918380830C94324080E50E948E
:1064F0006FC4882341F00E94DDC36230710510F043
:106500000C94324002C060E070E0660F771FFB0120
:10651000EB56FB4F118210820C9432408CE40E94A7
:1065200040C4882319F00E940DC404C060E070E0EC
:1065300080E090EC6BAF7CAF8DAF9EAF80E090E0E1
:10654000A8ECB2E489839A83AB83BC8380E090E0BB
:10655000A6E9B3E48D839E83AF83B88780E090E0A3
:10656000A0EAB1E489879A87AB87BC8788E50E9457
:106570006FC4882379F088E50E946FC4882319F0DE
:106580000E940DC403C060E070E0CB0169837A8390
:106590008B839C8389E50E946FC4882379F089E509
:1065A0000E946FC4882319F00E940DC403C060E0EC
:1065B00070E0CB016D837E838F8398878AE50E948C
:1065C0006FC4882379F08AE50E946FC4882319F08C
:1065D0000E940DC403C060E070E0CB0169877A8738
:1065E0008B879C8718A219A21AA21BA280919904DA
:1065F00081110C94324000E020E0AE01405E5F4F1C
:10660000BE016F5F7F4FCE01CB960E9438AD0C94D8
:1066100032401092B6040C94324081E08093B6046C
:106620000C94324083E50E946FC48823A1F00E943D
:106630000DC420E030E04AE754E40E94CBF20E940F
:10664000E8F7609311027093120280931302909303
:1066500014020C94324088E50E9440C481110C94CD
:106660009B4289E50E9440C481110C949B428AE5BB
:106670000E9440C481110C949B4285E40E9440C456
:1066800081110C949B420C94BE4283E50E9440C44D
:10669000882311F40C9432400E940DC420E030E0B5
:1066A0004AE754E40E94CBF20E94E8F760937E042C
:1066B00070937F0480938004909381040C94324003
:1066C000D6018D916D010E9440C4882309F46DC0EC
:1066D000133009F063C00E940DC44B015C0120E03F
:1066E00030E040EA51E40E9466F287FF4EC0A50107
:1066F0009401609115157091161580911715909160
:1067000018150E947BF72B013C019B01AC016091A5
:106710007A0470917B0480917C0490917D040E94A6
:10672000CBF260937A0470937B0480937C04909303
:106730007D04A301920160916A0470916B048091C1
:106740006C0490916D040E94CBF260936A04709384
:106750006B0480936C0490936D0460915A04709163
:106760005B0480915C0490915D040E946AF2A30135
:1067700092010E94CBF20E94E8F760935A04709352
:106780005B0480935C0490935D0480921515909255
:106790001615A0921715B092181507C00E940DC4C7
:1067A000F70160837183828393831F5FF4E0EF0EB0
:1067B000F11C143009F084CF0E940EC00C943240BA
:1067C0000E94E64B0E9452590C943240ECE5F5E0F1
:1067D00084918F010F5F1F4F882321F00E948584D1
:1067E000F801F6CF60E08CE495E00E940E5961E07C
:1067F00085E495E00E940E5961E08AE395E00E94ED
:106800000E5961E08AE295E00E940E5960E081E253
:1068100095E00E940E5961E087E195E00E940E59D3
:1068200060E08DE095E00E940E5960E085E095E023
:106830000E940E5960E087EF94E00E940E5961E0DB
:1068400089EE94E00E940E5960E08AED94E00E9487
:106850000E5960E08CEC94E00E940E5960E086EBEB
:1068600094E00E940E5961E085EA94E00E940E597E
:106870000C94324085E40E946FC4882319F00E9472
:10688000FEC303C085E40E9440C4882361F0E8EDA4
:10689000F6E184918F010F5F1F4F882321F00E9442
:1068A0008584F801F6CF81E40E946FC4882319F033
:1068B0000E94FEC303C081E40E9440C4882361F0AB
:1068C000E1EAF4E084918F010F5F1F4F882321F0EC
:1068D0000E948584F801F6CF00919B0410919C04DE
:1068E000D8018D918D01882309F459CD0E948584AA
:1068F000F7CFE7E8F4E084918F010F5F1F4F882303
:1069000021F00E948584F801F6CFEFE7F4E084914E
:106910008F010F5F1F4F882321F00E948584F801AB
:10692000F6CF1E9B03C00DEC12E002C002ED12E098
:10693000F80181918F01882319F00E948584F8CF96
:106940008AE00E948584E7E7F4E084918F010F5F7D
:106950001F4F882321F00E948584F801F6CF1D9BEC
:1069600003C00DEC12E002C002ED12E0D8018D91DF
:106970008D01882319F00E948584F8CF8AE00E9457
:106980008584EFE6F4E084918F010F5F1F4F882329
:1069900021F00E948584F801F6CF1C9B03C00DEC0A
:1069A00012E002C002ED12E0F80181918F0188230C
:1069B00009F4F5CC0E948584F7CF81E08093970D90
:1069C0008093960D0C9432400E942F5A0C943240C2
:1069D0000E94BC6D0C9432400E94756D0C94324044
:1069E0000E940C6D0C94324083E50E9440C48823C1
:1069F00051F00E940DC460934A0470934B0480933D
:106A00004C0490934D0484E50E9440C4882351F0C7
:106A10000E940DC460934604709347048093480419
:106A20009093490482E40E9440C4882351F00E945C
:106A3000CDC36093420470934304809344049093C5
:106A4000450488E50E9440C4882351F00E940DC48B
:106A500060936E0470936F0480937004909371043C
:106A600089E50E9440C4882351F00E940DC46093C0
:106A700072047093730480937404909375048AE590
:106A80000E9440C4882351F00E940DC46093760494
:106A900070937704809378049093790485E40E943E
:106AA00040C4882311F40C9432400E940DC46093BA
:106AB0007A0470937B0480937C0490937D040C94FF
:106AC00032400E94E36C0C94324084918F010F5F3E
:106AD0001F4F882321F00E948584F801F6CF83E5BB
:106AE0000E9440C4882321F00E94FEC380931002BC
:106AF000EFE5F4E084918F010F5F1F4F882321F0B1
:106B00000E948584F801F6CF80911002811103C0A4
:106B1000EBE5F4E002C0E7E5F4E084918F010F5F5C
:106B20001F4F882321F00E948584F801F6CFEFE4FF
:106B3000F4E084918F010F5F1F4F882321F00E94A2
:106B40008584F801F6CF40902A0450902B04609081
:106B50002C0470902D04209136043091370440911C
:106B6000380450913904C301B2010E949FF6AB0171
:106B7000BC018DE494E00E94C3A380902E04909009
:106B80002F04A0903004B090310420913A04309149
:106B90003B0440913C0450913D04C501B4010E9466
:106BA0009FF6AB01BC018AE494E00E94C3A3C090AD
:106BB0003204D0903304E0903404F09035042091F6
:106BC0003E0430913F044091400450914104C7017C
:106BD000B6010E949FF6AB01BC0187E494E00E94DD
:106BE000C3A3EFE3F4E084918F010F5F1F4F88236D
:106BF00021F00E948584F801F6CF209104023091A3
:106C000005024091060250910702C301B2010E94A1
:106C10009FF6AB01BC018DE394E00E94C3A32091D9
:106C200008023091090240910A0250910B02C501FD
:106C3000B4010E949FF6AB01BC018AE394E00E947C
:106C4000C3A320910C0230910D0240910E0250918D
:106C50000F02C701B6010E949FF6AB01BC0187E39A
:106C600094E00E94C3A38AE00E9485840C94324081
:106C700083E50E946FC4882311F40C9432400E9473
:106C8000DDC370931702609316020C9432408DEDB1
:106C900090E00E940DC581110C94324083E50E9462
:106CA0006FC4882311F40C9432400091860410E0E4
:106CB0000E94DDC3000F111FF801EE5FFD4F7183CD
:106CC00060838091860490E08C01000F111F000FFB
:106CD000111F9801245E3D4F7901880F991FFC0117
:106CE000EE5FFD4F60817181072E000C880B990BC0
:106CF0000E946CF22AE037ED43E25CE30E94CBF2A3
:106D0000F801EA5DFB4F20813181428153810E946D
:106D1000CBF2D7016D937D938D939C9313970C9435
:106D2000324080E50E9440C4882311F40C94324024
:106D30000E94DDC36B017C0183E50E946FC4882340
:106D400021F00E94DDC38B0102C00FEF1FEF9801FD
:106D50002F5F3F4F2330310510F00C943240D7FEA7
:106D600002C00C9432400E94E64B0F3FBFEF1B075E
:106D700031F00130110571F401E010E00DC08C2DEF
:106D80000E947A9E31E020E0892B09F030E0032F49
:106D9000122F02C000E010E08C2D0E947A9E801716
:106DA000910711F40C94324080E00E946967F4CF9F
:106DB00083E50E946FC4882319F00E94DDC302C0DE
:106DC00064E071E079A368A380E50E946FC4882322
:106DD00039F00E94DDC36938E3E17E0730F402C078
:106DE00068EE73E07A83698304C088E893E19A834C
:106DF0008983BE01605E7F4FCE0101960E949A5743
:106E00000C94324085E40E946FC4811110C080E56B
:106E10000E9440C4882391F00E940DC46093220414
:106E200070932304809324049093250407C00E9448
:106E3000EDC3882361F3E5EBFBE072C089E40E94B7
:106E400040C4882381F00E940DC42CEA35EC47E24F
:106E50005EE30E94CBF260931E0470931F04809344
:106E600020049093210484E40E9440C4882381F08C
:106E70000E940DC42CEA35EC47E25EE30E947BF7EA
:106E800060931A0470931B0480931C0490931D0458
:106E9000E8EDF6E184918F010F5F1F4F882321F009
:106EA0000E948584F801F6CF40912204509123047A
:106EB000609124047091250483E394E00E94C3A3AD
:106EC0002CEA35EC47E25EE360911E0470911F04EA
:106ED00080912004909121040E947BF7AB01BC01BA
:106EE0008FE294E00E94A6A32CEA35EC47E25EE331
:106EF00060911A0470911B0480911C0490911D04F0
:106F00000E94CBF2AB01BC018BE294E00E94A6A3ED
:106F10008AE00E9485840C9432400E948584F801A6
:106F200084918F010F5F1F4F8111F7CF0FEE12E099
:106F3000D8018D918D01882309F431CA0E9485847E
:106F4000F7CF80E50E9440C4882351F00E940DC411
:106F50006093160470931704809318049093190497
:106F600089E40E9440C4882381F00E940DC42CEA69
:106F700035EC47E25EE30E94CBF26093120470931B
:106F80001304809314049093150484E40E9440C475
:106F9000882381F00E940DC42CEA35EC47E25EE3C1
:106FA0000E947BF760930E0470930F04809310048B
:106FB00090931104E8EDF6E184918F010F5F1F4F6C
:106FC000882321F00E948584F801F6CF40911604B1
:106FD00050911704609118047091190487E294E0AD
:106FE0000E94C3A32CEA35EC47E25EE360911204F1
:106FF0007091130480911404909115040E947BF702
:10700000AB01BC0183E294E00E94A6A32CEA35EC1C
:1070100047E25EE360910E0470910F0480911004CA
:10702000909111040E94CBF2AB01BC018FE194E07E
:107030000E94A6A38AE00E9485840C94324083E5D6
:107040000E9440C4182F882371F00E940DC40E9432
:10705000E3F7709301026093000221E0672B09F0CF
:1070600020E020930D0480E50E9440C4882359F05D
:107070002091000230910102232B11F00E94FEC3E7
:1070800080930D04EFC71111EDC7E8EDF6E184918F
:107090008F010F5F1F4F882321F00E948584F80124
:1070A000F6CF80910D04811103C06CED72E002C037
:1070B0006FEC72E08CE094E00E9420A460910002EA
:1070C000709101028BEF93E00E9407A4E7EFF3E0D9
:1070D00084918F010F5F1F4F882309F4C3C70E945B
:1070E0008584F801F5CF85E40E946FC4882321F0E0
:1070F0000E94DDC37B0102C0E12CF12C83E40E94DD
:107100006FC4882341F00E94DDC3C757DF4F6883F7
:10711000C958D04006C045E0C757DF4F4883C9581B
:10712000D04085E50E946FC4882319F00E94FEC3F9
:1071300003C085E50E9440C4CB56DF4F8883C55904
:10714000D040F7FC07C0812C912C16E1A12E13E44E
:10715000B12E06C0812C912CBCE8AB2EB2E4BB2E24
:1071600083E50E946FC4882321F00E940DC44B0167
:107170005C01E114F10411F4109286042896EFAE3C
:1071800028970E94D09FA7966CAF7DAF8EAF9FAF20
:10719000A79728965FAD289757FF0FC080E090E033
:1071A000A0E0B1E4CA55DF4F88839983AA83BB83EB
:1071B000C65AD0401CE342E00EC080E090E0A8EA4E
:1071C000B1E4CA55DF4F88839983AA83BB83C65A2B
:1071D000D04018E24AE0CB57DF4F4883C558D04033
:1071E00061E06E0D623028F4A0E0EA2EA3E0FA2EF2
:1071F0000BC003E113E0D8018D918D01882309F4C0
:10720000CEC80E948584F7CFF70181917F01882342
:1072100019F00E948584F8CF8AE00E9485840E943C
:107220009DE42896FFAD2897F7FF09C087E6809375
:107230000C04F7E64F2E512C612C712C0FC02896B0
:107240002FAD2897E22F220FFF0BE55FFB4F8FE753
:107250008083EFE74E2E512C612C712CC501B401B7
:107260000E94E3F7072E000C880B990B0E946CF22A
:1072700064966FAF649768967FAF68976C968FAF90
:107280006C97A0969FAFA097212F30E0A8EEB3E0B7
:107290000E948FF6CA56DF4F688379838A839B8367
:1072A000C659D040DC01CB01A7962CAD3DAD4EAD0B
:1072B0005FADA797820F931FA41FB51FCE55DF4F59
:1072C00088839983AA83BB83C25AD04081E080938C
:1072D000150228963FAD289737FF05C08EEC90E049
:1072E000A0E0B0E004C08FEF90E0A0E0B0E09C012F
:1072F000AD012351310941095109C455DF4F28839C
:1073000039834A835B83CC5AD0409C01AD01245120
:10731000310941095109C055DF4F288339834A8318
:107320005B83C05BD0409C01AD0155954795379577
:107330002795CC54DF4F288339834A835B83C45B12
:10734000D0409C01AD012150310941095109C85477
:10735000DF4F288339834A835B83C85BD0406396C1
:107360004CAE5DAE6EAE7FAE6397A7968CAD9DAD15
:10737000AEADBFADA797C357DF4F88839983AA836C
:10738000BB83CD58D040C656DF4F88839983AA83EC
:10739000BB83CA59D040C457DF4F1882CC58D04065
:1073A000C256DF4F188219821A821B82CE59D040F2
:1073B000E8961FAEE89790E4EC969FAFEC97ACE1AF
:1073C000E096AFAFE097B6E4E496BFAFE497C1585C
:1073D000DF4F1882CF57D040C058DF4F1882C058B7
:1073E000D040CF57DF4F1882C158D040CE57DF4F23
:1073F0001882C258D040812C912C5401AF968CAE8B
:107400009DAEAEAEBFAEAF9775016401CF56DF4FF4
:10741000188219821A821B82C159D040E1E0C557F7
:10742000DF4FE883CB58D040A9961FAE1EAEA99778
:1074300010E000E0212C312C2896FFAD28978F2FEB
:10744000FF0F990B9C01255F3B4FC655DF4F3983DA
:107450002883CA5AD040880F991F880F991FAC0102
:1074600040575B4FCD57DF4F59834883C358D040B7
:10747000CB57DF4F8881C558D040082E000C990BA0
:10748000AA0BBB0BCB57DF4F88839983AA83BB839F
:10749000C558D040C757DF4FA881C958D0400A2EE1
:1074A000000CBB0BC757DF4FB983A883C958D04026
:1074B00080911502882309F455C10E94D09F2F9610
:1074C0006CAF7DAF8EAF9FAF2F9780910A0488235A
:1074D00009F425C10E9461E52896BFAD2897B7FF42
:1074E00009C010918204009183042090840430909C
:1074F00085040AC0CD57DF4FE881F981C358D040D9
:107500001081018122803380212F302FA101C158A9
:10751000DF4F6881CF57D040C058DF4F7881C058C7
:10752000D040CF57DF4F8881C158D040CE57DF4F72
:107530009881C258D0400E9466F287FF14C0C1589B
:10754000DF4F1883CF57D040C058DF4F0883C05853
:10755000D040CF57DF4F2882C158D040CE57DF4FA1
:107560003882C258D040212F302FA101E8966FAD4C
:10757000E897EC967FADEC97E0968FADE097E496B8
:107580009FADE4970E94C5F8181664F4E8961FAF03
:10759000E897EC960FAFEC97E0962FAEE097E49665
:1075A0003FAEE497C557DF4FF881CB58D040649683
:1075B0002FAD649768963FAD68976C964FAD6C970A
:1075C000A0965FADA097612F702FC101FF2309F432
:1075D00088C00E94C5F818160CF0A1C02F962CADDB
:1075E0003DAD4EAD5FAD2F97A7968CAD9DADAEADC9
:1075F000BFADA797281B390B4A0B5B0BC254DF4F5B
:10760000288339834A835B83CE5BD040DA01C9018A
:1076100088589341A109B109B7FD81C0D301C201C6
:1076200063962CAD3DAD4EAD5FAD6397821B930B62
:10763000A40BB50B28963FAD2897B595A7959795C0
:10764000879537FF03C080930C0407C0C655DF4FF2
:10765000E881F981CA5AD0408083C254DF4F288123
:1076600039814A815B81CE5BD040CF56DF4F288382
:1076700039834A835B83C159D04064963FAD649798
:10768000C158DF4F3883CF57D04068964FAD6897C9
:10769000C058DF4F4883C058D0406C965FAD6C97A0
:1076A000CF57DF4F5883C158D040A0968FADA097D9
:1076B000CE57DF4F8883C258D0402F962CAD3DADBA
:1076C0004EAD5FAD2F97C357DF4F288339834A8371
:1076D0005B83CD58D040C557DF4F1882CB58D04080
:1076E0001EC00E9466F287FF1AC02F968CAD9DAD1A
:1076F000AEADBFAD2F97C357DF4F288139814A8187
:107700005B81CD58D040821B930BA40BB50BAC0111
:10771000BD01485853416109710977FF34C720E022
:1077200030E040EA51E464966FAD649768967FADAF
:1077300068976C968FAD6C97A0969FADA0970E94AE
:107740009FF69B01AC01612F702FC1010E94C5F80B
:1077500018167CF4E3E8F3E084918F010F5F1F4F6C
:10776000811103C00E949DE47DC40E948584F801BC
:10777000F3CF2F968CAD9DADAEADBFAD2F97C65656
:10778000DF4F288139814A815B81CA59D040821BF1
:10779000930BA40BB50BB7FDC9C00E9484E38AE02C
:1077A0000E9485842F968CAD9DADAEADBFAD2F9759
:1077B0008053984FAF4FBF4FC656DF4F8883998392
:1077C000AA83BB83CA59D040C457DF4F9881CC5895
:1077D000D040911187C0C256DF4F288139814A813C
:1077E0005B81CE59D040612F702FC1010E94C5F836
:1077F00018160CF05EC0CA55DF4F288139814A81C6
:107800005B81C65AD04064966FAD649768967FAD31
:1078100068976C968FAD6C97A0969FADA0970E94CD
:107820009EF69B01AC01A1E0C457DF4FA883CC5862
:10783000D040612F702FC1010E94C5F818162CF09E
:10784000C457DF4F1882CC58D040CB57DF4F6881E8
:1078500079818A819B81C558D0400E946CF29B013E
:10786000AC01612F702FC1010E949FF6C256DF4FFD
:10787000688379838A839B83CE59D0402F962CAD21
:107880003DAD4EAD5FAD2F97CA56DF4F88819981D0
:10789000AA81BB81C659D040280F391F4A1F5B1FE0
:1078A000CE55DF4F288339834A835B83C25AD04049
:1078B0003DC02F968CAD9DADAEADBFAD2F97CE55D3
:1078C000DF4F288139814A815B81C25AD040821BB7
:1078D000930BA40BB50BB7FD29C045E653E064E755
:1078E00073E01FC020E030E040EA51E464966FADE1
:1078F000649768967FAD68976C968FAD6C97A096ED
:107900009FADA0970E949EF69B01AC01612F702F46
:10791000C1010E9466F287FF09C045E453E065E5B6
:1079200073E028968FAD28970E9484E52F968CAD42
:107930009DADAEADBFAD2F97880F991FAA1FBB1F7E
:10794000C357DF4F288139814A815B81CD58D040B0
:10795000821B930BA40BB50BA7962CAD3DAD4EAD82
:107960005FADA797821B930BA40BB50B81389F4487
:10797000A241B10568F0E7E2F3E084918F010F5F67
:107980001F4F882309F4EECE0E948584F801F5CFBD
:10799000A9964EAD5FADA997C757DF4F88819981F2
:1079A000C958D040841795070CF0ABC0EAECF2E060
:1079B00084918F010F5F1F4F882321F00E948584DF
:1079C000F801F6CF28969FAD289797FD03C00BEEE0
:1079D00013E002C000EE12E0B80188EB92E00E94D2
:1079E00020A4B701A60184EB92E00E94C3A38AE021
:1079F0000E948584B80182EA92E00E9420A4AF969A
:107A00004CAD5DAD6EAD7FADAF978EE992E00E945B
:107A1000C3A38AE00E948584B8018CE892E00E94AA
:107A200020A4B501A40188E892E00E94C3A38AE0E3
:107A30000E948584CB56DF4FA881C559D040AA2328
:107A400009F410C32896BFAD2897B7FF2DC0C09288
:107A50001604D0921704E0921804F09219042CEA4C
:107A600035EC47E25EE3AF966CAD7DAD8EAD9FAD7C
:107A7000AF970E94CBF2609312047093130480932B
:107A80001404909315042CEA35EC47E25EE3C5013B
:107A9000B4010E947BF760930E0470930F048093EF
:107AA000100490931104DEC2C0922204D0922304E9
:107AB000E0922404F09225042CEA35EC47E25EE3E0
:107AC000AF966CAD7DAD8EAD9FADAF970E94CBF202
:107AD00060931E0470931F048093200490932104EC
:107AE0002CEA35EC47E25EE3C501B4010E947BF766
:107AF00060931A0470931B0480931C0490931D04DC
:107B0000B1C20E94E273D4CC0E94E64BABC20E9489
:107B1000EAEC8111A7C22DE3822E22E0922EE9EF3A
:107B2000F4E12996FFAFEEAF29979E012F5F3F4FFB
:107B3000590105E812E0190133E0300F2C963FAFF0
:107B40002C97F40165917591859194912996AEAD2C
:107B5000BFAD2997CD90DD90ED90FD902996BFAFF8
:107B6000AEAF2997A70196010E949EF62B013C011A
:107B700020E030E040EA51EC0E94C5F887FD10C0DB
:107B800020E030E040EA51E4C301B2010E9466F215
:107B9000181634F0F10140825182628273820DC066
:107BA000F80184911816B4F7F7FAF094F7F8F09406
:107BB000F101C082D182E282F382D101CD90DD90C9
:107BC000ED90FD901D0120E030E040EA51ECC7014E
:107BD000B6010E94C5F887FF03C0E5EBFBE00BC0D0
:107BE00020E030E040EA51E4C701B6010E9466F2AD
:107BF000181674F5F2CF84918F010F5F1F4F882301
:107C000021F00E948584F801F6CFE7E6F2E0849146
:107C10008F010F5F1F4F882321F00E948584F80198
:107C2000F6CF61E089E592E00E941EC60E940066E0
:107C300088E290E099A388A388EC90E09CAF8BAF9A
:107C4000BE01605E7F4FCE01CB960E949A570AC25A
:107C5000B4E08B0E911C0F5F1F4F2C96EFAD2C974D
:107C6000E0136FCF9EEFE92E93E0F92E10E0F501BF
:107C700081919191A191B1915F01F70181939193CC
:107C8000A193B1937F01812F0E9499C21F5F13308E
:107C900071F70E94525960E089E492E00E941EC68A
:107CA00083E992E09CAF8BAF04E610E019A308A330
:107CB000BE01655C7F4FCE0180960E949A578AEB89
:107CC00092E09CAF8BAF19A308A3BE01655C7F4F08
:107CD000CE0180960E949A57C5C10E9483D5C2C129
:107CE0000E9475D0BFC10E943FCFBCC183E50E94F6
:107CF00040C4882321F00E94FEC391E089270E949E
:107D000066CBB0C183E50E9440C4882309F4AAC1B0
:107D10000E94FEC38093FD03A5C180E090E0A8EC23
:107D2000B2E489839A83AB83BC8380E090E0A6E9C8
:107D3000B3E48D839E83AF83B88780E090E0A0EAB0
:107D4000B1E489879A87AB87BC870E94EAEC8823D5
:107D500019F081E00E948D5E85E40E9440C4882372
:107D600019F00E940DC404C060E070E080E090EC67
:107D700027966CAF7DAF8EAF9FAF27978AE50E94A5
:107D80006FC4882379F08AE50E946FC4882319F0B4
:107D90000E940DC403C060E070E0CB0169877A8760
:107DA0008B879C8788E50E946FC4882379F088E5DB
:107DB0000E946FC4882319F00E940DC403C060E0C4
:107DC00070E0CB0169837A838B839C8389E50E9471
:107DD0006FC4882379F089E50E946FC4882319F065
:107DE0000E940DC403C060E070E0CB016D837E8310
:107DF0008F83988785E50E9440C4882319F00E94EC
:107E00000DC404C060E070E088EC92EC23966CAF87
:107E10007DAF8EAF9FAF23978CE40E9440C4882330
:107E200019F00E940DC403C060E070E0CB016BAF9D
:107E30007CAF8DAF9EAF82E40E946FC4882321F097
:107E40000E94DDC3162F01C015E0F090960A8091C4
:107E50009904811172C001E0212FAE01415C5F4F96
:107E6000BE016F5F7F4FCE018D5B9F4F0E9438AD8B
:107E7000882309F462C081E080939A0480919A0477
:107E8000882309F446C060E0812F0E948D5D8091B7
:107E9000480A8823D1F100934C0A8DE693E70E94AB
:107EA000169580919A04882321F081E00E946967E9
:107EB000F8CF1092F9031092FA031092FB0310927C
:107EC000FC031092480A0E9452E40E94305D009325
:107ED0004C0A86E193E70E9416950E94D09FDC0130
:107EE000CB0188539045AF4FBF4F8093F9039093D8
:107EF000FA03A093FB03B093FC031092480A00938B
:107F00009A0461E0812F0E948D5D81E00E94696783
:107F1000B5CF80E090E0A0EAB1E488A399A3AAA33A
:107F2000BBA380919904882341F0412FBE01605E7C
:107F30007F4FCE01CB960E942DAEF1E0FF1292C092
:107F40000E9481948FC00E94396C8CC00E94016C89
:107F500089C0E5EBFBE084918F010F5F1F4F882301
:107F600021F00E948584F801F6CFEEE2F2E08491E0
:107F70008F010F5F1F4F882309F474C00E9485840E
:107F8000F801F5CF81E0809320021092510A83E539
:107F90000E946FC4882319F00E94FEC303C083E5CA
:107FA0000E9440C481115EC00E94106A5BC0F090C4
:107FB000B804FF2029F1E8EDF6E184918F010F5F0D
:107FC0001F4F882321F00E948584F801F6CF84E5B5
:107FD0000E9485846F2D70E080E090E04AE00E946E
:107FE000BF9080E20E9485840FEE12E0D8018D914F
:107FF0008D01882311F40C94CF310E948584F6CF33
:108000001092A104E8EDF6E184918F010F5F1F4FFC
:10801000882321F00E948584F801F6CF60E070E0AB
:108020008CE192E00E9407A48AE00E9485841AC035
:10803000E8EDF6E184918F010F5F1F4F882321F057
:108040000E948584F801F6CF6091F6037091F703E2
:1080500089E092E00E9420A482E20E9485848AE066
:108060000E9485840E94A26970C40E947BC483EA36
:1080700094E00E944D690E947FA38091A20483FD39
:1080800086C0C090AF04D090B004E090B104F090EE
:10809000B2042091051530910615409107155091B5
:1080A0000815C701B6010E9466F2882309F46FC063
:1080B0000E9418AD882301F1C0920515D0920615D3
:1080C000E0920715F0920815E8EDF6E184918F0132
:1080D0000F5F1F4F882321F00E948584F801F6CF9F
:1080E000E7E1F8E084918F010F5F1F4F882321F0B3
:1080F0000E948584F801F6CFC090AF04D090B00400
:10810000E090B104F090B20420910515309106156D
:108110004091071550910815C701B6010E949EF6BF
:108120009F77E091A10424E0E29FF0011124E45E36
:10813000FD4F20813181428153810E94CBF220E0AA
:1081400030E048E453E40E94C5F8181604F5C092E4
:108150000515D0920615E0920715F0920815E8ED86
:10816000F6E184918F010F5F1F4F882321F00E9459
:108170008584F801F6CFE8EFF7E084918F010F5F77
:108180001F4F882321F00E948584F801F6CF60916B
:10819000160270911702072E000C880B990B0E9493
:1081A0006CF2209118023091190240911A025091FC
:1081B0001B020E94CBF22AE037ED43E25CE30E940F
:1081C000CBF20E9474C20E9466C54CCF0E94DDC3F0
:1081D000AB01BC014093480D5093490D60934A0D8B
:1081E00070934B0D87E99CE00E94DE793BCF802F96
:1081F0000E94C3926E2D802F0E94A29EF12CB70187
:10820000802F0E94D19E0630110529F4F092980427
:10821000E092970427CF0830110509F023CFF092A0
:108220009604E09295041ECF0E94EDC3853620F09F
:1082300084E68093940416CF8093940413CF0E9415
:108240000DC40E94E3F76739710514F066E970E028
:1082500070938D0460938C040E9407E460918C04F9
:1082600070918D04072E000C880B990B0E946CF204
:1082700020918204309183044091840450918504BC
:108280000E9466F287FF04C060E082E996E003C0C6
:1082900060E085E896E00E941EC681E080931502AA
:1082A0008091A104809386042F961CAE1DAE1EAE55
:1082B0001FAE2F9767961CAE1DAE1EAE1FAE679702
:1082C00028961FAE289768961FAE68974CE36C9669
:1082D0004FAF6C975CE1A0965FAFA09786E4A49641
:1082E0008FAFA497C12CD12CB0E8EB2E1FEBF12E51
:1082F000812C912C540160918C0470918D04072E77
:10830000000C880B990B0E946CF2162F072F782E09
:10831000692E262F372F482F592FB601C7010E94EB
:1083200066F2882331F120918204309183044091D8
:10833000840450918504612F702F872D962D0E9403
:1083400066F2881F8827881F28968FAF2897609627
:108350009FAD6097992389F0882379F08091150269
:10836000882309F47FCE60E087E796E00E941EC66E
:1083700079CE1C2D0D2D7E2C6F2C0E94D09F6B0171
:108380007C01DC01CB0167962CAD3DAD4EAD5FAD00
:108390006797821B930BA40BB50BB7FD3DC0D701AC
:1083A000C60188519C4FAF4FBF4F67968CAF9DAFB2
:1083B000AEAFBFAF67970E9484E3E1E8F6E0849137
:1083C0002F019FEF491A590A882321F00E948584C2
:1083D000F201F5CF81149104A104B104B9F0D501E3
:1083E000C40188519C4FAF4FBF4FBC01CD016C19E8
:1083F0007D098E099F0928EE33E040E050E00E949D
:1084000041F6CA01B9010E94279103C08FE30E947F
:1084100085848AE00E94858480E00E9469670E94CA
:108420007FA3209082043090830440908404509075
:1084300085049101A201612F702F872D962D0E9436
:108440009EF69F7720E030E040EA50E481149104EA
:10845000A104B10429F40E9466F287FF07C004C09A
:108460000E94C5F8181614F4460157012896AFADBE
:108470002897AA2309F443C02F962CAD3DAD4EADED
:108480005FAD2F97211531054105510541F0D70109
:10849000C601821B930BA40BB50BB7FD30C0910135
:1084A000A20168966FAD68976C967FAD6C97A096A9
:1084B0008FADA097A4969FADA4970E949EF620E052
:1084C00030E040EC5FE30E9466F287FD47CFD701C2
:1084D000C601805A9541AF4FBF4F2F968CAF9DAFCD
:1084E000AEAFBFAF2F9768962FAE68976C963FAE32
:1084F0006C97A0964FAEA097A4965FAEA49780917C
:108500001502882309F42ACF81149104A104B1042F
:1085100029F4C12ED02EE72CF62CEDCE98EEC91AF8
:1085200093E0D90AE108F108C818D908EA08FB085D
:10853000F7FE14CFEECF0E94E64B88E50E9440C4C0
:10854000882319F0179A1092191589E50E9440C4E2
:10855000882319F0169A10921A158AE50E9440C4D1
:10856000882319F0159A10921B1585E40E9440C4C7
:10857000882309F477CD0E94676774CD0E94E64B8B
:108580000E9444696FCDA9964EAD5FADA997452B6A
:1085900009F46FC1CF56DF4F288139814A815B8151
:1085A000C159D040280F391F4A1F5B1FA7962CAF17
:1085B0003DAF4EAF5FAFA797CF56DF4F28813981D0
:1085C0004A815B81C159D040281B390B4A0B5B0B98
:1085D000CA01B90163962CAD3DAD4EAD5FAD639759
:1085E0000E9432F6A7962CAD3DAD4EAD5FADA7977C
:1085F0000E9463F6420E531E641E751E34E143163C
:108600005104610471040CF487C1C455DF4F8881A3
:108610009981AA81BB81CC5AD040481659066A0676
:108620007B060CF089C1CC54DF4F288139814A8107
:108630005B81C45BD04024153505460557059CF485
:10864000C854DF4F88819981AA81BB81C85BD04023
:1086500084199509A609B70963968CAF9DAFAEAF93
:10866000BFAF639706C063964CAE5DAE6EAE7FAE95
:108670006397B301A2018FEE93E00E94E0A363969B
:108680004CAD5DAD6EAD7FAD63978AEE93E00E9419
:10869000E0A3E8964FADE897EC965FADEC97E096D7
:1086A0006FADE097E4967FADE49783EE93E00E9490
:1086B000C3A3C158DF4F4881CF57D040C058DF4FC8
:1086C0005881C058D040CF57DF4F6881C158D04043
:1086D000CE57DF4F7881C258D0408CED93E00E9496
:1086E000C3A3A996AEADBFADA99713970CF4C1C0B3
:1086F00063966CAD7DAD8EAD9FAD63970E946CF2BD
:1087000020E030E040E850E40E94CBF26B017C01B5
:10871000E8962FADE897EC963FADEC97E0964FAD1D
:10872000E097E4965FADE497C158DF4F6881CF577B
:10873000D040C058DF4F7881C058D040CF57DF4F6E
:108740008881C158D040CE57DF4F9881C258D04061
:108750000E949EF62BED3FE049E450E40E94CBF2EC
:1087600020E030E040E05FE30E94CBF29B01AC01EF
:10877000C701B6010E947BF76B017C01A7966CAD27
:108780007DAD8EAD9FADA7970E946CF22FE632E1D2
:1087900043E85AE30E94CBF24B015C01B701A6010A
:1087A00086ED93E00E94C3A3B501A40180ED93E0A0
:1087B0000E94C3A32AE939E949E15FE3C701B60191
:1087C0000E94CBF26B017C019B01AC010E949FF6E1
:1087D000A50194010E947BF7AF966CAF7DAF8EAF81
:1087E0009FAFAF97A5019401C701B6010E94CBF2DC
:1087F00020E030E040E05EE30E94CBF24B015C0100
:10880000E0ECF3E084919F012F5F3F4F8823C1F09C
:10881000C454DF4F2883CC5BD040C354DF4F388330
:10882000CD5BD0400E948584C454DF4F2881CC5B4F
:10883000D040C354DF4F3881CD5BD040F901E2CF47
:10884000B701A6018AEB93E00E94C3A3AF964CAD9B
:108850005DAD6EAD7FADAF9784EB93E00E94C3A397
:10886000B501A4018EEA93E00E94C3A38AE00E94AE
:10887000858463968CAD9DADAEADBFAD6397840D21
:10888000951DA61DB71D2896EFAD2897B595A79500
:1088900097958795E7FF03C080930C0407C0C655E2
:1088A000DF4FE881F981CA5AD0408083A9962EAD66
:1088B0003FADA9972F5F3F4FA9963FAF2EAFA99726
:1088C00064963FAD6497E8963FAFE89768964FADE2
:1088D0006897EC964FAFEC976C965FAD6C97E0960F
:1088E0005FAFE097A0968FADA097E4968FAFE49727
:1088F0002F962CAD3DAD4EAD5FAD2F97A7962CAF0B
:108900003DAF4EAF5FAFA79731E0C557DF4F38831C
:10891000CB58D0400C948F3B84E1482E512C612CD5
:10892000712C24E130E040E050E063962CAF3DAF85
:108930004EAF5FAF63979DCEC055DF4F48805980E3
:108940006A807B80C05BD0407BCECF53DF4F0FB6B9
:10895000F894DEBF0FBECDBFDF91CF911F910F9175
:10896000FF90EF90DF90CF90BF90AF909F908F904F
:108970007F906F905F904F903F902F900895AF92AF
:10898000BF92CF92DF92EF92FF920F931F93CF93FC
:10899000DF931F92CDB7DEB77C016B018A015901CD
:1089A00080918614811119C0F701808191810E9404
:1089B0001CF68983F60181936F01BE016F5F7F4FC3
:1089C000C5010E94D2ECF701408151814F5F5F4F9A
:1089D000518340830150110939F70F90DF91CF91F6
:1089E0001F910F91FF90EF90DF90CF90BF90AF90CD
:1089F00008958F929F92AF92BF92CF92DF92EF92A3
:108A0000FF920F931F93CF93DF931F921F92CDB7C7
:108A1000DEB7E0918614E1114AC059016C018B0167
:108A20007B01E40EF51E0E151F0509F440C0F6018A
:108A300080809180F80161918F016983C4016A830C
:108A40000E941CF66A81681729F1C4010E9424F66D
:108A5000C4010E941CF699818917E1F0E8EDF6E166
:108A600084918F010F5F1F4F882321F00E9485841E
:108A7000F801F6CFE6E5F8E084918F010F5F1F4F14
:108A8000882321F00E948584F801F6CF81E080934D
:108A900086140DC0BE016F5F7F4FC5010E94D2ECEE
:108AA000F60180819181019691838083BCCF0F90E4
:108AB0000F90DF91CF911F910F91FF90EF90DF907A
:108AC000CF90BF90AF909F908F900895CF93DF93FA
:108AD000CDB7DEB72C970FB6F894DEBF0FBECDBF73
:108AE0008091F9149091FA14A091FB14B091FC14A8
:108AF00089839A83AB83BC838091FD149091FE148B
:108B0000A091FF14B09100158D839E83AF83B88729
:108B10008091011590910215A0910315B091041553
:108B200089879A87AB87BC870E94E1BE0E94208418
:108B300080E00E9499C281E00E9499C282E00E9476
:108B400099C20E940EC04CE050E069EF74E1CE0182
:108B500001960E949AF9892B51F02C960FB6F89441
:108B6000DEBF0FBECDBFDF91CF910C9452592C9632
:108B70000FB6F894DEBF0FBECDBFDF91CF91089541
:108B800061E0FC0180810C94A29E8EBD0DB407FEB5
:108B9000FDCF08958FEF8EBD0DB407FEFDCF8EB5CE
:108BA00008950F931F93CF93DF938B010E94D09F63
:108BB000EB01F0DF8F3F49F00E94D09F6C1B7D0BD3
:108BC00060177107B0F380E001C081E0DF91CF91C1
:108BD0001F910F910895CF92DF92EF92FF921F9312
:108BE000CF93DF9300D01F92CDB7DEB76C01162F65
:108BF000FC019281892F806A86958CBD90FD03C00F
:108C000081E0963009F480E08DBD60E0F60180815E
:108C100029833A834B835C830E94A29E6CE271E0BD
:108C2000C601BFDF812F8064B0DF88E1E82EF12C20
:108C30005C814B813A812981DA01C9010E2C04C083
:108C4000B695A795979587950A94D2F729833A8385
:108C50004B835C839ADFF8E0EF1AF10829813A81AF
:108C60004B815C8188EFE8168FEFF80629F7112316
:108C700021F0183021F08FEF03C085E901C087E8AB
:108C800084DF1C3009F486DF10E084DFF601838383
:108C900087FF04C01F3F11F01F5FF7CF0F900F90A9
:108CA0000F900F90DF91CF911F91FF90EF90DF9089
:108CB000CF9008950F931F93CF93DF93EC01890119
:108CC0008C81833039F089E0440F551F661F771F70
:108CD0008A95D1F79A01AB0168E1CE017CDF882348
:108CE00011F086E02FC08EEF8EBD80E090E00DB4D5
:108CF00007FEFDCFF801E80FF91F20812EBD0DB44E
:108D000007FEFDCF21812EBD0296811522E092073C
:108D100071F70DB407FEFDCF8FEF37DF8FEF35DF33
:108D200039DF8B838F71853029F083E18983CE0110
:108D300027DF09C068E572E0CE0133DF182F81110B
:108D400006C087E18983CE011BDF10E00FC020E061
:108D500030E0A9016DE0CE013EDF811103C01ADFD2
:108D6000882311F086E1EECFCE010ADF812FDF915B
:108D7000CF911F910F910895EF92FF920F931F9340
:108D8000CF93DF93EC0179018C81833039F089E056
:108D9000440F551F661F771F8A95D1F79A01AB01C3
:108DA00061E1CE0118DF882329F084E08983CE01B8
:108DB000E7DE35C00E94D09F8B01ECDE8B838F3FB6
:108DC00049F40E94D09F601B710B6D327140A8F373
:108DD00081E103C08E3F39F08FE08983CE01D0DE80
:108DE0008FEFD3DE1CC08FEF8EBDF701D701A150EE
:108DF000BE4F0DB407FEFDCF9EB591938EBDEA1711
:108E0000FB07B9F70DB407FEFDCF8EB58C93C2DE1C
:108E1000C1DECE01B5DE8FEFB8DE81E001C080E0BB
:108E2000DF91CF911F910F91FF90EF9008958F9256
:108E30009F92AF92BF92CF92DF92EF92FF92CF9329
:108E4000FC01C080D180E280F38020E030E0A90105
:108E5000C701B6010E9466F287FF08C0C701B601CC
:108E6000905820E030E048EC52E406C020E030E0CA
:108E700048EC52E4C701B6010E94CBF20E94E3F72E
:108E80006B017C01603AF6E87F07F1E08F079105FE
:108E900084F020EA36E841E050E00E9463F6CA011F
:108EA000B9012AE030E040E050E00E9463F6605DE6
:108EB00001C060E26093C30480E1C81687E2D8066F
:108EC000E104F10494F0C701B60120E137E240E08B
:108ED00050E00E9463F6CA01B9012AE030E040E0A8
:108EE00050E00E9463F6605D01C060E26093C404DC
:108EF000E8EECE16E3E0DE06E104F10494F0C701EB
:108F0000B60128EE33E040E050E00E9463F6CA016B
:108F1000B9012AE030E040E050E00E9463F6605D75
:108F200001C060E26093C504C701B60124E630E0E9
:108F300040E050E00E9463F68AE0882E912CA12C3C
:108F4000B12CCA01B901A50194010E9463F6605DCC
:108F50006093C6048EE28093C704C701B601A501E1
:108F600094010E9463F6C62FCA01B901A5019401BC
:108F70000E9463F6605D6093C804C05DC093C9043D
:108F800083EC94E0CF91FF90EF90DF90CF90BF9073
:108F9000AF909F908F9008958F929F92AF92BF92C3
:108FA000CF92DF92EF92FF92CF9320E030E048EC37
:108FB00052E4FC0160817181828193810E94CBF235
:108FC0000E94E3F76B017C0197FF0AC0F094E094E4
:108FD000D094C094C11CD11CE11CF11C8DE201C0D5
:108FE0008BE28093C304C701B60120E137E240E081
:108FF00050E00E9463F68AE0882E912CA12CB12CBF
:10900000CA01B901A50194010E9463F6605D6093F5
:10901000C404C701B60128EE33E040E050E00E94EE
:1090200063F6CA01B901A50194010E9463F6605D6F
:109030006093C504C701B60124E630E040E050E08B
:109040000E9463F6CA01B901A50194010E9463F66A
:10905000605D6093C6048EE28093C704C701B601C9
:10906000A50194010E9463F6C62FCA01B901A501AA
:1090700094010E9463F6605D6093C804C05DC09374
:10908000C90483EC94E0CF91FF90EF90DF90CF90F4
:10909000BF90AF909F908F9008958F929F92AF92C4
:1090A000BF92CF92DF92EF92FF92FC01C080D180FD
:1090B000E280F38020E030E0A901C701B6010E9400
:1090C00066F287FF04C0C701B601905802C0C7010D
:1090D000B6010E94E3F76B017C016031F7E27F0784
:1090E0008105910584F020E137E240E050E00E94E4
:1090F00063F6CA01B9012AE030E040E050E00E9486
:1091000063F6605D01C060E26093C50488EEC81636
:1091100083E0D806E104F10494F0C701B60128EE1B
:1091200033E040E050E00E9463F6CA01B9012AE052
:1091300030E040E050E00E9463F6605D01C060E214
:109140006093C604E4E6CE16D104E104F10494F081
:10915000C701B60124E630E040E050E00E9463F62B
:10916000CA01B9012AE030E040E050E00E9463F615
:10917000605D01C060E26093C704FAE0CF16D104DD
:10918000E104F1049CF08AE0882E912CA12CB12CF2
:10919000C701B601A50194010E9463F6CA01B90195
:1091A000A50194010E9463F6605D01C060E26093D6
:1091B000C804C701B6012AE030E040E050E00E9458
:1091C00063F6605D6093C90485EC94E0FF90EF90D6
:1091D000DF90CF90BF90AF909F908F90089520E048
:1091E00030E040E251E4FC01608171818281938131
:1091F0000E94CBF20E94E3F79B0177FF06C0222773
:109200003327261B370B8DE201C08BE28093C40409
:10921000C90168EE73E00E9477F9CB01EAE0F0E063
:10922000BF010E9477F9805D8093C504C90164E69F
:1092300070E00E9477F9CB01BF010E9477F9805D51
:109240008093C604C901BF010E9477F9282FCB0182
:10925000BF010E9477F9805D8093C7048EE28093FE
:10926000C804205D2093C90484EC94E00895AC0107
:10927000952F991F9927991F29F022273327241BFF
:10928000350B01C09A01483E5340ACF0C90168EE6D
:1092900073E00E9477F9CB01EAE0F0E0BF010E94A1
:1092A00077F9805D8093C604C90164E670E00E948E
:1092B00077F9CB0112C024363105B4F0911102C008
:1092C00080E201C08DE28093C604C90164E670E0CB
:1092D0000E9477F9CB01EAE0F0E0BF010E9477F944
:1092E000805D8093C7040EC080E28093C6048093A3
:1092F000C7042A30310584F091118DE28093C704B0
:10930000EAE0F0E0C901BF010E9477F9CB01BF019B
:109310000E9477F9805D05C0911102C080E201C012
:109320008DE28093C804C9016AE070E00E9477F979
:10933000805D8093C90486EC94E008959C0197FDBC
:109340000EC08436910584F064E670E00E9477F9DF
:10935000CB016AE070E00E9477F9805D06C031952C
:10936000219531098DE201C080E28093C7042A3043
:10937000310564F0EAE0F0E0C901BF010E9477F92D
:10938000CB01BF010E9477F9805D01C080E280932C
:10939000C804C9016AE070E00E9477F9805D80939B
:1093A000C90487EC94E00895CF92DF92EF92FF9288
:1093B0006B017C0183E3C816D104E104F10470F071
:1093C00082E3C81AD108E108F10862E370E080E0A6
:1093D00090E00E94989F0E9474E7ECCFC701B6010D
:1093E0000E94989FFF90EF90DF90CF900C9474E7CD
:1093F000CF93DF93E8E4F8E08491EF01219688238E
:1094000021F00E948584FE01F7CFE4E4F8E0849126
:10941000EF012196882321F00E948584FE01F7CF79
:1094200062B36695617070E080E090E00E942791E1
:1094300062B3617070E080E090E00E9427918AE062
:109440000E948584E0E4F8E08491EF01219688236E
:1094500021F00E948584FE01F7CF60910601862FDE
:10946000660F990BAA0BBB0BBC01CD01662797FDBC
:1094700063957727882799270E94279162B362FB1B
:10948000662760F970E080E090E00E9427918AE012
:109490000E948584ECE3F8E08491EF012196882313
:1094A00021F00E948584FE01F7CF6091060166FBE2
:1094B000662760F970E080E090E00E94279160915B
:1094C000060165FB662760F970E080E090E00E948D
:1094D00027918AE00E948584E7E3F8E08491EF0118
:1094E0002196882321F00E948584FE01F7CF6091A8
:1094F000060163FB662760F970E080E090E00E945F
:109500002791609106016295617070E080E090E0C3
:109510000E9427918AE00E948584E2E3F8E084912A
:10952000EF012196882321F00E948584FE01F7CF68
:10953000609106016695617070E080E090E00E94A5
:1095400027916091060162FB662760F970E080E078
:1095500090E00E9427918AE0DF91CF910C9485845E
:1095600067FD5CC0823021F128F4882349F0813006
:1095700069F054C0833071F1843009F43DC04EC0AD
:10958000662311F0A19A8FC0A1988DC09FB7662362
:1095900029F0F89480910801806804C0F8948091C3
:1095A00008018F77809308019FBF47FF4CC07FC0A1
:1095B0009FB7662329F0F89480910801806404C065
:1095C000F894809108018F7B809308019FBF47FF2B
:1095D00040C06FC09FB7662329F0F89480910801BE
:1095E000886004C0F89480910801877F8093080107
:1095F0009FBF47FF3EC05AC09FB7662329F0F8942B
:1096000080910801826004C0F894809108018D7FE8
:10961000809308019FBF47FF39C04AC047FD49C03A
:109620008230B9F028F4882341F0813061F0089548
:109630008330F9F0843051F10895442311F0A09A59
:109640000895A0980895442311F0A29A0895A2982D
:1096500008959FB7442329F0F8948091080180620F
:1096600004C0F894809108018F7D809308019FBF0A
:1096700008959FB7442329F0F894809108018061F0
:10968000F4CFF894809108018F7EEFCF9FB74423E9
:1096900029F0F894809108018460E7CFF8948091D4
:1096A00008018B7FE2CF47FFC8CF08950895089542
:1096B00008950895643079F028F4613041F0623003
:1096C00041F00895683051F0603141F0089540E074
:1096D00003C040E004C041E060E002C041E061E05E
:1096E0003FCF5F988EBD00000DB407FEFDCF8EB555
:1096F0006EBD00000DB407FEFDCF8EB55F9A0895D4
:10970000CF93DF9300D01F921F92CDB7DEB795E0C5
:10971000E8E9F2E0DE01119601900D929A95E1F7E9
:10972000E1E0F0E0EC0FFD1FE80FF11D808190E01B
:109730000F900F900F900F900F90DF91CF91D1CF9E
:1097400024E08202C0011124FC01E751FB4E40815C
:10975000518162817381FC01E851FB4F4083518349
:1097600062837383E091BF04F091C004828993897E
:10977000A489B5898093BB049093BC04A093BD04D5
:10978000B093BE048FEF9FEF9093C2048093C10407
:109790000895CF93DF932FB7F89494E08902E00106
:1097A0001124FE01E751FB4E60817181828193811A
:1097B0002FBF0E946CF2C852DB4F288139814A8149
:1097C0005B810E94CBF2DF91CF9108950E9453C537
:1097D000882321F080E00E946967F8CF8091C1045E
:1097E0009091C204892BB1F70895BC0180E090E00C
:1097F0004AE00E94BF908DE00E9485848AE00C942C
:109800008584CF93DF931F92CDB7DEB7789484B56C
:10981000826084BD84B5816084BD85B5826085BD6C
:1098200085B5816085BD80916E00816080936E00FA
:1098300010928100809181008260809381008091EC
:10984000810081608093810080918000816080939D
:1098500080008091B10084608093B1008091B0005D
:1098600081608093B000809191008260809391002C
:10987000809191008160809391008091900081603F
:10988000809390008091A10082608093A1008091DC
:10989000A10081608093A1008091A00081608093ED
:1098A000A00080912101826080932101809121019B
:1098B000816080932101809120018160809320014B
:1098C00080917A00846080937A0080917A0082602F
:1098D00080937A0080917A00816080937A008091F1
:1098E0007A00806880937A001092C10082E08093B1
:1098F000C0001092C50087E08093C4008091C10031
:1099000080618093C1008091C10088608093C10014
:109910008091C10080688093C1008091C1008F7DDB
:109920008093C1001092CB04EBEEF9E084918F019B
:109930000F5F1F4F882321F00E948584F801F6CF26
:10994000E8EDF6E184918F010F5F1F4F882321F02E
:109950000E948584F801F6CF14B710FF0DC0E2EE27
:10996000F9E084917F019FEFE91AF90A882321F039
:109970000E948584F701F5CF11FF0DC0E1EDF9E0FC
:1099800084917F019FEFE91AF90A882321F00E9450
:109990008584F701F5CF12FF0DC0EFEBF9E084915C
:1099A0007F019FEFE91AF90A882321F00E9485843C
:1099B000F701F5CF13FF0DC0EEEAF9E084917F01C6
:1099C0009FEFE91AF90A882321F00E948584F701A4
:1099D000F5CF15FF0CC0EDE9F9E084918F010F5F21
:1099E0001F4F882321F00E948584F801F6CF14BE12
:1099F000E6E9F9E084918F010F5F1F4F882321F082
:109A00000E948584F801F6CF80E20E948584EFE809
:109A1000F9E084918F010F5F1F4F882321F00E948E
:109A20008584F801F6CF8AE00E948584E8EDF6E1AE
:109A300084918F010F5F1F4F882321F00E9485843E
:109A4000F801F6CFEFE7F9E084918F010F5F1F4F28
:109A5000882321F00E948584F801F6CFEBE6F9E037
:109A600084918F010F5F1F4F882321F00E9485840E
:109A7000F801F6CFE2E3F9E084918F010F5F1F4F09
:109A8000882321F00E948584F801F6CFE8EDF6E105
:109A900084918F010F5F1F4F882321F00E948584DE
:109AA000F801F6CFEBE1F9E084918F010F5F1F4FD2
:109AB000882321F00E948584F801F6CFE8EDF6E1D5
:109AC00084918F010F5F1F4F882321F00E948584AE
:109AD000F801F6CF80911F1590912015BE016F5FA0
:109AE0007F4F009719F0681B790B02C065527541D2
:109AF0008CE099E00E9407A460EF74E085EF98E0A5
:109B00000E9407A48AE00E94858481E08093D304A8
:109B10008093D4048093D5048093D6048093D70493
:109B20000E9475D08CE0EEEFF3E0A9EFB4E1019074
:109B30000D928A95E1F70E9454C3809101018064DF
:109B400080930101809101018061809301018091E6
:109B500001018860809301016D9A8091010180620A
:109B60008093010188E00E94C5ED80910101886029
:109B70008093010186E00E94C5ED6C9A82E00E940C
:109B8000C5ED87ED80937A0010927E0010927D00E3
:109B900080917E00816080937E0080917E00846051
:109BA00080937E0080E888BD80916E008460809301
:109BB0006E006AEF70E080E090E00E94989F85E080
:109BC00090E09093D1048093D00460E080912302D0
:109BD000909124020E942E8120E030E040EA50E47F
:109BE0000E9466F287FF0AC08091230290912402AE
:109BF00040979093240280932302E7CF81E391E082
:109C0000909326028093250260E08091CE0490918B
:109C1000CF040E942E8120E030E848E953E40E94FE
:109C2000C5F8181654F48091CE049091CF04409654
:109C30009093CF048093CE04E7CF8091210290913E
:109C400022020E94C2E420E030E040EA50E40E9498
:109C500066F287FF0AC0809121029091220240970C
:109C60009093220280932102E8CF8091CC049091BE
:109C7000CD040E94C2E420E030E046E153E40E94BB
:109C8000C5F8181654F48091CC049091CD044096F8
:109C90009093CD048093CC04E8CF98E288E10FB68E
:109CA000F894A895809360000FBE909360001FB752
:109CB000F8948091D204811124C0E1E9F7E1849104
:109CC000E7EDF7E19491E82FF0E0EE0FFF1FEE5B78
:109CD000F84EA591B491EC91E92321F461E085E37C
:109CE0000E94A29E85E30E94C3928CB580618CBDC8
:109CF0008CB580648CBD84E30E94C39283E30E9490
:109D0000C3928091D2048F5F8093D2041FBF579A71
:109D10001AE5E12E13E0F12E10E0F70161917F01C9
:109D200070E0812FEDDC1F5F1530B9F7999A989A92
:109D3000809107018068809307019A9A80910701BA
:109D400080648093070180910701806280930701FE
:109D500080910701886080930701809107018061ED
:109D600080930701809107018260809307018091B1
:109D70000701846080930701BFE5EB2EB3E0FB2E63
:109D800010E0F70161917F01812F94DC1F5F153096
:109D9000C1F780910A01826080930A0180910A01D3
:109DA000816080930A0180910A01846080930A0196
:109DB00080910A01806480930A0180910A01806881
:109DC00080930A010F9A179A0E9A169A0D9A159A6D
:109DD0000C9A149A0B9A139A26982E9A25982D9AD3
:109DE00024982C9A389A4098179A10921915399AF3
:109DF0004198169A10921A153A9A4298159A10920A
:109E00001B153B9A4398149A3C9A44988091800081
:109E10008C7F8093800080918100877E8860809312
:109E20008100809180008F738093800080918100F9
:109E3000887F82608093810080E090E49093890025
:109E400080938800109285001092840080916F00AA
:109E5000826080936F0081E08093970D78940E94D8
:109E600051B76C9A0E9409770E947DA220915C0DE7
:109E700030E07901F8E3EF1AF108F7FE04C0790148
:109E800087E3E81AF108F594E7942E5131093695E5
:109E90002795F22E0E94E49400E718E023E147E0C2
:109EA0006CE08E2D0E941A9384E00E94C3A2009160
:109EB0005C0D10E0025711091695079560915D0D34
:109EC000625140E453E08F2D0E94979360915D0DA5
:109ED000665046E453E0802F0E9497930E94E292DE
:109EE0008111DACF64EC79E080E090E05DDA40E661
:109EF000542E5DE0452E69E0C62E6AE0D62E70E055
:109F0000A72E70E0B72E2AE0722E30E2632E8091E9
:109F1000D606853010F40E943DC68091500D8823EE
:109F2000E9F00E94D09F00914C0D10914D0D2091B1
:109F30004E0D30914F0DDC01CB01801B910BA20B1C
:109F4000B30BB7FD0BC01092500D8091A60A811182
:109F500012C16AD68091A60A81110DC18091D606E0
:109F6000882309F498C08091A30A882309F480C04B
:109F70000091D506509E800111240B501B4F6CE4BC
:109F80007AE0C8010E94E5F1892BF9F087E99CE0AD
:109F90000E94687C87E99CE00E941C7E1092A40AC3
:109FA0001092A30AE9E3FAE084918F010F5F1F4F3B
:109FB000882341F00E948584F801F6CF8091A40A9D
:109FC000811156C00E94A26955C0F801019000207D
:109FD000E9F731977F01E01AF10A1092970C6EE4CD
:109FE00070E0C8010E94CEF94C01009729F4F701F6
:109FF0003197E00FF11F0EC060E270E00E94CEF9D1
:10A000008C010F5F1F4F6AE270E0C4010E94CEF91D
:10A01000FC013197418272821382F8010190002085
:10A02000E9F73197AF01401B510BB80187E99CE07C
:10A030000E949A7C8091970C882309F4BFCFE5EBAE
:10A04000FBE084918F010F5F1F4F882321F00E9456
:10A050008584F801F6CFE2EFF9E084918F010F5F7C
:10A060001F4F882309F4AACF0E948584F801F5CFF9
:10A070000E943A6A8091D606882369F081508093C5
:10A08000D6068091D5068F5F853018F48093D5066B
:10A0900002C01092D5068091F404882309F461C0AF
:10A0A000E8EDF6E184918F010F5F1F4F882321F0C7
:10A0B0000E948584F801F6CFEAE2FAE084918F01EC
:10A0C0000F5F1F4F882321F00E948584F801F6CF8F
:10A0D0008091F40480FD51C08091F40484FD4DC052
:10A0E00090E2F92E8091F40481FD64C08091F40423
:10A0F00085FD60C000E28091F40482FD77C080910C
:10A10000F40486FD73C010E28AE00E9485841F92E9
:10A110006F921F921F931F920F931F92FF92DF92D5
:10A12000CF921F920E94BA941092F4040FB6F89442
:10A13000DEBF0FBECDBF8091FD03882391F010924A
:10A14000A50A87E99CE00E94687C87E99CE00E9460
:10A150001C7E1092A40A1092A30A0E94876C0E948F
:10A160009DE480E00E946967A114B10409F4CFCE98
:10A170000E940000C8CEA7D4F1CE6091E80470918F
:10A18000E9048091EA049091EB040E946CF2209122
:10A19000D8043091D9044091DA045091DB040E9434
:10A1A000CBF2AB01BC0186E29AE00E94C3A388E532
:10A1B000F82E98CF6091EC047091ED048091EE043C
:10A1C0009091EF040E946CF22091DC043091DD0448
:10A1D0004091DE045091DF040E94CBF2AB01BC0140
:10A1E00082E29AE00E94C3A309E585CF6091F00462
:10A1F0007091F1048091F2049091F3040E946CF24A
:10A200002091E0043091E1044091E2045091E30494
:10A210000E94CBF2AB01BC018EE19AE00E94C3A385
:10A220001AE572CF4F925F926F927F928F929F92B8
:10A23000AF92BF92FF920F931F93CF93DF93182F8C
:10A2400080E79CE09093F8088093F70810928C0CBC
:10A2500082E090E0A0E0B0E08093750C9093760CE3
:10A26000A093770CB093780C1092F6081092F20835
:10A270001092F3081092F4081092F5088FEF9FEFF8
:10A28000DC018093EE089093EF08A093F008B09360
:10A29000F108112379F1153008F0F9C040E060E0D1
:10A2A00070E0CB010E941FC9882309F4F0C020E1AF
:10A2B000129FC00111248252994FFC01E254FE4FBB
:10A2C00020812F7709F0E3C03C9640815181628163
:10A2D0007381443651056105710508F4D8C034977F
:10A2E00080809180A280B38081149104A104B10484
:10A2F00021F4CDC0812C912C540140E0C501B40162
:10A300000E941FC9F82E882309F4C1C08091F90664
:10A310009091FA068115924009F0B9C0A091FE060D
:10A32000AA2309F4B4C06091FC067091FD06611582
:10A33000710509F4ACC02091FB06222309F4A7C0E3
:10A34000A093870C2093790C80E030E0E1E0F0E00E
:10A35000C82FAF01082E02C0440F551F0A94E2F720
:10A360002417350741F0982F8F5F983089F789E0DF
:10A370008093820C8CC08093820C209104073091D2
:10A3800005072115310519F040E050E008C0209183
:10A39000120730911307409114075091150720932D
:10A3A0007A0C30937B0C40937C0C50937D0C2401F1
:10A3B0003501460E571E611C711C4092880C50924C
:10A3C000890C60928A0C70928B0CE091FF06F091E0
:10A3D0000007F0938E0CE0938D0CB0E00E947FF6A6
:10A3E000460E571E681E791E40928F0C5092900C9C
:10A3F0006092910C7092920C85E0EE0FFF1F8A958F
:10A40000E1F7E150FE4FEF2FFF27E6954E0E5F1E5E
:10A41000611C711C4092830C5092840C6092850CDC
:10A420007092860C209101073091020721153105A9
:10A4300021F0890120E030E008C000910E07109162
:10A440000F072091100730911107B501A40144199D
:10A45000550966097709400F511F621F731F04C019
:10A460007695679557954795CA95D2F740937E0C98
:10A4700050937F0C6093800C7093810C453F2FE0CC
:10A4800052076105710528F48CE080938C0CF12C47
:10A490001AC0453F5F4F6105710510F480E111C09E
:10A4A00080911A0790911B07A0911C07B0911D077E
:10A4B00080938F0C9093900CA093910CB093920C7E
:10A4C00080E280938C0C8F2DDF91CF911F910F91A3
:10A4D000FF90BF90AF909F908F907F906F905F9014
:10A4E0004F900895EF92FF920F931F93CF93DF93B6
:10A4F000CDB7DEB76F970FB6F894DEBF0FBECDBFF6
:10A500007B0108E11BE02AE13BE0F8013183208375
:10A5100022E02093510D90933E0A80933D0A40E043
:10A5200050E0BA018EE19BE00E94DE79F801808163
:10A5300091812BE1FC013496DE01159601900D927C
:10A540002A95E1F7FC01828193819C838B838BE8C0
:10A5500093E09A838983A701BE016F5F7F4F8BEEE3
:10A5600093E00E94D996CE0101960E9456AF6F9655
:10A570000FB6F894DEBF0FBECDBFDF91CF911F9114
:10A580000F91FF90EF9008951092A50A80919A0C78
:10A59000882321F087E99CE00C941C7E08956F923B
:10A5A0007F928F929F92AF92BF92DF92EF92FF9233
:10A5B0000F931F93CF93DF93CDB7DEB7AE970FB650
:10A5C000F894DEBF0FBECDBF2091A60A222309F466
:10A5D00006C2D62E7C0180919A0C882309F4A5C06E
:10A5E000442309F4CFC18091B20C882329F1E5EB13
:10A5F000FBE084918F010F5F1F4F882321F00E94A1
:10A600008584F801F6CFE2E7FBE084918F010F5FCC
:10A610001F4F882321F00E948584F801F6CF61E066
:10A6200070E080E090E00E9427918AE00E9485849B
:10A6300089E69BE00E945EAF88EB9CE09EA78DA719
:10A640008FE28093B70C81E0898310E00FE1809165
:10A650006F0C181778F4019FC0011124AE014F5FF1
:10A660005F4FBE01635D7F4F875C944F0E949BBE2E
:10A670001F5FEDCF898187FD0FC0AE014F5F5F4F38
:10A68000BE01635D7F4F83E99CE00E949BBE8DA568
:10A690009EA501979EA78DA7EDA5FEA51082E0912E
:10A6A000B20C84E0E89FF0011124ED54F34F809147
:10A6B000480D9091490DA0914A0DB0914B0D8083AA
:10A6C0009183A283B383E8EDF6E184918F010F5F5C
:10A6D0001F4F882321F00E948584F801F6CFB7012F
:10A6E00080E59BE00E9420A46091B20C9DE8699FE8
:10A6F000B00111246954734F85E49BE00E9420A4AB
:10A700004091480D5091490D60914A0D70914B0D4B
:10A710008FE39BE00E9489A38AE00E948584809158
:10A72000B20C8F5F8093B20C27C04423C1F0E8EDD8
:10A73000F6E184918F010F5F1F4F882321F00E9463
:10A740008584F801F6CFEFE2FBE084918F010F5F83
:10A750001F4F882389F00E948584F801F6CF10925C
:10A76000B20C82E0B82E10C1B70186E19BE00E94D6
:10A7700020A48AE00E94858407DF1D8218861C823F
:10A780001B828BE893E09A83898389EF9AE0909308
:10A79000190B8093180BF70180818F3209F05CC090
:10A7A00087010F5F1F4FCE0101964C010115110566
:10A7B00009F458C06FE270E0C8010E94CEF95C0154
:10A7C000009709F450C00817190708F04CC03C0165
:10A7D000601A710AA301B801CE0180960E94EEF9B9
:10A7E000E0E2F0E0EC0FFD1FE60DF71D1082609136
:10A7F000180B7091190B6115710511F06C5F7F4F8B
:10A8000021E0AE01405E5F4FCE0105960E940D80B3
:10A8100081111AC0E2E0FBE084918F010F5F1F4FAE
:10A82000811104C08E01005E1F4F04C00E94858408
:10A83000F801F2CFF80181918F01882319F00E946D
:10A840008584F8CF8EE287C09092190B8092180B06
:10A8500085010F5F1F4FAACF8AE19BE09093190BF0
:10A860008093180B87019091180B8091190B692F19
:10A87000782FDD2009F459C06115710511F06C5F66
:10A880007F4F21E0A80187E99CE00E940D8088238A
:10A8900009F447C08091A80C9091A90CA091AA0C32
:10A8A000B091AB0C8093440D9093450DA093460D51
:10A8B000B093470D1092480D1092490D10924A0D19
:10A8C00010924B0DB80184EF9AE00E9420A44091B1
:10A8D000440D5091450D6091460D7091470D8CEEE1
:10A8E0009AE00E9489A38AE00E948584EDEDFAE057
:10A8F00084917F019FEFE91AF90A882321F00E94D1
:10A900008584F701F5CFB80180E090E0EBDD809120
:10A91000B50A882319F085EB9AE001C0C80160E010
:10A920002AC0B80189EC9AE010C06115710511F0D8
:10A930006C5F7F4F26E5A80187E99CE00E940D80AF
:10A9400081110CC0B80185EB9AE00E9420A48EE230
:10A950000E9485848AE00E9485840FC081E08093F4
:10A96000A30AB70183EA9AE00E9420A48AE00E9429
:10A97000858460E0C8010E94BCC8CE0101960E9497
:10A9800056AF2DC0BB24B394E8EDF6E184918F015E
:10A990000F5F1F4F882321F00E948584F801F6CFB6
:10A9A000EAE2FBE084918F010F5F1F4F882321F0C3
:10A9B0000E948584F801F6CFE1E0BE1619F0E4E2CA
:10A9C000FBE002C0EEE1FBE084918F010F5F1F4FBF
:10A9D000882309F4C9CE0E948584F801F5CFAE968C
:10A9E0000FB6F894DEBF0FBECDBFDF91CF911F91A0
:10A9F0000F91FF90EF90DF90BF90AF909F908F905E
:10AA00007F906F900895CF92DF92EF92FF920F9315
:10AA10001F93CF93DF93CDB7DEB7EDB6FEB6DC0163
:10AA20000D900020E9F79D01281B390B2C5F3F4F4B
:10AA30004DB75EB7421B530B0FB6F8945EBF0FBE07
:10AA40004DBF0DB71EB70F5F1F4F9F938F938CE9BC
:10AA50009AE09F938F931F930F930E94FFF16801D9
:10AA600054E0C50ED11C0F900F900F900F900F90D7
:10AA70000F90F6018081882339F090E00E9492F9CE
:10AA8000F60181936F01F5CF60E0C8010E94D9C241
:10AA9000882319F0C8010E94F7AC88E99AE09093E6
:10AAA000FA088093F9080E94F5C20FB6F894FEBE2A
:10AAB0000FBEEDBEDF91CF911F910F91FF90EF90F0
:10AAC000DF90CF900895AF92BF92CF92DF92EF9236
:10AAD000FF920F931F93CF93DF93CDB7DEB7AA9763
:10AAE0000FB6F894DEBF0FBECDBF8091F80A8F93EA
:10AAF0008091F70A8F938FE89AE09F938F937E015E
:10AB000081E2E80EF11CFF92EF920E94FFF10F909C
:10AB10000F900F900F900F900F9010E0F7010190A1
:10AB20000020E9F73197EE19FF091E1774F4670149
:10AB3000C10ED11C17FDDA94F601808190E00E94CD
:10AB400092F9F60180831F5FE9CF40E050E0BA013F
:10AB50008DEF9AE00E94DE7900E0CE0101966C0153
:10AB60008091000B823028F4011114C08FEF9FEF09
:10AB700016C08091050B9091060BA091070BB09128
:10AB8000080B8F719927AA27BB27892B8A2B8B2B20
:10AB900059F71AC08091F70A9091F80A019690939C
:10ABA000F80A8093F70AAA960FB6F894DEBF0FBE94
:10ABB000CDBFDF91CF911F910F91FF90EF90DF906C
:10ABC000CF90BF90AF90089540E050E0B6018DEF78
:10ABD0009AE00E94987B18163CF6F601019000203E
:10ABE000E9F731971E2F1C19115068F05601A10E7C
:10ABF000B11C17FDBA94F501808190E00E9492F992
:10AC0000F5018083F1CF8A858E3709F4A9CF45E01D
:10AC100050E0B701C6010E94E0F9892B09F0A0CFEE
:10AC2000C701F1DE01E09CCFCF92DF92EF92FF925D
:10AC30001F93CF93DF931092A60A8091000B882375
:10AC400021F08DEF9AE00E941C7E1092740C1092FD
:10AC5000710C85E38093700C0E94D09FEB01A89546
:10AC60008091700C0E94C39280E79CE00E94C045D6
:10AC70002398229A219A209A289A85E08093720C30
:10AC800082E58CBD1DBC1AE08FEF0E94C5451150B6
:10AC9000D9F720E030E0A90160E080E79CE00E9465
:10ACA000EB45182F8093730C813049F00E94D09FA0
:10ACB0006C1B7D0B613D774060F381E054C02AEA54
:10ACC00031E040E050E068E080E79CE00E94EB4526
:10ACD00082FF03C01093740C0EC014E00E94CA459A
:10ACE0008093730C1150D1F78A3A11F082E03BC087
:10ACF00082E08093740C8091740C823021F0C12C1E
:10AD0000D12C760105C0C12CD12CE12C80E4F82E89
:10AD100020E030E0A90167E380E79CE00E94EB457A
:10AD2000A701960169E280E79CE00E94EB458093D1
:10AD3000730C882349F00E94D09F6C1B7D0B613DF2
:10AD4000774030F38AE00FC08091740C823011F5A7
:10AD500020E030E0A9016AE380E79CE00E94EB4537
:10AD6000882351F088E08093710C80E79CE00E947A
:10AD7000C045E8EDF6E119C00E94CA45807C803CE0
:10AD800019F483E08093740C0E94CA450E94CA455E
:10AD90000E94CA4580E79CE00E94C0451092720C58
:10ADA00081E040DA811131C015C08491EF01219614
:10ADB000882321F00E948584FE01F7CFE1E8FAE0C4
:10ADC0008491EF012196882309F456C00E9485845E
:10ADD000FE01F6CF80E026DA811117C0E5EBFBE03B
:10ADE0008491EF012196882321F00E948584FE0141
:10ADF000F7CFEDE6FAE08491EF012196882309F47C
:10AE00003BC00E948584FE01F6CF65E77CE08DEFB4
:10AE10009AE00E94F97B811116C0E5EBFBE084917A
:10AE2000EF012196882321F00E948584FE01F7CF4F
:10AE3000ECE5FAE08491EF0121968823E9F00E9485
:10AE40008584FE01F7CF81E08093A60AE8EDF6E164
:10AE50008491EF012196882321F00E948584FE01D0
:10AE6000F7CFE0E5FAE08491EF012196882321F005
:10AE70000E948584FE01F7CF8BE1EDEFFAE0AEE1B1
:10AE8000BBE001900D928A95E1F78091FB0A9091C9
:10AE9000FC0A90931D0B80931C0B8AE19BE090931E
:10AEA000190B8093180BDF91CF911F91FF90EF90BA
:10AEB000DF90CF900895EF92FF921F93CF93DF938F
:10AEC0001F92CDB7DEB7182FE5EBFBE084917F0131
:10AED0002FEFE21AF20A882331F099830E948584C9
:10AEE000F7019981F3CFE12FF92F84917F019FEF33
:10AEF000E91AF90A882321F00E948584F701F5CF29
:10AF00006091EA067091EB068091EC069091ED0657
:10AF10000E9427918AE00E9485840E94106A109204
:10AF2000E9061092E8060F90DF91CF911F91FF90F4
:10AF3000EF9008950F931F93CF93DF938C01EB0154
:10AF40009091840A2091850A921307C088E79AE0BD
:10AF50000E9412A20E9474E7F3CFF801A081B18190
:10AF6000488159818091830A34E0839FF001112444
:10AF7000E458F54FB387A287558744879F5F909326
:10AF8000840A8F5F821719F08093830A02C010929F
:10AF9000830ADF91CF911F910F910895EF92FF9255
:10AFA0000F931F93CF93DF931F92CDB7DEB78B0123
:10AFB000622F49830E94A5669091900D8091E706CB
:10AFC0004981891708F43FC09091920D8091E6065F
:10AFD000981708F438C0442399F120E030E0F801D4
:10AFE000E20FF31FE491EE2319F02F5F3F4FF7CFED
:10AFF00086E190E0821B930B97FD019695958795CE
:10B0000036E1F32E49EEE42EE80E8E2D8F0D87FDEE
:10B010000EC080E20E941894FA94F7CFF801849150
:10B02000882339F00E94DDA2F81A0F5F1F4F1F140A
:10B03000ACF31F1444F480E20E941894FA94F9CF00
:10B0400086E1F82EF4CF0F90DF91CF911F910F91F1
:10B05000FF90EF900895CF92DF92EF92FF920F93BF
:10B060001F93CF93DF9300D01F92CDB7DEB77C0143
:10B070008B0129833A834B835C830E94E06583E0E4
:10B0800080932A02F092E206E092E1061093E00635
:10B090000093DF0629813A814B815C81CA01B901A5
:10B0A0000E946AF22AE037ED43E25CE30E94CBF2B1
:10B0B0000E94E3F76093DB067093DC068093DD0665
:10B0C0009093DE060E946CF26B017C019B01AC0147
:10B0D00060E070E887E794E40E949EF60E94E3F740
:10B0E0006093D7067093D8068093D9069093DA06BA
:10B0F000F80160817181828193810E946AF22AE065
:10B1000037ED43E25CE30E94CBF2A70196010E9477
:10B110009EF60E94E8F760934D0A70934E0A809362
:10B120004F0A9093500A85E490E790932902809308
:10B1300028028CE893EB9093E5068093E406109246
:10B14000E3060F900F900F900F90DF91CF911F911A
:10B150000F91FF90EF90DF90CF900895AF92BF9244
:10B16000CF92DF92EF92FF920F931F93CF93DF93D3
:10B170007C01EB015A0169010E94E06523E0209304
:10B180002A02F092E206E092E106D093E006C09334
:10B19000DF06A501BB0C660B770B4093DB065093D3
:10B1A000DC066093DD067093DE06C601DD0CAA0B9B
:10B1B000BB0B841B950BA60BB70B8093D706909304
:10B1C000D806A093D906B093DA0688819981092E12
:10B1D000000CAA0BBB0B841B950BA60BB70B809323
:10B1E0004D0A90934E0AA0934F0AB093500A89E2F9
:10B1F00092E790932902809328021093E50600932A
:10B20000E4061092E306DF91CF911F910F91FF901A
:10B21000EF90DF90CF90BF90AF900895EF92FF92A4
:10B220000F931F93CF93DF931F92CDB7DEB7082FF5
:10B23000162FE6E7FCE084917F012FEFE21AF20A75
:10B24000882331F099830E948584F7019981F3CF97
:10B25000E02FF92F84917F019FEFE91AF90A8823E3
:10B2600021F00E948584F701F5CFE4E7FCE08491AA
:10B270007F012FEFE21AF20A882321F00E948584D1
:10B28000F701F5CF612F70E080E090E00E942791F8
:10B290008AE00F90DF91CF911F910F91FF90EF9077
:10B2A0000C9485844F925F926F927F928F929F92BF
:10B2B000AF92BF92CF92DF92EF92FF92CF93DF9344
:10B2C000E1E7FCE08491EF012196882321F00E94C0
:10B2D0008584FE01F7CF20912A0430912B04409100
:10B2E0002C0450912D046091F9147091FA148091FE
:10B2F000FB149091FC140E949FF642E00E94429140
:10B30000EDE6FCE08491EF012196882321F00E9474
:10B310008584FE01F7CF20912E0430912F044091B7
:10B320003004509131046091FD147091FE148091AD
:10B33000FF14909100150E949FF642E00E944291F6
:10B34000E9E6FCE08491EF012196882321F00E9438
:10B350008584FE01F7CF209132043091330440916F
:10B36000340450913504609101157091021580915B
:10B370000315909104150E949FF642E00E944291AD
:10B38000E5E6FCE08491EF012196882321F00E94FC
:10B390008584FE01F7CF60910515709106158091A7
:10B3A00007159091081542E00E9442918FB7F894DA
:10B3B0004090E9145090EA146090EB147090EC14F3
:10B3C0008090ED149090EE14A090EF14B090F014D3
:10B3D000C090F114D090F214E090F314F090F414B3
:10B3E0008FBFEBE5FCE08491EF012196882321F0EB
:10B3F0000E948584FE01F7CFC301B2010E9427910C
:10B40000E7E5FCE08491EF012196882321F00E947A
:10B410008584FE01F7CFC501B4010E942791E3E5C1
:10B42000FCE08491EF012196882321F00E9485841D
:10B43000FE01F7CFC701B6010E9427918AE0DF9194
:10B44000CF91FF90EF90DF90CF90BF90AF909F9003
:10B450008F907F906F905F904F900C948584CF93E6
:10B46000DF9383E50E946FC4882321F00E94DDC32F
:10B47000EB0102C0C0E0D0E0DD27C230D105BCF056
:10B48000E5EBFBE08491EF012196882321F00E94F7
:10B490008584FE01F7CFE1E3FCE08491EF01219682
:10B4A000882309F450C00E948584FE01F6CF88E409
:10B4B0000E946FC48823A9F00E94DDC3683771051C
:10B4C0003CF0633281E078072CF062E271E002C068
:10B4D00068E770E0FE01EE0FFF1FEF59FB4E71832E
:10B4E000608386E40E946FC48823A9F00E94DDC3B4
:10B4F000FE01EE0FFF1FE75AFB4E718360836F3F23
:10B50000710519F014F06FEF70E077FF02C060E092
:10B5100070E07183608382E40E946FC4882399F095
:10B520000E94DDC36530710534F0683871052CF078
:10B5300067E870E002C065E070E0CC0FDD1FC35A21
:10B54000DB4E79836883DF91CF9108952F923F92EC
:10B550004F925F926F927F928F929F92AF92BF9223
:10B56000CF92DF92EF92FF920F931F93CF93DF93CF
:10B57000CDB7DEB72E970FB6F894DEBF0FBECDBFA6
:10B580008DE690E00E940DC581117DC18091A204DD
:10B5900083FD79C183E50E946FC4482E811106C0E6
:10B5A00082E50E946FC4882309F46DC10E940DC416
:10B5B0000E94E3F770938F0460938E0480E00E94F2
:10B5C00052E460918E0470918F04072E000C880B5A
:10B5D000990B0E946CF2209190043091910440915B
:10B5E0009204509193040E94C5F818160CF046C1BD
:10B5F00084EE92E09F938F9385E29CE09F938F93DC
:10B600001F920E94BA940F900F900F900F900F907E
:10B6100081E08093150219821A821B821C821D828E
:10B620001E821F8218861D8619862CE32A873CE11C
:10B630003B8746E44C87E12CF12C00E81FEB812C82
:10B64000912C540160918E0470918F04072E000C90
:10B65000880B990B0E946CF26E87772E682E592EFC
:10B66000262F372F482F592FB701C8010E9466F2A5
:10B670008823C9F020919004309191044091920464
:10B68000509193046E85772D862D952D0E9466F23C
:10B69000881F8827881F8D87442049F0882339F028
:10B6A00051E05D87C4C0EE867F2C602E512E0E9433
:10B6B000D09F6B017C01DC01CB012D813E814F814C
:10B6C0005885821B930BA40BB50BB7FD3AC0D7016D
:10B6D000C60188519C4FAF4FBF4F8D839E83AF8370
:10B6E000B8870E9484E3E1E2FCE084918F010F5F60
:10B6F0001F4F882321F00E948584F801F6CF811422
:10B700009104A104B104B9F0D501C40188519C4F42
:10B71000AF4FBF4FBC01CD016C197D098E099F0948
:10B7200028EE33E040E050E00E9441F6CA01B90142
:10B730000E94279103C08FE30E9485848AE00E94C3
:10B74000858480E00E9469670E947FA32090900416
:10B750003090910400919204109193049101A801FA
:10B760006E85772D862D952D0E949EF69F7720E081
:10B7700030E040E251E481149104A104B10429F4C1
:10B780000E9466F287FF07C004C00E94C5F8181621
:10B7900014F4460157019D85992379F129813A8155
:10B7A0004B815C81211531054105510541F0D701DF
:10B7B000C601821B930BA40BB50BB7FD1EC09101F4
:10B7C000A80169857A858B859C850E949EF620E07C
:10B7D00030E040EC5FE30E9466F287FD61CFD70165
:10B7E000C601805A9541AF4FBF4F89839A83AB837F
:10B7F000BC8329863A860B871C8780911502882393
:10B80000B1F081149104A104B10429F4EE84F72C61
:10B81000062D152D17CF98EEC91A93E0D90AE10825
:10B82000F108C818D908EA08FB08F7FCEFCF8091A7
:10B830001502882341F1AD8560E0AA2319F085E067
:10B840009CE002C083E19CE02E960FB6F894DEBF28
:10B850000FBECDBFDF91CF911F910F91FF90EF9061
:10B86000DF90CF90BF90AF909F908F907F906F9020
:10B870005F904F903F902F900C941EC64110C8CE01
:10B8800084E693E0B7CE2E960FB6F894DEBF0FBED7
:10B89000CDBFDF91CF911F910F91FF90EF90DF907F
:10B8A000CF90BF90AF909F908F907F906F905F9060
:10B8B0004F903F902F90089580919B0490919C040D
:10B8C00021E02093A40A40E060E00C94CF52CF9393
:10B8D0008091A50A81110E94E64B8091A60A8823D7
:10B8E000A9F180E50E946FC4882319F00E94FEC36D
:10B8F00003C080E50E9440C4C82F482F61E08091BA
:10B900009B0490919C040E94CF5283E50E946FC4D7
:10B91000882381F00E94DDC3AB01BC014093480D38
:10B920005093490D60934A0D70934B0D87E99CE04D
:10B930000E94DE798091A60A882319F081E0809325
:10B94000A50AC11103C0CF910C948194CF910895A1
:10B95000CF93DF938091A60A882349F1E2EEFBE0C2
:10B960008491EF012196882321F00E948584FE01B5
:10B97000F7CF6091480D7091490D80914A0D9091DB
:10B980004B0D4AE00E94BF908FE20E948584609137
:10B99000440D7091450D8091460D9091470D4AE000
:10B9A0000E94BF908AE0DF91CF910C948584E4EFF0
:10B9B000FBE08491EF012196882321F00E94858489
:10B9C000FE01F7CFDF91CF910895E0919B04F091B4
:10B9D0009C048081882329F0803209F410823196FA
:10B9E000F8CF40E061E080919B0490919C040C941E
:10B9F000CF52CF92DF92EF92FF92CF93DF936A0103
:10BA00007B01C9EFD4E1E091A10424E0E29FF001C1
:10BA10001124E45EFD4F2081318142815381FC017C
:10BA200060817181828193810E947BF79B01AC01CF
:10BA30006C857D858E859F850E949FF66C877D87AE
:10BA40008E879F870E945CC5C701B6010E9474C2A1
:10BA5000DF91CF91FF90EF90DF90CF900C94E64B69
:10BA6000CF92DF92EF92FF92CF93DF9381E08093AA
:10BA70001502D1E0C1E080911502882309F446C087
:10BA8000CC2309F443C080E00E94696760918E0472
:10BA900070918F04C0E06115710569F3072E000CE9
:10BAA000880B990B0E946CF29B01AC016091900491
:10BAB0007091910480919204909193040E949EF65B
:10BAC0006B017C0120E030E0A9010E94C5F8181646
:10BAD0005CF020E030E040E251ECC701B6010E948A
:10BAE00066F287FFC8CF0BC020E030E040E251E4AF
:10BAF000C701B6010E94C5F818160CF0BCCFD09350
:10BB00004C0A8FE895EA0E941695B4CFDF91CF9149
:10BB1000FF90EF90DF90CF900895CF92DF92EF9259
:10BB2000FF920F931F93CF93DF9300D01F92CDB757
:10BB3000DEB7182F662351F0109205091092010903
:10BB40001092020910920309109204090E94D09FDA
:10BB5000C0900109D0900209E0900309F090040917
:10BB60009B01AC012C193D094E095F0957FD3DC0F1
:10BB700017FD16C040910509212F012E000C330B33
:10BB80002C5F3F4FE42F042E000CFF0B2E173F07B6
:10BB900064F141172CF000E911E020E030E004C02E
:10BBA00004EC19E020E030E0DC01CB01800F911FB4
:10BBB000A21FB31F8093010990930209A093030968
:10BBC000B093040980ED97E09C838B838CE291E035
:10BBD0009A838983BE016D5F7F4FCE010196AAD9FA
:10BBE000809105098F5F809305090F900F900F904A
:10BBF0000F90DF91CF911F910F91FF90EF90DF9009
:10BC0000CF90089560E089ED9BE00E941EC61798D2
:10BC100016981598149808953F924F925F926F92DC
:10BC20007F928F929F92AF92BF92CF92DF92EF92CC
:10BC3000FF920F931F93CF93DF930E94E64B8CE309
:10BC4000C82E83E0D82E09EF14E19AE2E92E94E0A1
:10BC5000F92EC0E0312CD0E0F60181916F010E94F5
:10BC60006FC48823B9F10E940DC44B015C01C3303D
:10BC700049F0F70120813181428153810E949EF673
:10BC80004B015C01F8012081318142815381C50162
:10BC9000B4010E949EF62B013C012DEB37E346E8F0
:10BCA00055EB0E94C5F887FD0AC02DEB37E346E847
:10BCB00055E3C301B2010E9466F218165CF4C3306A
:10BCC00019F03324339401C0D1E0F80180829182CD
:10BCD000A282B382CF5F0C5F1F4FF4E0EF0EF11C26
:10BCE000C43009F0B9CF332019F00E9454C303C007
:10BCF000D1110E9488EDDF91CF911F910F91FF909C
:10BD0000EF90DF90CF90BF90AF909F908F907F90FB
:10BD10006F905F904F903F90C5CA2F923F924F9285
:10BD20005F926F927F928F929F92AF92BF92CF92CB
:10BD3000DF92EF92FF920F931F93CF93DF93CDB7D4
:10BD4000DEB762970FB6F894DEBF0FBECDBF8A8B09
:10BD50000E94E64B409118025091190260911A021C
:10BD600070911B024093FD085093FE086093FF08FA
:10BD70007093000920911602309117023093FC084D
:10BD80002093FB0824E630E030931702209316023C
:10BD90000E947FA391E09093970D8A89811119C029
:10BDA00088E50E9440C4082F89E50E9440C4182FEE
:10BDB0008AE50E9440C4282E011106C0111113C04B
:10BDC000882361F0012F0FC0112369F0012F382E55
:10BDD0000BC011E001E02224239402C0182F082F89
:10BDE0003324339401C0312C0E945CC5311005C04E
:10BDF000011103C0112309F408C180E090E0A0EA1A
:10BE0000B0E48093AB049093AC04A093AD04B093E2
:10BE1000AE049C01AD0160910115709102158091F5
:10BE20000315909104150E9466F287FF0BC01982DA
:10BE30001A821B821C82BE016F5F7F4F8BEA94E0E7
:10BE40000E946DC231100DC0011103C01111D8C084
:10BE5000DCC0111106C080E00E9418AC3320B1F3A1
:10BE6000CFC01092FD141092FE141092FF14109285
:10BE700000151092F9141092FA141092FB141092FB
:10BE8000FC140E9454C3E5E8F2E02491298BEEEF04
:10BE9000FEE2C590D590E590F490E2E0FFE2859057
:10BEA0009590A590B490A5019401C701B6010E9498
:10BEB000C5F818162CF4A7019601C501B40104C0F9
:10BEC000A5019401C701B6010E947BF76D877E87AB
:10BED0008F87988B8DEB682E8EE2782EF30165911B
:10BEE00075918591949121EC422E2EE2522EF20111
:10BEF00025913591459154910E9466F287FF02C0C9
:10BF0000F30101C0F20145905590659074902D8524
:10BF10003E854F855889CA01B9010E94CBF220E0C5
:10BF200030E040E85FE30E949FF60E940AF99B011F
:10BF3000AC01C301B2010E94CBF269877A878B877B
:10BF40009C87E6E8F2E084918D8720E030E040ECC9
:10BF50005FE3C501B4010E94CBF22B013C012D85AA
:10BF6000622F220F770B880B990B0E946CF29B01BA
:10BF7000AC01C301B2010E94CBF269837A838B8347
:10BF80009C8320E030E040EC5FE3C701B6010E94F3
:10BF9000CBF26B017C012989622F220F770B880B72
:10BFA000990B0E946CF29B01AC01C701B6010E9483
:10BFB000CBF26D837E838F8398879E01275F3F4FEF
:10BFC00041E055E1BE016F5F7F4FCE0105960E94B3
:10BFD0008AC11092F4041092FD141092FE14109273
:10BFE000FF14109200151092F9141092FA14109286
:10BFF000FB141092FC1431102ECF01112CCF26CF40
:10C0000081E00E9418AC311003C0222009F45DC009
:10C0100080911915882321F080911A1581111DC076
:10C0200060E08BEC9BE00E941EC6E8EDF6E1849197
:10C030008F010F5F1F4F882321F00E948584F80134
:10C04000F6CFECEBFBE084918F010F5F1F4F88234D
:10C05000E1F10E948584F801F6CF0E9454C380E08C
:10C0600090E0A0E2B1E48093A3049093A404A09391
:10C07000A504B093A6048093A7049093A804A0936A
:10C08000A904B093AA048091011590910215A09182
:10C090000315B09104158093AB049093AC04A09366
:10C0A000AD04B093AE0419821A821B821C829E01D9
:10C0B0002F5F3F4F41E055E167EA74E083EA94E087
:10C0C0000E948AC182E00E9418AC0E9454C38091F1
:10C0D000960D8093970D8091FD089091FE08A09198
:10C0E000FF08B09100098093180290931902A09361
:10C0F0001A02B0931B028091FB089091FC08909368
:10C100001702809316020E947FA383E080932A0285
:10C11000C9D862960FB6F894DEBF0FBECDBFDF91CF
:10C12000CF911F910F91FF90EF90DF90CF90BF9034
:10C13000AF909F908F907F906F905F904F903F90C7
:10C140002F9008954F925F926F927F928F929F925D
:10C15000AF92BF92FF920F931F93CF93DF93CDB710
:10C16000DEB72A970FB6F894DEBF0FBECDBF109290
:10C170008B0980919109882339F00E945EA282E0A8
:10C1800099EE0E941695A9C42091160230911702CB
:10C1900040914D0A50914E0A60914F0A7091500A99
:10C1A000C901840F951F2436310524F48536910585
:10C1B0003CF416C02436310531F08436910584F400
:10C1C00084E690E00DC0473051056105710514F01B
:10C1D000069706C04A3F5F4F6F4F7F4F6CF406963D
:10C1E000909317028093160210924D0A10924E0AF5
:10C1F00010924F0A1092500A8091160290911702E5
:10C200008A3091053CF0883E43E094072CF087EE9D
:10C2100093E002C08AE090E09093170280931602A8
:10C220000E94D176F82E0E94BFC58091900D853175
:10C2300098F4FF2049F08091950490919604892B01
:10C2400019F008ED12E102C00BEB11E123E14FE020
:10C2500061E089E00E941A938091900D8D3108F081
:10C2600084C1883008F03FC08091480AF11002C0B4
:10C27000811139C060918E0470918F04072E000CDB
:10C28000880B990B0E946CF220E030E040E05FE305
:10C290000E949FF60E94E3F7643671052CF46A3021
:10C2A000710524F446E003C042E101C04CE022E104
:10C2B00030E0241B310937FF02C02F5F3F4F359517
:10C2C00027953195219531092B5F2093930D27E018
:10C2D0002093940DCB010E949E490E9415A388EBE8
:10C2E00091E10E9408A38091900D8D31D0F580914D
:10C2F000920D8531B0F120E030E040E05FE36091E5
:10C3000090047091910480919204909193040E9402
:10C310009FF60E94E3F79B01643671050CF0D6C2CC
:10C320002A3031050CF0D0C246E022E130E0241B77
:10C33000310937FF02C02F5F3F4F35952795319563
:10C34000219531092B5F2093930D2CE12093940DBF
:10C35000CB010E949E490E9415A388EB91E10E94A7
:10C3600008A38091900D853140F58091920D813127
:10C3700020F160918E0470918F04072E000C880BC1
:10C38000990B0E946CF2209190043091910440919D
:10C390009204509193040E94C5F818160CF098C2AC
:10C3A00010927C0D02E022E041E16DE08CE59DE021
:10C3B0000E94A29C81E080937C0D8091900D88303A
:10C3C00008F03FC080913F0AF11002C0811139C0CE
:10C3D00060918C0470918D04072E000C880B990BD2
:10C3E0000E946CF220E030E040E05FE30E949FF6A4
:10C3F0000E94E3F7643671052CF46A30710524F469
:10C4000046E003C042E101C04CE022E130E0241BE1
:10C41000310937FF02C02F5F3F4F35952795319582
:10C42000219531092F5A2093930D27E02093940DE5
:10C43000CB010E949E490E9415A388EB91E10E94C6
:10C4400008A38091900D8D31D0F58091920D8531AA
:10C45000B0F120E030E040E05FE360918204709151
:10C46000830480918404909185040E949FF60E9429
:10C47000E3F79B01643671050CF035C22A303105B3
:10C480000CF02FC246E022E130E0241B310937FFD7
:10C4900002C02F5F3F4F3595279531952195310982
:10C4A0002F5A2093930D2CE12093940DCB010E94E1
:10C4B0009E490E9415A388EB91E10E9408A38091F8
:10C4C000900D853140F58091920D813120F1609180
:10C4D0008C0470918D04072E000C880B990B0E9420
:10C4E0006CF2209182043091830440918404509135
:10C4F00085040E94C5F818160CF0F7C110927C0D47
:10C5000002E022E042E168E58CE59DE00E94A29C09
:10C5100081E080937C0D8091900D8C3130F580917D
:10C52000920D843110F180919504909196040196BA
:10C5300044E6489F9001499F300D112437FF02C007
:10C5400021503F4F832F932F990F990B009769F03C
:10C5500028E62093930D2BE12093940D0E949E4991
:10C560000E9415A385E20E94189480919A0C88235A
:10C5700049F08091900D843328F48091920D8A3295
:10C5800008F0BCC18091900D853328F48091920D04
:10C59000813308F0D9C160919404623048F08091F1
:10C5A000900D843328F48091920D823308F0D1C12C
:10C5B0008091900D813308F060C08091920D893296
:10C5C00008F45BC00E944D942B013C018CE3882E43
:10C5D000912CA12CB12CC301B201A50194010E94A0
:10C5E00041F6CA01B901A50194010E9441F6CA01B0
:10C5F000B62EA72E49018E010F5F1F4F41E844164A
:10C6000041E5540641E06406710408F4BDC1B90176
:10C6100028E130E040E050E00E9441F629013A0173
:10C62000AF92BF92C40168E170E00E9463F99F93EA
:10C630008F935F924F928DE89CE09F938F931F930F
:10C640000F930E94FFF10FB6F894DEBF0FBECDBF6F
:10C650009AE0491651046104710408F0BFC197E0E3
:10C66000892F880F980F9195955A9093930D80E399
:10C670008093940DC8010E9415A3E091560DF0918E
:10C68000570D84818111ECC020912A0430912B0434
:10C6900040912C0450912D046091F9147091FA147A
:10C6A0008091FB149091FC140E949FF60E94E3F786
:10C6B000CB010E943749BC0186E399E00E94D9F979
:10C6C00020912E0430912F04409130045091310478
:10C6D0006091FD147091FE148091FF1490910015EB
:10C6E0000E949FF60E94E3F7CB010E943749BC01EC
:10C6F00081E399E00E94D9F920913204309133040A
:10C7000040913404509135046091011570910215E7
:10C7100080910315909104150E949FF62CEA35EC48
:10C7200047E257E30E949FF620E030E048EC52E4F5
:10C730000E94CBF20E94E3F74B015C0197FD19C008
:10C7400090E1891697E29906A104B104E4F0C501CD
:10C75000B40120E137E240E050E00E9463F6CA01F4
:10C76000B9012AE030E040E050E00E9463F6605DED
:10C770000BC0B094A09490948094811C911CA11C37
:10C78000B11C6DE201C060E26093C40428EE821621
:10C7900023E09206A104B10494F0C501B40128EE8F
:10C7A00033E040E050E00E9463F6CA01B9012AE09C
:10C7B00030E040E050E00E9463F6605D01C060E25E
:10C7C0006093C504C501B40124E630E040E050E0C8
:10C7D0000E9463F69AE0492E512C612C712CCA01FB
:10C7E000B901A30192010E9463F6605D6093C604E3
:10C7F000C501B401A30192010E9463F64B015C01E3
:10C80000672B682B692B79F08EE28093C704CA01ED
:10C81000B901A30192010E9463F6605D6093C804B0
:10C8200080E3880D15C0CA01B901A30192010E94DD
:10C8300063F6662339F08EE28093C704605D6093EF
:10C84000C80405C080E28093C8048093C70480E2D6
:10C850008093C90464EC74E08AE299E00E94D9F9FB
:10C860008091900D8632A8F48091920D8E3188F0DF
:10C8700008E020E84EE160E08CE59DE00E94A29C8B
:10C880008091900D863228F48091920D8F3108F0BE
:10C89000A7C08091900D823328F48091920D8C3244
:10C8A00008F0FCC08091900D8F3308F016C1809184
:10C8B000920D883308F411C11092930D8EE380938A
:10C8C000940D0E94D59409C14CE02FCD42E12DCDAD
:10C8D00002E022E041E16DE08CE59DE00E94A29C37
:10C8E0006CCD4CE0D0CD42E1CECD02E022E042E181
:10C8F00068E58CE59DE00E94A29C0DCE07E028E053
:10C900004AE26AE28CE59DE00E94A29C05E022E0FA
:10C910004CE262E38CE59DE00E94A29C6AE08AE220
:10C920000E946E9360915E0D70915F0D82E3809323
:10C93000780D8BE28093790D28E73DE042E38CE5AA
:10C940009DE00E94E09A1ECE6AE486E30E946E9308
:10C9500022CE48E4649FB0011124072E000C880BFE
:10C96000990B0E946CF22AE037ED43E25CE30E94EF
:10C97000CBF20E94E8F7262F02E042E367E38CE562
:10C980009DE00E94A29C14CE44E68416910498F483
:10C99000AF92BF923F932F9383E89CE09F938F9336
:10C9A0001F930F930E94FFF10FB6F894DEBF0FBEE6
:10C9B000CDBF95E055CEAF92BF923F932F938BE7BB
:10C9C0009CE09F938F931F930F930E94FFF10FB6EC
:10C9D000F894DEBF0FBECDBF96E042CE98E040CEC9
:10C9E00010927C0D83E08093930D85E28093940DEB
:10C9F000FF2029F086EB91E10E9408A307C08091F7
:10CA0000B70E8111F7CF8FE30E9418948BE08093CB
:10CA1000930D15E21093940D86E399E00E9415A3FF
:10CA20008BE28093930D1093940DFF2029F084EBFB
:10CA300091E10E9408A307C08091B80E8111F7CF41
:10CA40008FE30E94189483E38093930D15E2109373
:10CA5000940D81E399E00E9415A383E58093930DE3
:10CA60001093940DFF2029F082EB91E10E9408A31E
:10CA700007C08091B90E8111F7CF8FE30E941894FF
:10CA80008BE58093930D85E28093940D8AE299E083
:10CA90000E9415A381E080937C0DFBCE84E00E9470
:10CAA000C3A283E08093930D12E31093940D86E06C
:10CAB0000E94F4A20E94BFC58CE08093930D109356
:10CAC000940D80911602909117020E949E490E9437
:10CAD00015A385E20E941894E5CE2A960FB6F89425
:10CAE000DEBF0FBECDBFDF91CF911F910F91FF90A1
:10CAF000BF90AF909F908F907F906F905F904F907E
:10CB00000895282F80914D0A90914E0AA0914F0AC6
:10CB1000B091500A81309048A105B10540F01092C3
:10CB20004D0A10924E0A10924F0A1092500A8091AC
:10CB30008009882331F080914D0A8093AA0E1092CB
:10CB40004A0A809175091816FCF4082E000C990BFE
:10CB5000821B91092091AA0E022E000C330B28177C
:10CB6000390794F097FF02C080E090E08093AA0E0E
:10CB7000092E000CAA0BBB0B80934D0A90934E0A12
:10CB8000A0934F0AB093500A8091AA0E6623A9F091
:10CB900090917609891714F480937609209176098B
:10CBA000022E000C330B2C5F3F4F482F082E000C39
:10CBB000550B241735071CF484508093760908958B
:10CBC00080914B0A8630D8F496E0899FF0011124B9
:10CBD000EA5FF64F209128023091290231832083A9
:10CBE00040914D0A50914E0A60914F0A7091500A3F
:10CBF00042835383648375838F5F80934B0A0895C8
:10CC000082EA90E60C941695E0914B0AEE2369F0C7
:10CC1000E150E0934B0A86E0E89FF0011124EA5FBF
:10CC2000F64F808191810C941695EACF10924C0AB0
:10CC3000EBCFAF92BF92CF92DF92EF92FF920F9322
:10CC40001F93CF93DF935C017B0120E030E0F5017F
:10CC5000E20FF31FE491EE2319F02F5F3F4FF7CF60
:10CC6000F701CF018E199F0941914111FACF04E1DB
:10CC700010E0081B11093327021713071CF0DD24ED
:10CC8000D39402C082E0D82E80915D0D90E06D2D8E
:10CC900070E06F5F7F4F0E9477F9C62EC6E0C60F27
:10CCA0008091900DC81750F08091920D90E02C2F3C
:10CCB00030E02B503109821793079CF5D0E0E11446
:10CCC000F104C1F18AE30E94189482E0D8120FC0E7
:10CCD000CC0D8091900DC81768F12091920D30E035
:10CCE0008C2F90E00B97281739071CF423C0DD2305
:10CCF00009F1802F880F080F000F0093930DC09348
:10CD0000940D80E20E941894C701DF91CF911F918A
:10CD10000F91FF90EF90DF90CF90BF90AF900C9469
:10CD200015A31092930DC093940DC5010E9408A302
:10CD3000D1E0C5CFDF91CF911F910F91FF90EF9080
:10CD4000DF90CF90BF90AF9008950F934CE0849FF9
:10CD5000402D112421E0240F2093E6068CE0840F5F
:10CD60008093E706E091900DF0E090E002968E1738
:10CD70009F070CF1822F90E02091920D30E08217F6
:10CD80009307CCF4662371F081E080937C0D4D5FB6
:10CD90000BE020E860E08CE59DE00E94A29C1092F0
:10CDA0007C0D03C081E080937C0D8091E70610929A
:10CDB000930D8093940D0F910895CF92DF92EF928F
:10CDC000FF920F93CF93DF93982F862F6A017901FB
:10CDD000692FBBDF9091900D8091E706891708F4C9
:10CDE00053C09091920D8091E606981708F44CC0BC
:10CDF000002359F060E070E0F701E60FF71FE491BF
:10CE0000EE2351F06F5F7F4FF7CFD701BD016E1951
:10CE10007F098D918111FACFC62FD4E1D61BF6017F
:10CE20008491882339F00E94DDA2D81BFFEFCF1A2E
:10CE3000DF0AF5CF8AE30E941894DD2329F080E20F
:10CE40000E941894D150F9CF8091E7066AEFC69FEF
:10CE5000602D112460586093930D8093940DC70149
:10CE6000002349F0DF91CF910F91FF90EF90DF9079
:10CE7000CF900C9408A3DF91CF910F91FF90EF908A
:10CE8000DF90CF900C9415A3DF91CF910F91FF907D
:10CE9000EF90DF90CF9008950F93CF93DF93CDB7AE
:10CEA000DEB7ED85FE8560817181828193810E946C
:10CEB000E3F7CB010E949E4900E09C0149855A8519
:10CEC00068858F817ADFDF91CF910F910895149A51
:10CED0000895CF92DF92EF92FF920F931F93CF931B
:10CEE000DF93C82F0E94E27380918B04882391F016
:10CEF0000E94D09F0091870410918804209189049A
:10CF000030918A04DC01CB01801B910BA20BB30B87
:10CF1000B7FF35C18091D606853010F40E943DC61A
:10CF20000E94D09FC0907E04D0907F04E090800447
:10CF3000F0908104C114D104E104F10471F1009175
:10CF40009D0410919E0420919F043091A0040C0D2B
:10CF50001D1D2E1D3F1D6B017C01C01AD10AE20A66
:10CF6000F30AF7FC1AC0E5EBFBE08491EF01219690
:10CF7000882321F00E948584FE01F7CF6091F6039B
:10CF80007091F70382E994E10E9420A48AE00E9454
:10CF9000858489E894E10E945EAF20919904211173
:10CFA00028C0C0901102D0901202E0901302F090BD
:10CFB0001402C114D104E104F104D9F000919D04DC
:10CFC00010919E0420919F043091A0040C0D1D1D12
:10CFD0002E1D3F1DDC01CB01801B910BA20BB30B5F
:10CFE000B7FD07C0C11105C00E9453C5882309F4CD
:10CFF000E5C00E94D09F0091690910916A092091B3
:10D000006B0930916C096B017C01C01AD10AE20AEC
:10D01000F30AF7FC3AC08B019C010C53164F2F4FBB
:10D020003F4F0093690910936A0920936B0930936D
:10D030006C09079BCEC0069BCCC0059BCAC0209143
:10D040000C042111C6C0049BC4C000916509109155
:10D0500066092091670930916809011511052105BC
:10D06000310509F4BFC0DC01CB01801B910BA20B81
:10D07000B30B80569A4EA109B109B7FFB3C0749A99
:10D080006FEF70E082E00E94D19E0E9453C5811133
:10D0900005C0D0919504C09197041AC0E091770A19
:10D0A0008FE48E9FF0011124E75CF04FD081E09176
:10D0B000770A8E9FF0011124E55CF04FC0818091CA
:10D0C000770A9091760A891719F08F5F8F70F9CFE0
:10D0D000DD2329F10E94D09F00916D0910916E0906
:10D0E00020916F0930917009DC01CB010115110508
:10D0F0002105310569F48C599F4FAF4FBF4F809385
:10D100006D0990936E09A0936F09B0937009B0C038
:10D11000801B910BA20BB30BB7FFABC0A9C0109241
:10D120006D0910926E0910926F0910927009CC234C
:10D1300009F478C00E94D09F009171091091720982
:10D140002091730930917409DC01CB01011511059F
:10D150002105310569F48C599F4FAF4FBF4F809324
:10D16000710990937209A0937309B09374093DC03B
:10D17000801B910BA20BB30BB7FF38C036C00E94C7
:10D18000D09F6B017C0120918B0430E0A8EEB3E0CE
:10D190000E948FF6DC01CB018C0D9D1DAE1DBF1DC5
:10D1A0008093870490938804A0938904B0938A04A1
:10D1B0000E9484E38AE00E948584ACCE179A109284
:10D1C0001915169A10921A15159A10921B157FDED2
:10D1D00010CF6093650970936609809367099093F7
:10D1E000680933CF749860E04CCFCFEFDD23D1F1E5
:10D1F00029EBD29FC00111246FEF70E00E9477F9F4
:10D200006A5B7F4F88E00E94D19ECC23C1F029EB5E
:10D21000C29FC00111246FEF70E00E9477F96A5B32
:10D220007F4F0FC01092710910927209109273090A
:10D230001092740960E070E088E00E94D19E60E086
:10D2400070E086E00E94D19E0E9474E788E79AE031
:10D25000DF91CF911F910F91FF90EF90DF90CF90D2
:10D260000C9412A260E070E088E00E94D19ECFCFC3
:10D27000DFEFC1115FCF1092710910927209109205
:10D28000730910927409B4CF179AE9E1F5E110829D
:10D29000169A1182159A12821ACECF92DF92EF92CD
:10D2A000FF92CF93DF9320911002222309F443C011
:10D2B000EC01C0900402D0900502E0900602F090CC
:10D2C0000702A7019601688179818A819B810E946A
:10D2D000C5F8181624F4C882D982EA82FB82C0906D
:10D2E0000802D0900902E0900A02F0900B02A70118
:10D2F00096016C817D818E819F810E94C5F81816F0
:10D3000024F4CC82DD82EE82FF82C0900C02D090A9
:10D310000D02E0900E02F0900F02A70196016885C1
:10D3200079858A859B850E94C5F8181624F4C886DD
:10D33000D986EA86FB86DF91CF91FF90EF90DF9050
:10D34000CF900895CF93DF930E947FA3E091D506FD
:10D35000F0E0ED52FB4F8081882309F45EC0E6E8DF
:10D36000F4E18491EF012196882321F00E948584C5
:10D37000FE01F7CFC091D50680E6C89FE0011124D9
:10D38000CB50DB4F88818E3419F0E3E8F4E110C014
:10D3900080E20E94858489910E948584899190ED24
:10D3A000980F9A30C8F38D32B9F38B32A9F3EDCFD1
:10D3B0008491EF012196882321F00E948584FE014B
:10D3C000F7CF8091760A9091770A891B8F706FE072
:10D3D00070E0681B7109072E000C880B990B0E94E6
:10D3E0002791E0E8F4E18491EF012196882321F070
:10D3F0000E948584FE01F7CF8091D60665E070E03B
:10D40000681B7109072E000C880B990B0E9427914D
:10D410008AE0DF91CF910C948584DF91CF910895BC
:10D42000CF93DF938FB7F8949091150A9093140AD5
:10D430008FBFE7E7F4E18491EF012196882321F083
:10D440000E948584FE01F7CF8091EA069091EB0659
:10D45000A091EC06B091ED06BC01CD016F5F7F4F4E
:10D460008F4F9F4F0E9427918AE00E948584DF9111
:10D47000CF9168CFEF92FF920F931F93CF93DF93DB
:10D48000C091D50680E6C89FE0011124CB50DB4F48
:10D490008091A20480FF19C0E8EDF6E184918F012C
:10D4A0000F5F1F4F811102C08E0104C00E9485844E
:10D4B000F801F4CFD8018D918D01882319F00E94D5
:10D4C0008584F8CF8AE00E94858410929C04109293
:10D4D0009B048FE38093BA041092B9041092B804AD
:10D4E0001092610910926209109263091092640906
:10D4F000FE01888121968032D9F38E34B1F4818186
:10D5000090ED980F9A3020F08D3211F08B3269F443
:10D510003296DF0131962C9120532A30D0F3CD0181
:10D52000FC01019620812032D9F3F093F703E093B8
:10D53000F6038F010F5F1F4FC0816AE270E0C801E0
:10D540000E94CEF9009731F0FC0131978081803242
:10D55000E1F31182CD3429F0C43519F0C73409F054
:10D56000E5C0F80180810F5F1F4F8032D1F38053F7
:10D570008A3008F0DBC0C093BA041092B90410924C
:10D58000B8046AE08091B8049091B904689FA00142
:10D59000699F500D11245093B9044093B8043196FB
:10D5A000DF0111978C91282F30E020533109240F8F
:10D5B000351F3093B9042093B804808180538A309A
:10D5C00008F3DF0131968C918032D9F3CD34B9F470
:10D5D0002E31310579F03CF42731310559F02C31E9
:10D5E000310569F407C02537310521F0203AE3E021
:10D5F0003E0729F4B0939C04A0939B0497C010921B
:10D600009C0410929B04D091F60361E070E0CD0180
:10D6100001964C91442309F489C0413299F4CD34E8
:10D6200089F42032310571F490939C0480939B041B
:10D6300063E270E00E94CEF9009709F477C0DC0144
:10D640001C9274C041544A3108F043C0DC01FD0112
:10D650005D915032E1F3CF01A0EDA50FAA30C8F0E3
:10D660005E3229F4518150535A3098F067C05D32D0
:10D6700019F05B3209F062C05181A0EDA50FAA300C
:10D6800048F05E3209F05AC0528150535A3010F0BF
:10D6900055C0FC01042F10E0D80153E0B595A795C3
:10D6A0005A95E1F7AF59B64F47707B0102C0EE0CB7
:10D6B000FF1C4A95E2F7A7015C91452B4C933097EC
:10D6C00011F0ED1B01C0E0E0D801A95BB64FEC936F
:10D6D0000AC040919B0450919C04452B21F4B093C7
:10D6E0009C04A0939B04DC014C9141544A3110F4FA
:10D6F000DC018DCFFC018E2FAF2F9191911103C0D2
:10D70000482F5A2F0BC040ED490F4A30A0F343ED8C
:10D71000490F423080F39B3271F3F2CFCA014F5F61
:10D720005F4FDC01EC91E032C9F3E2CFDF91CF91A2
:10D730001F910F91FF90EF900C94A925A0919B044D
:10D74000B0919C04AB2B29F43197F0939C04E093A7
:10D750009B04E0E0F0E09ECF0F931F93CF9383E50F
:10D760000E946FC4882309F447C00E94EDC3813032
:10D7700039F0823009F040C00CE313E0C0E021C072
:10D780000CE313E0C0E0F80181918F010E946FC4A7
:10D79000882339F00E94EDC34FEF682F8C2F0E9431
:10D7A000B04ACF5FC43079F782E40E946FC4882307
:10D7B00019F10E94EDC34FEF682F1BC0CF5FC4303B
:10D7C00079F0F80181918F010E946FC48823B1F331
:10D7D0000E94EDC3482F6FEF8C2F0E94B04AEECF0E
:10D7E00082E40E946FC4882339F00E94EDC3482F61
:10D7F0006FEF84E00E94B04ACF911F910F910C947B
:10D80000F8490F931F93CF9383E50E9440C4811181
:10D8100004C00CE313E0C0E00EC0C0E00E94EDC302
:10D82000682F8C2F0E945A4BCF5FC530B9F7F1CFCC
:10D83000CF5FC43071F0F80181918F010E9440C424
:10D840008823B1F30E94EDC3682F8C2F0E945A4B9E
:10D85000EFCF82E40E9440C4882331F00E94EDC3E0
:10D86000682F84E00E945A4BCF911F910F910C9426
:10D87000F849CF93DF9383E50E946FC4882321F09A
:10D880000E94DDC3EB0102C0C0E0D0E080E50E9451
:10D890006FC4882321F00E94DDC3CB0102C080E069
:10D8A00090E0BE01DF91CF910C94714B0F931F93C9
:10D8B000CF930CE313E0C0E0F80181918F010E9447
:10D8C00040C4882329F00E94DDC38C2F0E94804B26
:10D8D000CF5FC43089F782E40E9440C4882329F0D6
:10D8E0000E94DDC384E00E94804B83E50E9440C417
:10D8F000882349F0C0E00E94DDC38C2F0E94804B3A
:10D90000CF5FC530C1F7CF911F910F91089588E87F
:10D9100093E19093C2048093C10480916F008D7F46
:10D9200080936F000E9453C5882359F00E9453C50D
:10D930008823C1F38091770A8F5F8F708093770A75
:10D94000F1CF1092C0041092BF0480916F008260EA
:10D9500080936F008FB7F8941092CF0E1092D00E74
:10D960001092D10E1092D20E8FBF0E94E64B80E033
:10D970000E94C94B60933B0970933C0980933D0919
:10D9800090933E0981E00E94C94B60933F097093D8
:10D990004009809341099093420982E00E94C94B5B
:10D9A0006093430970934409809345099093460915
:10D9B0008CE0EBE3F9E0A9EFB4E101900D928A95D8
:10D9C000E1F70C9454C3EF92FF920F931F93CF9300
:10D9D0008CE3E82E83E0F82E0EEF13E0C0E0F701B1
:10D9E00081917F010E9440C4882351F00E940DC4A0
:10D9F000F80160837183828393838C2F0E9499C284
:10DA0000CF5F0C5F1F4FC33051F7CF911F910F9124
:10DA1000FF90EF900C94525983E50E9440C48823F4
:10DA2000D9F00E940DC4AB01BC0140936D1450931A
:10DA30006E1460936F147093701440936514509338
:10DA4000661460936714709368148FE494E10E94E5
:10DA5000C3A38AE00E94858480E50E9440C4882395
:10DA600099F00E940DC4AB01BC0140936D1450931A
:10DA70006E1460936F147093701482E394E10E94AB
:10DA8000C3A38AE00E94858482E50E9440C4882363
:10DA900099F00E940DC4AB01BC01409369145093EE
:10DAA0006A1460936B1470936C1483E194E10E9488
:10DAB000C3A38AE00E94858484E50E9440C4882331
:10DAC00099F00E940DC4AB01BC01409365145093C2
:10DAD0006614609367147093681485EF93E10E9455
:10DAE000C3A38AE00C9485840895FF920F931F933B
:10DAF000CF93DF930EE514E0CCE3D3E0FC2E84E07B
:10DB0000F80E89910E9440C4882339F00E940DC408
:10DB1000F80160837183828393830C5F1F4FFC1233
:10DB2000F0CFDF91CF911F910F91FF900895FF9259
:10DB30000F931F93CF93DF9301E714E1CCE3D3E07E
:10DB4000FC2E84E0F80E89910E9440C4882349F09D
:10DB50000E940DC40E94E8F7F801608371838283FC
:10DB600093830C5F1F4FFC12EECFDF91CF911F917B
:10DB70000F91FF900C94E1BECF9388EC90E00E944F
:10DB80000DC5811140C084E40E9440C48823C1F1C6
:10DB90000E940DC4C1E020E030E0A9010E9466F2BD
:10DBA000811101C0C0E0C0938514CC2349F10E94CB
:10DBB0000DC4E091860424E0E29FF0011124EF57A8
:10DBC000FB4E608371838283938320E030E0A90160
:10DBD00060918114709182148091831490918414C7
:10DBE0000E9466F281110CC080E090E0A0E4B0E4F5
:10DBF0008093811490938214A0938314B09384141F
:10DC0000CF910C942084CF910895CF92DF92EF9220
:10DC1000FF920F931F93CF93DF9300D01F92CDB746
:10DC2000DEB780914D0A90914E0AA0914F0AB091B3
:10DC3000500AB7FF08C010924D0A10924E0A109277
:10DC40004F0A1092500A8091D7069091D806A09161
:10DC5000D906B091DA0640914D0A50914E0A609172
:10DC60004F0A7091500A84179507A607B70744F426
:10DC700080934D0A90934E0AA0934F0AB093500A96
:10DC800080912A02882379F140914D0A50914E0AE1
:10DC900060914F0A7091500A8091DB069091DC06EA
:10DCA000A091DD06B091DE066A017B01C80ED91E87
:10DCB000EA1EFB1EC701B6010E946CF22AE037ED96
:10DCC00043E25CE30E94CBF269837A838B839C837B
:10DCD000CE0101960E941747BC018091E106909108
:10DCE000E2060E941966809191091091E306811164
:10DCF00006C01123D1F180912A028823B1F140910D
:10DD00004D0A50914E0A60914F0A7091500A8091CD
:10DD1000DB069091DC06A091DD06B091DE066A017B
:10DD20007B01C80ED91EEA1EFB1EC701B6010E9468
:10DD30006CF22AE037ED43E25CE30E94CBF2E09123
:10DD4000DF06F091E006309721F0608371838283D3
:10DD50009383112329F0E091E406F091E5061995EB
:10DD60008091910981110E94046680919109882314
:10DD700029F0E091E406F091E50619950F900F90D7
:10DD80000F900F90DF91CF911F910F91FF90EF9027
:10DD9000DF90CF900895CF92DF92EF92FF920F9392
:10DDA0001F93CF93DF9300D01F92CDB7DEB7809142
:10DDB0004D0A90914E0AA0914F0AB091500AB7FFB8
:10DDC00008C010924D0A10924E0A10924F0A1092FB
:10DDD000500A8091D7069091D806A091D906B091AB
:10DDE000DA0640914D0A50914E0A60914F0A7091A7
:10DDF000500A84179507A607B70744F480934D0A85
:10DE000090934E0AA0934F0AB093500A80912A0231
:10DE1000882379F140914D0A50914E0A60914F0A42
:10DE20007091500A8091DB069091DC06A091DD068E
:10DE3000B091DE066A017B01C80ED91EEA1EFB1EE8
:10DE4000C701B6010E946CF22AE037ED43E25CE3C1
:10DE50000E94CBF269837A838B839C83CE010196E7
:10DE60000E94CC47BC018091E1069091E2060E949D
:10DE70001966809191091091E306811106C0112362
:10DE8000D1F180912A028823B1F140914D0A50913D
:10DE90004E0A60914F0A7091500A8091DB06909172
:10DEA000DC06A091DD06B091DE066A017B01C80E9A
:10DEB000D91EEA1EFB1EC701B6010E946CF22AE0C1
:10DEC00037ED43E25CE30E94CBF2E091DF06F09194
:10DED000E006309721F0608371838283938311235E
:10DEE00029F0E091E406F091E506199580919109F9
:10DEF00081110E9404660F900F900F900F90DF9198
:10DF0000CF911F910F91FF90EF90DF90CF900895E8
:10DF1000CF92DF92EF92FF920F931F93CF93DF93F5
:10DF200000D01F92CDB7DEB780914D0A90914E0A76
:10DF3000A0914F0AB091500AB7FF08C010924D0A45
:10DF400010924E0A10924F0A1092500A8091D706F2
:10DF50009091D806A091D906B091DA0640914D0A69
:10DF600050914E0A60914F0A7091500A841795079C
:10DF7000A607B70744F480934D0A90934E0AA093E6
:10DF80004F0AB093500A80912A02882379F1409178
:10DF90004D0A50914E0A60914F0A7091500A80913B
:10DFA000DB069091DC06A091DD06B091DE066A01E9
:10DFB0007B01C80ED91EEA1EFB1EC701B6010E94D6
:10DFC0006CF220E030E048EC52E40E94CBF269832E
:10DFD0007A838B839C83CE0101960E944D48BC01BD
:10DFE0008091E1069091E2060E9419668091910964
:10DFF0001091E306811106C01123D1F180912A020C
:10E000008823B1F140914D0A50914E0A60914F0A18
:10E010007091500A8091DB069091DC06A091DD069C
:10E02000B091DE066A017B01C80ED91EEA1EFB1EF6
:10E03000C701B6010E946CF220E030E048EC52E4E7
:10E040000E94CBF2E091DF06F091E006309721F0DC
:10E050006083718382839383112329F0E091E40626
:10E06000F091E50619958091910981110E9404664D
:10E070000F900F900F900F90DF91CF911F910F9104
:10E08000FF90EF90DF90CF900895CF92DF92EF92C4
:10E09000FF920F931F93CF93DF9300D01F92CDB7C2
:10E0A000DEB780914D0A90914E0AA0914F0AB0912F
:10E0B000500AB7FF08C010924D0A10924E0A1092F3
:10E0C0004F0A1092500A8091D7069091D806A091DD
:10E0D000D906B091DA0640914D0A50914E0A6091EE
:10E0E0004F0A7091500A84179507A607B70744F4A2
:10E0F00080934D0A90934E0AA0934F0AB093500A12
:10E1000080912A02882379F140914D0A50914E0A5C
:10E1100060914F0A7091500A8091DB069091DC0665
:10E12000A091DD06B091DE066A017B01C80ED91E02
:10E13000EA1EFB1EC701B6010E946AF220E030E031
:10E1400048EC52E40E94CBF269837A838B839C83F0
:10E15000CE0101960E944D48BC018091E10690914C
:10E16000E2060E941966809191091091E3068111DF
:10E1700006C01123E1F180912A028823C1F1409168
:10E180004D0A50914E0A60914F0A7091500A809149
:10E19000DB069091DC06A091DD06B091DE066A01F7
:10E1A0007B01C80ED91EEA1EFB1EC701B6010E94E4
:10E1B0006AF220E030E048EC52E40E94CBF20E9488
:10E1C000E8F7E091DF06F091E006309721F06083F8
:10E1D000718382839383112329F0E091E406F09107
:10E1E000E50619958091910981110E94046680913C
:10E1F0009109882329F0E091E406F091E50619954C
:10E200000F900F900F900F90DF91CF911F910F9172
:10E21000FF90EF90DF90CF9008950F931F93CF93CF
:10E2200080914D0A90914E0AA0914F0AB091500AE8
:10E23000B7FF08C010924D0A10924E0A10924F0A72
:10E240001092500A8091D7069091D806A091D906D5
:10E25000B091DA0640914D0A50914E0A60914F0AF2
:10E260007091500A84179507A607B70744F4809366
:10E270004D0A90934E0AA0934F0AB093500A809192
:10E280002A02882331F140914D0A50914E0A609143
:10E290004F0A7091500A8091DB069091DC06A091A4
:10E2A000DD06B091DE068A019B01080F191F2A1FA7
:10E2B0003B1FC901B8010E946CF20E94E3F7CB0139
:10E2C0000E949E49BC018091E1069091E2060E9465
:10E2D000196680919109C091E306811106C0CC2393
:10E2E000A1F180912A02882381F140914D0A509139
:10E2F0004E0A60914F0A7091500A8091DB0690910E
:10E30000DC06A091DD06B091DE068A019B01080FB4
:10E31000191F2A1F3B1FC901B8010E946CF2E0912E
:10E32000DF06F091E006309721F0608371838283ED
:10E330009383CC2329F0E091E406F091E50619954A
:10E340008091910981110E94046680919109CF9179
:10E350001F910F91089561CF60DF882329F0E0912C
:10E36000E406F091E5061994089580914D0A909184
:10E370004E0AA0914F0AB091500AB7FF08C0109200
:10E380004D0A10924E0A10924F0A1092500A809134
:10E39000D7069091D806A091D906B091DA0640919F
:10E3A0004D0A50914E0A60914F0A7091500A84179D
:10E3B0009507A607B70744F480934D0A90934E0A39
:10E3C000A0934F0AB093500A80912A02882399F0B3
:10E3D0002091DB063091DC0680914D0A90914E0A27
:10E3E000820F931F0E949E49BC018091E10690918B
:10E3F000E2060E941966809191092091E30681113D
:10E4000006C0222311F180912A028823F1F0409165
:10E41000DB065091DC0680914D0A90914E0A840FE4
:10E42000951FE091DF06F091E006309711F091839F
:10E430008083222329F0E091E406F091E506199506
:10E440008091910981110E9404668091910908953B
:10E450008CCF8BDF882329F0E091E406F091E5066C
:10E4600019940895CF93DF9360E085E00E94816561
:10E47000D0917609C0E0D11109C080912A02882389
:10E48000E9F021E041E069EC75E115C0D13049F4D3
:10E4900080912A02882391F020E041E06AEB75E147
:10E4A0000AC0D23059F480912A02882339F020E042
:10E4B00041E060EB75E18C2F0E94CE57CF5FDF5FAC
:10E4C000C530C9F683E080937509DF91CF91089537
:10E4D0001F93CF93DF9360E085E00E948165D09128
:10E4E0007609C0E012E0D11109C080912A02882388
:10E4F000D9F121E041E063EA75E115C0D13049F47A
:10E5000080912A02882381F120E041E06AE975E1E7
:10E510000AC0D23061F480912A02882329F120E0D8
:10E5200041E069E875E18C2F0E94CE571DC0D330C1
:10E5300049F480912A028823B9F020E041E067E89D
:10E5400075E1F1CFD43081F480912A02882351F013
:10E5500021E040E06CE775E18C2F0E94CE578C2FB4
:10E560000E9420A310932A02CF5FDF5FC53009F01D
:10E57000BACFC0937509DF91CF911F9108951F9372
:10E58000CF93DF9360E085E00E948165D0917609AA
:10E59000C0E012E0D11109C080912A028823D9F18C
:10E5A00021E041E06FE675E115C0D13049F480917A
:10E5B0002A02882381F120E041E066E675E10AC085
:10E5C000D23061F480912A02882329F120E041E0D1
:10E5D00068E575E18C2F0E94CE571DC0D33049F4F9
:10E5E00080912A028823B9F020E041E066E575E1D8
:10E5F000F1CFD43081F480912A02882351F021E0B8
:10E6000040E06BE475E18C2F0E94CE578C2F0E9466
:10E6100020A310932A02CF5FDF5FC53009F0BACF85
:10E62000C0937509DF91CF911F9108951F93CF93E8
:10E63000DF9360E085E00E948165D0917609C0E0BB
:10E6400012E0D11109C080912A028823D9F121E07A
:10E6500041E06EE375E115C0D13049F480912A02A2
:10E66000882381F120E041E06EE275E10AC0D230FA
:10E6700061F480912A02882329F120E041E06DE1D4
:10E6800075E18C2F0E94CE571DC0D33049F4809184
:10E690002A028823B9F020E041E06EE075E1F1CF75
:10E6A000D43081F480912A02882351F021E040E0A7
:10E6B00063E075E18C2F0E94CE578C2F0E9420A31F
:10E6C00010932A02CF5FDF5FC53009F0BACFC09345
:10E6D0007509DF91CF911F9108951F93CF93DF9319
:10E6E00060E085E00E948165D0917609C0E012E08B
:10E6F000D11109C080912A028823D9F121E041E09B
:10E7000066EF74E115C0D13049F480912A02882364
:10E7100081F120E041E066EE74E10AC0D23061F49C
:10E7200080912A02882329F120E041E069ED74E11B
:10E730008C2F0E94CE571DC0D33049F480912A02FD
:10E740008823B9F020E041E067ED74E1F1CFD430E7
:10E7500081F480912A02882351F021E040E06CECA2
:10E7600074E18C2F0E94CE578C2F0E9420A310930F
:10E770002A02CF5FDF5FC53009F0BACFC0937509B9
:10E78000DF91CF911F910895EBE2F2E080E091914B
:10E79000911104C0982F981B50E206C0863111F0E9
:10E7A0008F5FF5CF96E1F7CF282F30E0492F480F44
:10E7B000F901E55DFD4F463118F450838F5FF4CFCA
:10E7C000108208954F925F926F927F928F929F92E4
:10E7D000AF92BF92CF92DF92EF92FF920F931F936F
:10E7E000CF93DF9300D01F92CDB7DEB710912702F1
:10E7F0001F3F01F10E94D09FC0907C09D0907D09FD
:10E80000E0907E09F0907F09DC01CB018C199D0915
:10E81000AE09BF09B7FD0EC02091770A8091760A34
:10E8200030E08F5F8F70082E000C990B2817390786
:10E8300009F029C20E94C7C58091E91382FF39C03F
:10E8400080919209811137C081E080939209909163
:10E850009A0489278093910910929A0483E0809307
:10E860002A021092E9130E94D09FDC01CB018C5048
:10E870009E4FAF4FBF4F8093EA139093EB13A0933B
:10E88000EC13B093ED1348E853E162E070E080E0F0
:10E8900090E00E9476EB16E0115069F088E79AE06C
:10E8A0000E9412A262E070E080E090E00E94989FD7
:10E8B000F3CF1092920919B11295117081E01827C7
:10E8C00080919009412F50E0282F30E042175307E4
:10E8D000A9F0112309F4FDC10E94145680919009FA
:10E8E000823029F060E083EE95E10E941EC610930D
:10E8F000900983E080932A020E945EA20E94D09F2A
:10E900006B017C0180918C0990918D09A0918E09F9
:10E91000B0918F09A7019601281B390B4A0B5B0B9D
:10E9200057FF05C08091490A882309F425C2D70101
:10E93000C6018C599F4FAF4FBF4F80938C09909366
:10E940008D09A0938E09B0938F098091E713181653
:10E950002CF48091E713823074F408C08091E7139F
:10E96000992781950CF4909502972CF48091910948
:10E9700081119BC0ABC080918B09882309F46EC0C4
:10E980008091E713181654F48091E713082E000CB9
:10E99000990B97FD0196959587950CC08091E7138B
:10E9A000082E000C990B97FD0196959587959195EA
:10E9B000819591098090870990908809A090890994
:10E9C000B0908A0981149104A104B104D1F1BC0171
:10E9D000990F880B990B0E946CF22B013C01C70127
:10E9E000B601681979098A099B090E946AF29B019C
:10E9F000AC01C301B2010E947BF720E030E04AE79E
:10EA000054E40E94CBF24B015C0120E030E040E294
:10EA100053E40E94C5F887FF0FC020E030E046E9CC
:10EA200052E4C501B4010E94C5F887FD0AC02AE07E
:10EA300030E040E050E009C024E630E040E050E043
:10EA400004C021E030E040E050E0C0928709D0925D
:10EA50008809E0928909F0928A0904C021E030E037
:10EA600040E050E0A091E7130A2E000CBB0B0E947F
:10EA700089F622E030E040E050E00E9463F68091A9
:10EA80004D0A90914E0AA0914F0AB091500A820F00
:10EA9000931FA41FB51F80934D0A90934E0AA09315
:10EAA0004F0AB093500A1092E713D701C601885657
:10EAB000954CAF4FBF4F8093830990938409A093E7
:10EAC0008509B093860981E080932A02209128026B
:10EAD0003091290240E6223A340741F480919702AE
:10EAE000882309F401C1815080939702275C374A3B
:10EAF00071F480911C1590911D15891740F4909127
:10EB00009702992309F400C19150909397022FB76F
:10EB1000F8948091CF0E9091D00EA091D10EB0912B
:10EB2000D20E2FBF3AE0B695A795979587953A955F
:10EB3000D1F7009721E0A207B10520F08FEF9FEFFA
:10EB4000A0E0B0E09695879520912A02211105C09A
:10EB50003091490A31110CC159C0009741F04091E0
:10EB60008109509182094817590708F04FC08091D8
:10EB7000490A811113C0223050F0243028F024308B
:10EB800031F410922A0203C081E080932A020E948D
:10EB9000E49481E0809380098093490A84E00E9494
:10EBA000C3A281E080937C0DE0912802F0912902BC
:10EBB000199510929109109280098091490A882331
:10EBC00051F00E94E29291E0811101C090E0909397
:10EBD000490A9111B1C08090810990908209A12CBD
:10EBE000B12C0E94D09FDC01CB018C199D09AE098C
:10EBF000BF0988169906AA06BB0640F40E94D09F5A
:10EC00006C197D09709382096093810980912802B3
:10EC100090912902825A904621F080914C0A8823D3
:10EC200079F048E9C40E4AE3D41EE11CF11CC092FD
:10EC30008309D0928409E0928509F09286090FC079
:10EC40008091830990918409A0918509B0918609EA
:10EC5000C81AD90AEA0AFB0AF7FE0E9400668091E8
:10EC6000490A811189C080912A02813049F008F453
:10EC700083C0843008F080C081E080932A027CC089
:10EC800010922A0279C054E01502F0011124E159D2
:10EC9000FC4F20E030E040E752E4608171818281E6
:10ECA00093810E947BF769837A838B839C83E12C19
:10ECB0008E010F5F1F4F25E035E141E055E16DEF1B
:10ECC00074E189EF94E10E9438C08FEF80932702AE
:10ECD000B1CD1092A50A1092A60A823009F407CE8F
:10ECE00060E086ED95E101CE8CE080939702809103
:10ECF00081099091820901979093820980938109FB
:10ED000081E080932A02F2CE96E09093970291E000
:10ED100090932A028F5F80931C15D701C6018856F5
:10ED2000954CAF4FBF4F8093830990938409A09374
:10ED30008509B0938609EBCE809081099090820975
:10ED4000A12CB12C0E94D09FDC01CB018C199D0914
:10ED5000AE09BF0988169906AA06BB0668F40E9488
:10ED6000D09F6C197D09709382096093810904C05A
:10ED7000009709F413CFF3CE0F900F900F900F90E0
:10ED8000DF91CF911F910F91FF90EF90DF90CF9087
:10ED9000BF90AF909F908F907F906F905F904F90BB
:10EDA0000895CF92DF92EF92FF920F931F930E94EC
:10EDB000D09F009178091091790920917A093091BA
:10EDC0007B096B017C01C01AD10AE20AF30AF7FC45
:10EDD00013C020917709209520937709DC01CB019E
:10EDE0008A549C4FAF4FBF4F809378099093790915
:10EDF000A0937A09B0937B0981E0909177099111F2
:10EE000001C080E01F910F91FF90EF90DF90CF90B5
:10EE100008950E945EA2A4E0B1E08C918F7D8C9356
:10EE20009FB7F894E5E0F1E08081806280839FBF26
:10EE30008C918F7B8C939FB7F894808180648083C2
:10EE40009FBF6A98729A54985C9A82E08093900966
:10EE50000E94C7C51092E7130895CF93DF931F92C6
:10EE60001F92CDB7DEB789839A830E94E0658981BE
:10EE70009A810F900F90DF91CF910C9416956F921D
:10EE80007F928F929F92AF92BF92CF92DF92EF923A
:10EE9000FF920F931F93CF93DF9300D01F92CDB7B4
:10EEA000DEB76C013B014701580129833A834B834C
:10EEB0005C830E94E06583E080932A02D092E206A0
:10EEC000C092E1067092E0066092DF0629813A81E5
:10EED0004B815C81CA01B9010E94E3F76093DB06B4
:10EEE0007093DC068093DD069093DE060E946CF240
:10EEF0006B017C019B01AC01C501B4010E949EF62F
:10EF00000E94E3F76093D7067093D8068093D906E2
:10EF10009093DA06A7019601F301608171818281E5
:10EF200093810E949EF60E94E8F760934D0A7093C9
:10EF30004E0A80934F0A9093500A8BEA91E7909380
:10EF40002902809328020F900F900F900F90DF916D
:10EF5000CF911F910F91FF90EF90DF90CF90BF90D6
:10EF6000AF909F908F907F906F900895CF92DF9297
:10EF7000EF92FF920F931F93CF93DF938C01EB01DE
:10EF80006A0179010E94E06523E020932A02109330
:10EF9000E2060093E106D093E006C093DF06A601E7
:10EFA000DD0C660B770B4093DB065093DC06609319
:10EFB000DD067093DE06C701FF0CAA0BBB0B841B9A
:10EFC000950BA60BB70B8093D7069093D806A0930A
:10EFD000D906B093DA0688819981092E000CAA0B14
:10EFE000BB0B841B950BA60BB70B80934D0A90931C
:10EFF0004E0AA0934F0AB093500A88E292E790938A
:10F00000290280932802DF91CF911F910F91FF90E9
:10F01000EF90DF90CF9008953F924F925F926F9262
:10F020007F928F929F92AF92BF92CF92DF92EF9298
:10F03000FF920F931F93CF93DF93CDB7DEB72C973B
:10F040000FB6F894DEBF0FBECDBF5C01DC01599650
:10F050008D909C905A97F40181859285A385B48503
:10F060009C01AD012F5F3F4F4F4F5F4F29873A877C
:10F070004B875C87D5011496CD90DD90ED90FC9088
:10F080001797C114D104E104F10439F0BFEFCB1A92
:10F09000DB0AEB0AFB0A312C07C0F401C080D180E7
:10F0A000E280F38033243394260137011D821E82CF
:10F0B0001F821886F40181859285A385B4852D81F0
:10F0C0003E814F815885281739074A075B0708F0AA
:10F0D00064C089859A85AB85BC858C159D05AE0578
:10F0E000BF0550F482E0C82ED12CE12CF12C92E027
:10F0F000492E512C612C712C9E012F5F3F4FB7017F
:10F10000A601C4010E94E8C9882309F446C0898188
:10F110009A81AB81BC81892B8A2B8B2B41F02601F4
:10F1200037019FEF491A590A690A790A05C0C414C0
:10F13000D504E604F70491F02D813E814F81588576
:10F140002F5F3F4F4F4F5F4F2D833E834F83588735
:10F150003FEFC31AD30AE30AF30AACCF0FEF1FEF56
:10F160002FEF3FE0B301A201C4010E9457C9F82E5E
:10F17000882399F0D50114964D915D916D917C9104
:10F180001797411551056105710549F093018201F9
:10F19000C4010E9457C9811102C0F12C29C0D501B8
:10F1A00014964D925D926D927C921797332051F098
:10F1B000D301C2010196A11DB11DF4018083918389
:10F1C000A283B383F50185899689A789B08D892BA0
:10F1D0008A2B8B2B69F4D50155964D925D926D92D9
:10F1E0007C92589711968C911197806811968C9308
:10F1F0008F2D2C960FB6F894DEBF0FBECDBFDF91DA
:10F20000CF911F910F91FF90EF90DF90CF90BF9023
:10F21000AF909F908F907F906F905F904F903F90B6
:10F2200008951F920F920FB60F9211240BB60F92F2
:10F230002F933F934F935F936F937F938F939F93FE
:10F24000AF93BF93EF93FF93E091140A81E08E0F89
:10F250008F779091C6002091150A821731F0F0E067
:10F26000EC56F64F90838093140A20919309422F15
:10F2700050E04C30510508F046C0FA018827EE589E
:10F28000FF4F8F4F0C948AF99D3441F09E34B9F4AE
:10F2900081E005C09A3330F09D3471F582E08093AF
:10F2A000930946C0903308F043C0903209F440C03F
:10F2B0009D3211F53DC0913329F0943329F09032FD
:10F2C000D9F436C083E0EBCF88E0E9CF903321F06A
:10F2D000913391F486E0E3CF84E0E1CF983361F499
:10F2E00085E0DDCF923341F487E0D9CF913321F42B
:10F2F00089E0D5CF903311F08BE0D1CF8AE0CFCF2A
:10F300009A30B1F413C09A3099F4273049F02A307A
:10F3100059F0253059F41092150210929A0406C043
:10F3200081E896E10E945EAF0E94876C109293097B
:10F33000FF91EF91BF91AF919F918F917F916F91CD
:10F340005F914F913F912F910F900BBE0F900FBE89
:10F350000F901F9018951F920F920FB60F921124C5
:10F360000BB60F928F939F93EF93FF938091370A81
:10F37000E82FF0E0EA5EF54F90818F5F8F71809308
:10F38000370A9093C6008091C00080648093C000CB
:10F390009091360A8091370A981305C08091C10078
:10F3A0008F7D8093C100FF91EF919F918F910F907E
:10F3B0000BBE0F900FBE0F901F9018958F929F92CB
:10F3C000AF92BF92CF92DF92EF92FF920F931F9373
:10F3D000CF93DF93EC018B81811102C080E077C075
:10F3E00009891A892B893C890417150726073707CD
:10F3F000A8F36A017B01823029F4C886D986EA869F
:10F40000FB860DC0C114D104E104F10451F4188647
:10F4100019861A861B861C821D821E821F8281E02D
:10F4200056C088849984AA84BB84E98DFA8D258589
:10F4300030E0275F3F4FB501A401415051096109F8
:10F440007109022E04C076956795579547950A94E1
:10F45000D2F7D701C6010197A109B10904C0B69539
:10F46000A795979587952A95D2F784179507A607AC
:10F47000B70720F089288A288B2849F44D895E89AE
:10F480006F89788D4C835D836E837F8304C0841B7A
:10F49000950BA60BB70B4C015D018E010C5F1F4F46
:10F4A00081149104A104B10409F4A7CF4C815D81BA
:10F4B0006E817F819801898D9A8D0E94E8C991E0C3
:10F4C000891A9108A108B1088111EACF87CFDF918D
:10F4D000CF911F910F91FF90EF90DF90CF90BF9051
:10F4E000AF909F908F9008952F923F924F925F928E
:10F4F0006F927F928F929F92AF92BF92CF92DF9244
:10F50000EF92FF920F931F93CF93DF9300D01F9240
:10F51000CDB7DEB79C838B834B015A01DC01139678
:10F520008C91811103C08FEF9FEFEBC0EB81FC81C9
:10F53000818180FFF8CFAB81BC8151960D911D91E7
:10F540002D913C91549718964D915D916D917C91C0
:10F550001B97C501A0E0B0E068017901C41AD50A83
:10F56000E60AF70AC816D906EA06FB0618F4580197
:10F57000A41AB50A75018B819C8104969A838983AC
:10F58000612C92E0792EE114F10409F48BC0AB8177
:10F59000BC8118964D915D916D917C911B976A018C
:10F5A000B1E0DB22EB81FC8123811A012B0189E090
:10F5B00056944794379427948A95D1F7818D928DEC
:10F5C000223061F4FC01828D938DA48DB58DBC0138
:10F5D000CD01620D731D841D951D4AC0DC0114967A
:10F5E0001C9111501221C114D10401F511111EC03A
:10F5F000452B462B472B59F4EB81FC818589968955
:10F60000A789B08D84839583A683B7830FC0AB8110
:10F61000BC8114964D915D916D917C9117972981D4
:10F620003A810E94E8C9882309F47DCFEB81FC81EF
:10F63000218D328D84819581A681B7810297A109A0
:10F64000B109F901058404C0880F991FAA1FBB1FC7
:10F650000A94D2F74685578560897189840F951F72
:10F66000A61FB71FBC01CD01610F711D811D911D2A
:10F6700093012C193D0987012E153F0508F48901D6
:10F680000115F2E01F0779F52091EE083091EF089F
:10F690004091F0085091F1086217730784079507AD
:10F6A00019F421C0C5012DC09401AB01BC018091AA
:10F6B000F7089091F8080E94BC46882309F433CFDC
:10F6C000800E911EEB81FC8180859185A285B3859A
:10F6D000800F911FA11DB11D80879187A287B387DD
:10F6E000E01AF10A50CF40E00E941FC9882309F4B4
:10F6F0001ACFB6016251794FA801C4010E94A7F93F
:10F70000DFCF0F900F900F900F90DF91CF911F914F
:10F710000F91FF90EF90DF90CF90BF90AF909F90B0
:10F720008F907F906F905F904F903F902F900895B3
:10F73000DF92EF92FF920F931F93CF93DF937C01A1
:10F74000EB018A018DE0D82E40E250E0BE01C701F6
:10F75000CBDE8032910539F021E0892B09F420E0DD
:10F76000822F81953EC02881222399F1253E61F3A5
:10F770002E3251F30115110541F13B853F733F30A6
:10F7800021F54A8D5B8D452B01F52F713FEF320F2F
:10F790003530D8F430E021503109D29EC001D39EDB
:10F7A000900D1124D801A80FB91FFE0120E0AD0172
:10F7B000253088F431813D932F5F32962D30C1F78B
:10F7C000288126FF02C0FA0115862B8523FDBCCFB8
:10F7D00008C080E006C02B3010F43481ECCF3681B5
:10F7E000EACFDF91CF911F910F91FF90EF90DF90C3
:10F7F00008950F931F93CF93DF93FC01238122235E
:10F8000011F080E044C08B01EC01FB01878980315D
:10F8100039F18032B1F783E08B83F801428D538D4B
:10F82000648D758D4D8B5E8B6F8B788F9E012F5EF7
:10F830003F4FC8010E9468CA882319F31A8F098FA5
:10F8400081E08983188619861A861B861C821D8290
:10F850001E821F82188A1C861D861E861F8617C060
:10F8600082E08B831D8A1E8A1F8A188EFB01808D81
:10F87000918DA0E0B0E025E0880F991FAA1FBB1F63
:10F880002A95D1F7898B9A8BAB8BBC8BD7CFDF9125
:10F89000CF911F910F910895CF93DF93EC0141E039
:10F8A000611101C040E06C857D858E859F850E9439
:10F8B0001FC9882341F0888920E2829FC00111245A
:10F8C0008251994F02C080E090E0DF91CF9108957E
:10F8D000CF93DF93EC018B81882331F1898187FFFE
:10F8E0001FC061E0CE01D8DFFC01892BE9F08081E7
:10F8F000853ED1F08B81823040F489899A89AB8929
:10F90000BC89848F958FA68FB78F8D899E89AF898B
:10F91000B88D938F828FB58BA48B89818F778983E4
:10F92000DF91CF910C94DFC881E0888380E0DF9184
:10F93000CF9108952F923F924F925F926F927F9254
:10F940008F929F92AF92BF92CF92DF92EF92FF92EF
:10F950000F931F93CF93DF9300D01F92CDB7DEB7E5
:10F960008C014B011A01DC0113968C9113978130A5
:10F97000C1F411968C9181FF14C082FF18C0F80168
:10F98000418952896389748980859185A285B3856F
:10F9900084179507A607B70751F0C8010FDD81113D
:10F9A00006C081E0F80180838FEF9FEF2EC16101D7
:10F9B00085C0D80159968D919C915A97FC0124815C
:10F9C00021502A013B0139E076946794579447947B
:10F9D0003A95D1F7722E74207A01F1E0FF22772058
:10F9E00009F478C080E092E08E199F0956018C15C9
:10F9F0009D0508F45C01D80159962D913C915A97C8
:10FA000014968D919D910D90BC91A02D0297A10906
:10FA1000B109F901058404C0880F991FAA1FBB1FF3
:10FA20000A94D2F74685578560897189840F951F9E
:10FA3000A61FB71F9C01AD01270D311D411D511D92
:10FA400029013A01A11432E0B30609F089C080917E
:10FA5000EE089091EF08A091F008B091F10884159C
:10FA60009505A605B70569F41092F6088FEF9FEF8C
:10FA7000DC018093EE089093EF08A093F008B09318
:10FA8000F1089401B301A2018091F7089091F80860
:10FA90000E945A46882309F484CFF8018085918515
:10FAA000A285B3858A0D9B1DA11DB11D80879187FD
:10FAB000A287B3878A0C9B1CCA18DB08D80118964A
:10FAC0004D915D916D917C911B97C114D10409F00A
:10FAD00070CF7CC0E114F10409F084CF14964D91ED
:10FAE0005D916D917C9117974115510561057105E7
:10FAF00059F455968D919D910D90BC91A02D009734
:10FB0000A105B10539F521C09E012F5F3F4F0E942D
:10FB1000E8C9882309F445CF89819A81AB81BC81EA
:10FB2000F801218D328DF9012789203139F4883F80
:10FB3000FFEF9F07A105B10540F40CC0883F2FEFF0
:10FB40009207A2072FE0B20728F0C80165DA8111F9
:10FB500049CF27CFF80184839583A683B78342CF0B
:10FB6000E114F10419F5D80118964D915D916D914C
:10FB70007C911B9751968D919D910D90BC91A02DDC
:10FB8000481759076A077B0788F00E94DFC8882357
:10FB900009F407CF81E08093F6084092EE08509276
:10FBA000EF086092F0087092F10808C041E0C301CC
:10FBB000B2010E941FC9882309F4F3CEA501B40144
:10FBC000C7018251994F0E94A7F967CF51968D9135
:10FBD0009D910D90BC91A02D84179507A607B7079E
:10FBE00040F4F801418B528B638B748B8181806868
:10FBF0008183D80111968C9183FD02C0C10105C09B
:10FC0000C80166DE8111FACFCCCE0F900F900F9015
:10FC10000F90DF91CF911F910F91FF90EF90DF90A8
:10FC2000CF90BF90AF909F908F907F906F905F909C
:10FC30004F903F902F900895CF93DF93EC0148DED3
:10FC40001B82DF91CF9108954F925F926F927F92C6
:10FC5000AF92BF92CF92DF92EF92FF920F931F93DA
:10FC6000CF93DF931F92CDB7DEB78C017B015A0192
:10FC7000D22EDB0159968D919C915A97F801928F63
:10FC8000818F40E050E0BA01C70198DBC12CF70139
:10FC900080859185A285B38541895289638974895C
:10FCA00084179507A607B70708F062C025E0B69548
:10FCB000A795979587952A95D1F7F82FFF707F2EF6
:10FCC000D70113968C91823008F462C041E050E075
:10FCD000BE016F5F7F4FC70107DC019719F489816F
:10FCE00090E002C08FEF9FEF019609F451C0F70139
:10FCF00080859185A285B3854F96A11DB11D808712
:10FD00009187A287B387F0E27F9EC0011124BC01D6
:10FD10006251794F61157105D9F1DB012C912223D4
:10FD200019F0253ED1F466C1C1100EC04091EE0815
:10FD30005091EF086091F0087091F108F801448744
:10FD4000558766877787708AFC01E251F94F808179
:10FD5000882361F0CC24C3949ACF4BE050E0C501D6
:10FD60000E949AF9892B09F092CF14C0CC24C39435
:10FD70008D2D8274823461F4CC2009F489C0D801BD
:10FD800050967C9061E0C80187DD009709F006C1BC
:10FD900080E033C1D7FCFCCFF0E27F9EA0011124AC
:10FDA0009A012251394FD9011B968C91817121F012
:10FDB0008D2D827109F068C08091EE089091EF0856
:10FDC000A091F008B091F108F80184879587A68783
:10FDD000B787708AFA01E251F94F4489558960E08A
:10FDE00070E0BA0155274427D80155964D935D938D
:10FDF0006D937C935897828D938DA0E0B0E0482B53
:10FE0000592B6A2B7B2BD80155964D935D936D939F
:10FE10007C935897D9011B968C91887159F4848DE5
:10FE2000958DA68DB78DF801818B928BA38BB48BAA
:10FE300081E010C0803141F598012F5E3F4FD8011D
:10FE400059968D919C915A970E9468CA8823E1F037
:10FE500084E0F80183838D2D8F70D80111968C93E7
:10FE60001197F801148215821682178218961D9236
:10FE70001D921D921C921B97D4FEB0C0C8010E9417
:10FE800047968111ABC084CFD80113961C9280CFC6
:10FE9000F7018381823009F47BCF81899289A3891C
:10FEA000B489803E9F4FAF41B10508F071CFC701C3
:10FEB000B3D8882309F46CCF0E94DFC8882309F4E3
:10FEC00067CFD70159962D913C915A9714968D91F1
:10FED0009D910D90BC91A02D0297A109B109F90146
:10FEE000058404C0880F991FAA1FBB1F0A94D2F76C
:10FEF0004684578460887188480E591E6A1E7B1E8E
:10FF000081E08093F6084092EE085092EF086092EC
:10FF1000F0087092F10880E092E0EEEEF6E0DF018A
:10FF20009C011D9221503040E1F7CC24C394D701AD
:10FF30005996ED91FC915A978481C81698F42EEE4B
:10FF400036E0B301A2014C0D511D611D711D809160
:10FF5000F7089091F8080E945A46882309F418CFB0
:10FF6000C394E5CF80E092E0A0E0B0E0058404C057
:10FF7000880F991FAA1FBB1F0A94D2F7F701418966
:10FF8000528963897489840F951FA61FB71F818BBF
:10FF9000928BA38BB48B8EEE96E0712C20E2DC0169
:10FFA0001D922A95E9F72BE0F501DC0101900D92F5
:10FFB0002A95E1F721E238E2FC01318B208B40E009
:10FFC00058E057874687338B228B318F208F578B92
:10FFD000468B0E94DFC88111DFCEDACED5FE08C085
:10FFE000F8014189528963897489C801E7D905C03C
:10FFF00081E003C0C110AECE99CE0F90DF91CF91BA
:020000021000EC
:100000001F910F91FF90EF90DF90CF90BF90AF9036
:100010007F906F905F904F9008952F923F924F92F4
:100020005F926F927F928F929F92AF92BF92CF9288
:10003000DF92EF92FF920F931F93CF93DF93CDB791
:10004000DEB7C254D1090FB6F894DEBF0FBECDBFE4
:100050004C015B018A01322E1C8E1F8E19821C827C
:100060006115710511F410E0A3C0FC0183818111B9
:10007000FACFFA0180818F3209F098C0F5018381AF
:100080008250823058F0618D728DCE010196B1DBC5
:10009000882349F3CE0101967C0101C07501C80196
:1000A0008C010196F80120812F32D1F36E01FCE121
:1000B000CF0ED11C3601CE0101962C012396CFAE76
:1000C00023972D2C9BE09150E7E3F0E0EC0FFD1F10
:1000D000E90FF11D80E280839111F5CFD80127E06F
:1000E0004A2F3B2F8D91811107C08FA9803209F4CF
:1000F000BACF842F932F2CC08F32B9F38E3231F4C4
:100100002A3009F4B0CF98E02AE0EACFE1E7F6E13F
:100110003491332321F031963813FACFA4CF291725
:1001200008F4A1CF813208F49ECF8F3709F49BCF1A
:1001300031E0390FE7E3F0E0EC0FFD1FE90FF11DAF
:100140009FE9980F9A3108F480528083932FC8CF8B
:100150008C01FC01208101962F32D1F32223E9F09A
:1001600021E0AE01495C5F4FB701C6016DDD882318
:1001700009F479CFEA14FB0411F0C7015DDDC61460
:10018000D70441F023969FAD2397822D7601C92E87
:10019000D82E98CF942D852DF9CF232DAE01495C13
:1001A0005F4FB701C40150DD182F02C07B017ECF25
:1001B000CE0101960E944DC5CE014C960E944DC5C0
:1001C000812FCE5BDF4F0FB6F894DEBF0FBECDBFE1
:1001D000DF91CF911F910F91FF90EF90DF90CF9023
:1001E000BF90AF909F908F907F906F905F904F9057
:1001F0003F902F900895CF93DF93EB01FC01238173
:10020000211102C080E027C02250223020F48FE26A
:10021000888319821FC060E03FDB009799F3FC01DF
:1002200090E080E02EE23081303269F0883029F4AD
:10023000DE01A90FB11D2C939F5F3081DE01A90F54
:10024000B11D3C939F5F8F5F31968B3061F7C90F73
:10025000D11D188281E0DF91CF9108952F923F92B6
:100260004F925F926F927F928F929F92AF92BF92C6
:10027000CF92DF92EF92FF920F931F93CF93DF9372
:10028000EC0145EF55E181E090E0FA0125913491D0
:10029000C217D3070CF05DC09C0121503109220F19
:1002A000331F220F331FD901AD50BA4EFD016591A6
:1002B00074912F503A4EF901A590B490FC01EE0FC5
:1002C000FF1FEE0FFF1FED50FA4EE590F490FD0179
:1002D000C590D490FA0105911491F90125903490BC
:1002E000072E000C880B990B0E946CF22B013C012D
:1002F000CA19DB09BE01DD0F880B990B0E946CF255
:100300004B015C01B7016C197D09072E000C880BAD
:10031000990B0E946CF29B01AC01C501B4010E94D3
:10032000CBF26B017C01B80162197309072E000C36
:10033000880B990B0E946CF29B01AC01C701B601BE
:100340000E947BF79B01AC01C301B2010E949FF6A2
:1003500011C001964C5F5F4F8032910509F095CF37
:10036000EFE6F6E165917491072E000C880B990B6E
:100370000E946CF2DF91CF911F910F91FF90EF904F
:10038000DF90CF90BF90AF909F908F907F906F90B5
:100390005F904F903F902F900895609190047091DE
:1003A0009104809192049091930408954F925F92EA
:1003B0006F927F92AF92BF92CF92DF92EF92FF92B5
:1003C0000F931F93CF93DF93009709F456C0FC015E
:1003D000208121FD52C0EB018C0147A050A461A4F3
:1003E00072A4AFA0B8A4C9A4DAA49501A601C30160
:1003F000B2010E9466F287FF40C0A3019201C301CF
:10040000B2010E94CBF22B013C01F80183A994A90F
:10041000A5A9B6A9BC01CD0190589B01AC010E94D1
:100420009FF6F80127A530A941A952A90E94CBF255
:100430009B01AC01C301B2010E949EF60E940AF921
:100440007B018C019B01AC01B501C6010E9466F2E3
:1004500087FF02C0750186019701A801B501C60199
:100460000E9466F2882349F0A701B8014FA358A75C
:1004700069A77AA7888181608883DF91CF911F91D6
:100480000F91FF90EF90DF90CF90BF90AF907F9053
:100490006F905F904F9008952F923F924F925F928E
:1004A0006F927F928F929F92AF92BF92CF92DF9284
:1004B000EF92FF920F931F93CF93DF93CDB7DEB7E9
:1004C00068970FB6F894DEBF0FBECDBF1C015B016D
:1004D0008A01DC01D7966D917D918D919C91DA977F
:1004E0000E946AF26B017C01F50120813181428119
:1004F00053810E94CBF20E9465F70E94E8F769875A
:100500007A878B879C87D8012D913D914D915C9185
:10051000C701B6010E94CBF20E9465F70E94E8F77E
:100520006D877E878F87988B29853A854B855C857B
:10053000283731054105510540F488E790E0A0E0F7
:10054000B0E089879A87AB87BC872D853E854F852C
:100550005889283731054105510540F488E790E076
:10056000A0E0B0E08D879E87AF87B88B91012D5BAF
:100570003F4FD9018D919D910D90BC91A02D8D8300
:100580009E83AF83B887BC01CD010E946CF2698362
:100590007A838B839C8369857A858B859C850E9471
:1005A0006AF2698B7A8B8B8B9C8B20E030E0A901FF
:1005B00069817A818B819C810E9466F2882339F15E
:1005C000A7019601C701B6010E94CBF24B015C0165
:1005D00029893A894B895C89CA01B9010E94CBF209
:1005E0009B01AC01C501B4010E949EF64B015C0168
:1005F00029813A814B815C81CA01B9010E949FF631
:100600009B01AC01C501B4010E947BF703C060E00F
:1006100070E0CB010E9465F70E94E3F72B013C01DB
:100620006D817E818F81988590958095709561957B
:100630007F4F8F4F9F4F0E946CF24B015C016D8585
:100640007E858F8598890E946AF26D837E838F8371
:10065000988720E030E0A901C501B4010E9466F24C
:10066000882349F12D813E814F815885CA01B90106
:100670000E94CBF26D8B7E8B8F8B988FA70196019A
:10068000C701B6010E94CBF29B01AC016D897E8946
:100690008F89988D0E949EF66B017C01A5019401C3
:1006A000C501B4010E949FF69B01AC01C701B601D0
:1006B0000E947BF703C060E070E0CB010E9414F859
:1006C000F10182889388A488B58875016401C418F3
:1006D000D508E608F7080E94E3F7C61AD70AE80A21
:1006E000F90AF7FE6BC020E030E0A90169817A8148
:1006F0008B819C810E9466F2882309F447C029817E
:100700003A814B815C81CA01B9010E949FF66B015D
:100710007C01C501B4010E946AF29B01AC01C701D2
:10072000B6010E94CBF26B017C0129893A894B8981
:100730005C89CA01B9010E94CBF29B01AC01C701DF
:10074000B6010E949EF66B017C012D813E814F8196
:100750005885CA01B9010E94CBF29B01AC01C701C7
:10076000B6010E949FF66B017C0120E030E040E87A
:1007700050E469817A818B819C810E94CBF29B013C
:10078000AC01C701B6010E947BF703C060E070E0D6
:10079000CB010E9465F70E94E3F72B013C0197FF14
:1007A00003C0412C512C3201481459046A047B04C3
:1007B00010F024013501C12CD12C76018FB7F894AB
:1007C000D1019C9193FD22C0F101468A578A608E27
:1007D000718EC40CD51CE61CF71C5A96CD92DD9286
:1007E000ED92FC925D9729853A854B855C85DB9679
:1007F0002D933D934D935C93DE97FF962D853E851B
:100800004F85588920833183428353838FBF6896F5
:100810000FB6F894DEBF0FBECDBFDF91CF911F9111
:100820000F91FF90EF90DF90CF90BF90AF909F908F
:100830008F907F906F905F904F903F902F90089592
:10084000CF92DF92EF92FF9280918514882371F10D
:10085000C0908114D0908214E0908314F09084149E
:1008600020E030E0A901C701B6010E9466F28823AA
:10087000E9F020E030E040E05FE3C701B6010E940C
:10088000CBF29B01AC010E94CBF22BED3FE049E49F
:1008900050E40E94CBF29B01AC0160E070E080E884
:1008A0009FE30E947BF76B017C0106C0C12CD12C19
:1008B00080E8E82E8FE3F82EC0922604D092270419
:1008C000E0922804F09229046091020270910302E0
:1008D000072E000C880B990B0E946CF22AE037ED72
:1008E00043E25CE30E94CBF2A70196010E94CBF2A7
:1008F00060931C0270931D0280931E0290931F024E
:10090000FF90EF90DF90CF90089591E09093CB040B
:100910003FB7F8942091360A9091370A3FBF2913C8
:1009200004C09091C00095FD3EC09091360A9F5F33
:100930009F712091370A921325C00FB607FCF9CF9B
:100940002091C00025FFF5CF2091370AE22FF0E07B
:10095000EA5EF54F30812F5F2F712093370A309375
:10096000C6002091C00020642093C0003091360A58
:100970002091370A3213DDCF2091C1002F7D2093C3
:10098000C100D7CFE091360AF0E0EA5EF54F8083F0
:100990002FB7F8949093360A8091C10080628093BB
:1009A000C1002FBF08959FB7F8948093C60080912F
:1009B000C00080648093C0009FBF08952F923F9233
:1009C0004F925F926F927F928F929F92AF92BF925F
:1009D000CF92DF92EF92FF920F931F93CF93DF930B
:1009E000CDB7DEB7C456D1090FB6F894DEBF0FBE3F
:1009F000CDBF60969FAF8EAF609749AB59AF6EAFDA
:100A000021967FAF2197322EDC01CD90DD90ED90C5
:100A1000FC908091660A9091670AA091680AB09153
:100A2000690AC81AD90AEA0AFB0A6096EEADFFAD58
:100A30006097448155816681778180916A0A90919F
:100A40006B0AA0916C0AB0916D0A8A019B01081B88
:100A5000190B2A0B3B0B0DA71EA72FA738AB408500
:100A600051856285738580916E0A90916F0AA0917D
:100A7000700AB091710A8A019B01081B190B2A0B9D
:100A80003B0B0DAB1EAB2FAB38AF44845584668453
:100A900077848091720A9091730AA091740AB09140
:100AA000750A53014201881A990AAA0ABB0A09F475
:100AB00096C080910D04811139C06091000270913F
:100AC0000102072E000C880B990B0E946CF29B010F
:100AD000AC01609190047091910480919204909186
:100AE00093040E9466F287FF21C04092720A5092DE
:100AF000730A6092740A7092750AE8EDF6E18491C7
:100B00008F010F5F1F4F882319F0FFDEF801F7CF29
:100B1000E9EAF6E184918F010F5F1F4F882319F0F6
:100B2000F4DEF801F7CF812C912C5401C501B401FA
:100B30000E946CF214E0319EF0011124E45EFD4F3E
:100B400020813181428153810E94CBF20E94E3F7E0
:100B50002B013C0197FF08C070946094509440941E
:100B6000411C511C611C711C60911515709116156A
:100B700080911715909118150E94E3F79B01AC0125
:100B8000A8ECB0E00E947FF6641575058605970510
:100B90004CF56096EEADFFAD609784859585A68592
:100BA000B7858093720A9093730AA093740AB093E6
:100BB000750AE8EDF6E184918F010F5F1F4F8823DE
:100BC00019F0A3DEF801F7CFEAE8F6E184918F018E
:100BD0000F5F1F4F882319F098DEF801F7CF812CA3
:100BE000912C5401D701C6018827B7FD8395992719
:100BF000AA27BB27182F2DA53EA54FA558A957FDFD
:100C000012608DA99EA9AFA9B8ADB7FD1460B7FC5D
:100C10001860C501B4010E946CF2A4E03A9EF00194
:100C20001124E45EFD4F20813181428153810E9475
:100C3000CBF24B015C0120E030E0A9010E94C5F835
:100C400018164CF420E030E040E05FE3C501B40149
:100C50000E949FF608C0A501940160E070E080E06A
:100C60009FE30E949EF60E94E3F76AAF7BAF8CAFD2
:100C70009DAF8091760A8F5F8F706B968FAF6B9769
:100C80008091770A6B960FAD6B97801304C080E05C
:100C90000E946967F5CFE091760A2E2F30E03CA7DD
:100CA0002BA73FE4E39FF0011124EE50F14F108297
:100CB00012A3D701C601F7FE07C088279927DC01D8
:100CC0008C199D09AE09BF0982839383A483B583E0
:100CD0008FE40BA51CA5809FF001819FF00D1124CE
:100CE000EE50F14F8DA59EA5AFA5B8A9B7FF07C0DF
:100CF000B095A095909581959F4FAF4FBF4F86833C
:100D00009783A087B1878FE40BA51CA5809FF00176
:100D1000819FF00D1124EE50F14F8DA99EA9AFA92E
:100D2000B8ADB7FF07C0B095A095909581959F4F3E
:100D3000AF4FBF4F82879387A487B5878FE40BA5FA
:100D40001CA5809FF001819FF00D1124EE50F14F02
:100D50002AAD3BAD4CAD5DAD26873787408B518BBF
:100D60004281538164817581068117812085318597
:100D7000041715072607370714F48A019B018FE42F
:100D8000ABA5BCA58A9FF0018B9FF00D1124EE50FE
:100D9000F14F82859385A485B58580179107A207B9
:100DA000B30764F48AAD9BADACADBDAD80179107C0
:100DB000A207B30764F4D901C8010DC00AAD1BAD89
:100DC0002CAD3DAD081719072A073B0724F08AAD63
:100DD0009BADACADBDAD2FE40BA51CA5209FF001D4
:100DE000219FF00D1124EE50F14F828B938BA48B39
:100DF000B58B0697A105B10510F40C94A590DF0101
:100E0000A95BBF4F809195049091960411969C9395
:100E10008E93129680919704909198048D939C9351
:100E20003182452B462B472B09F017988FE40BA5F1
:100E30001CA5809FF001819FF00D1124EE50F14F11
:100E400086819781A085B185892B8A2B8B2B09F010
:100E500016988FE40BA51CA5809FF001819FF00DD3
:100E60001124EE50F14F82859385A485B585892B99
:100E70008A2B8B2B09F015982AAD3BAD4CAD5DAD9F
:100E8000232B242B252BB1F080913C0A882319F0C9
:100E9000815080933C0A311004C0149880E2809302
:100EA0003C0A30904A0420904B0400914C0410916D
:100EB0004D0408C030904604209047040091480437
:100EC00010914904232D322DA80169A979AD8EAD69
:100ED00021969FAD21970E9466F287FD02C00C9477
:100EE0009D90C701B6010E946CF22091D804309108
:100EF000D9044091DA045091DB040E94CBF22B011B
:100F00003C01698B7A8B8B8B9C8B6DA57EA58FA505
:100F100098A90E946CF22091DC043091DD0440918C
:100F2000DE045091DF040E94CBF26DA77EA78FA74D
:100F300098AB6D8B7E8B8F8B988F6DA97EA98FA9B7
:100F400098AD0E946CF22091E0043091E104409150
:100F5000E2045091E3040E94CBF26B017C01698FA3
:100F60007A8F8B8F9C8F2091E4043091E50440911F
:100F7000E6045091E704C501B4010E94CBF26D8FE5
:100F80007E8F8F8F98A32FE44BA55CA5249FF00143
:100F9000259FF00D1124EE50F14F82809380A480A4
:100FA000B58056E085169104A104B104E4F486806E
:100FB0009780A084B184A6E08A169104A104B104AC
:100FC00094F482849384A484B584B6E08B1691044F
:100FD000A104B10444F4DC01CB01BF7787A790AB37
:100FE000A1ABB2AB34C0A3019201C301B2010E9414
:100FF000CBF22B013C012DA53EA54FA558A9CA0156
:10100000B9010E94CBF29B01AC01C301B2010E9465
:101010009FF64B015C01A7019601C701B6010E9432
:10102000CBF29B01AC01C501B4010E949FF60E9466
:101030000AF92FE44BA55CA5249FF001259FF00D34
:101040001124EE50F14F67A770AB81AB92AB8FE4E8
:10105000ABA5BCA58A9FF0018B9FF00D1124EE502B
:10106000F14F27A530A941A952A960E070E080E8BE
:101070009FE30E947BF726966CAF7DAF8EAF9FAF4C
:1010800026979B01AC01632D722DC8010E94CBF203
:101090006B017C018091760A9091770A891B8F7091
:1010A00027968FAF2797A701960160E074E284E747
:1010B00099E40E947BF70E94D0F84B015C012796CF
:1010C0008FAD279782508630D0F580914204909161
:1010D0004304A0914404B091450488169906AA06D9
:1010E000BB0668F588199909AA09BB09BC01CD019D
:1010F000660F771F881F991F2796BFAD27970B2F65
:1011000010E020E030E0A90198010E9441F6CA01F8
:10111000B9010E946AF20E94D0F8860E971EA81E9E
:10112000B91EC501B4010E946AF29B01AC0160E0E6
:1011300074E284E799E40E947BF76B017C012FB78E
:10114000F8948091CF0E9091D00EA091D10EB091D5
:10115000D20E880E991EAA1EBB1E8092CF0E9092B0
:10116000D00EA092D10EB092D20E2FBF8FE4EBA57D
:10117000FCA58E9F80018F9F100D11240E50114FE2
:10118000D8019F962D913D914D915C91D2976F968C
:101190002CAF3DAF4EAF5FAF6F97A70196016F9633
:1011A0006CAD7DAD8EAD9FAD6F970E94CBF22E964C
:1011B0006CAF7DAF8EAF9FAF2E97F80163A374A382
:1011C00085A396A322893389448955892DA73EA7F3
:1011D0004FA758ABCA01B9010E946AF26DAB7EAB52
:1011E0008FAB98AFA70196010E94CBF20E9465F7E2
:1011F0000E94E8F764966CAF7DAF8EAF9FAF6497A7
:10120000F80167AB70AF81AF92AF8E010F5E1F4FD9
:101210001FAF0EAF0051110966961FAF0EAF669754
:101220000EE514E068961FAF0EAF68978E010F5D54
:101230001F4F1AA709A766960EAD1FAD6697229697
:101240001FAF0EAF2297212C312C10E819AB0FE302
:1012500009AFAEADBFAD6D917D918D919D91BFAF49
:10126000AEAFA70196010E94CBF22296EEADFFAD84
:10127000229761937193819391932296FFAFEEAF82
:1012800022974B015C01E894B7F86896AEADBFAD0C
:1012900068974D905D906D907D906896BFAFAEAFB2
:1012A0006897A3019201C501B4010E94C5F8181600
:1012B000A4F4A5019401C301B2010E947BF75B0174
:1012C0008C019B01AC01B10189A999AD0E94C5F8BF
:1012D00018161CF4150109AB19AF0EAD1FAD29A5E9
:1012E0003AA50217130709F0B4CF20E030E040E838
:1012F0005FE3B10189A999AD0E9466F287FF4BC0F7
:101300007E0131E1E30EF11C66960EAD1FAD6697CE
:10131000910149A959ADD8016D917D918D919C9113
:101320000E94CBF2F80161937193819391938F01A5
:10133000EE15FF0569F78FE42BA53CA5829F800180
:10134000839F100D11240E50114F910149A959ADE1
:101350002E966CAD7DAD8EAD9FAD2E970E94CBF2DB
:10136000D80193966D937D938D939C9396976496F5
:101370006CAD7DAD8EAD9FAD64970E946AF2910118
:1013800049A959AD0E94CBF20E94E8F7F80167AB7A
:1013900070AF81AF92AF26962CAD3DAD4EAD5FAD37
:1013A00026976DA97EA98FA998AD0E94CBF269AB53
:1013B0007AAB8BAB9CAB8FE40BA51CA5809FF00197
:1013C000819FF00D1124EE50F14F82809380A48014
:1013D000B58081149104A104B10409F58681978137
:1013E000A085B185892B8A2B8B2BC9F482859385A7
:1013F000A485B585892B8A2B8B2B89F420916914C0
:1014000030916A1440916B1450916C1469A97AA9B7
:101410008BA99CA90E94CBF20E9465F727C22AAD36
:101420003BAD4CAD5DAD232B242B252B49F06091BA
:101430006D1470916E1480916F149091701408C0A7
:10144000609165147091661480916714909168148E
:1014500029A93AA94BA95CA90E94CBF20E9465F781
:101460000E94E8F76B017C018091CB0E9091CC0E2D
:10147000A091CD0EB091CE0E0DA51EA52FA538A919
:1014800080179107A207B30708F4E2C08114910402
:10149000A104B10441F120914E0430914F044091D8
:1014A0005004509151042C153D054E055F05D8F4AC
:1014B0006DA57EA58FA598A90E9432F62B013C014F
:1014C000A7019601C501B4010E9432F646165706DF
:1014D0006806790640F4C301B201A50194010E9497
:1014E00041F669017A018FE40BA51CA5809FF001EC
:1014F000819FF00D1124EE50F14F86809780A084DB
:10150000B18481149104A104B10441F120915204E9
:101510003091530440915404509155042C153D05CD
:101520004E055F05D8F46DA57EA58FA598A90E94EC
:1015300032F62B013C01A7019601C501B4010E94BE
:1015400032F6461657066806790640F4C301B20122
:10155000A50194010E9441F669017A018FE40BA56F
:101560001CA5809FF001819FF00D1124EE50F14FDA
:1015700082849384A484B58481149104A104B10469
:1015800041F12091560430915704409158045091F4
:1015900059042C153D054E055F05D8F46DA57EA5B3
:1015A0008FA598A90E9432F62B013C01A701960154
:1015B000C501B4010E9432F6461657066806790640
:1015C00040F4C301B201A50194010E9441F66901F2
:1015D0007A018FE40BA51CA5809FF001819FF00D7F
:1015E0001124EE50F14F86849784A088B18881142D
:1015F0009104A104B10409F43DC120915A04309131
:101600005B0440915C0450915D042C153D054E0532
:101610005F0508F02FC16DA57EA58FA598A90E9432
:1016200032F62B013C01A7019601C501B4010E94CD
:1016300032F6461657066806790608F01BC1C30144
:10164000B201A50194010E9441F669017A0112C11B
:1016500081149104A104B104A9F160914E04709128
:101660004F0480915004909151046C157D058E05B6
:101670009F0540F50E946AF22DA93EA94FA958ADD9
:101680000E94CBF22B013C01C501B4010E946CF217
:101690004B015C01C701B6010E946AF2A5019401E9
:1016A0000E94CBF2A30192010E94C5F8181654F4CF
:1016B000A5019401C301B2010E947BF70E94E8F7E3
:1016C0006B017C018FE40BA51CA5809FF001819F1D
:1016D000F00D1124EE50F14F4680578060847184E4
:1016E0004114510461047104A9F160915204709194
:1016F000530480915404909155046C157D058E051A
:101700009F0540F50E946AF22DA93EA94FA958AD48
:101710000E94CBF24B015C01C301B2010E946CF24A
:101720002B013C01C701B6010E946AF2A30192019C
:101730000E94CBF2A50194010E94C5F8181654F43A
:10174000A3019201C501B4010E947BF70E94E8F752
:101750006B017C018FE40BA51CA5809FF001819F8C
:10176000F00D1124EE50F14F42845384648475844B
:101770004114510461047104A9F1609156047091FF
:10178000570480915804909159046C157D058E057D
:101790009F0540F50E946AF22DA93EA94FA958ADB8
:1017A0000E94CBF24B015C01C301B2010E946CF2BA
:1017B0002B013C01C701B6010E946AF2A30192010C
:1017C0000E94CBF2A50194010E94C5F8181654F4AA
:1017D000A3019201C501B4010E947BF70E94E8F7C2
:1017E0006B017C018FE40BA51CA5809FF001819FFC
:1017F000F00D1124EE50F14F86849784A088B188B3
:1018000081149104A104B104A9F160915A0470916A
:101810005B0480915C0490915D046C157D058E05E0
:101820009F0540F50E946AF22DA93EA94FA958AD27
:101830000E94CBF22B013C01C501B4010E946CF265
:101840004B015C01C701B6010E946AF2A501940137
:101850000E94CBF2A30192010E94C5F8181654F41D
:10186000A5019401C301B2010E947BF70E94E8F731
:101870006B017C018FE42BA53CA5829F8001839F97
:10188000100D11240E50114FF801ED5BFF4FC08277
:10189000D182E282F382C701B6010E946AF26B0133
:1018A0007C0129A93AA94BA95CA90E947BF76A96F9
:1018B0006CAF7DAF8EAF9FAF6A97D801D3966D9313
:1018C0007D938D939C93D69720E030E040E85BE4D5
:1018D000C701B6010E94CBF220E034E244EF59E4A4
:1018E0000E947BF70E94E3F7F801668F778F80A351
:1018F00091A3F3A1F9AFD8019496BC91BEAFF801C2
:10190000F5A12196FFAF2197D8019696BC91239619
:10191000BFAF23970EE614E0A1961FAF0EAFA197BD
:101920002E0111E1410E511C4EE6242E44E0342ECE
:1019300066966EAC7FAC669709AD0AAF1EAD1DA76B
:10194000FDABB9AB10E0D3018D909D90AD90BD90F3
:101950003D01E894B7F8F101C190D190E190F19088
:101960001F01A7019601C501B4010E94C5F8181610
:1019700074F5112339F129AD3EAD21964FAD219774
:1019800023965FAD2397C701B6010E94CBF26B018E
:101990007C012AAD3DA54DA959A9C501B4010E94FC
:1019A000CBF2A70196010E94C5F818167CF4A50198
:1019B0009401C701B6010E947BF76AAF7DA78DAB8A
:1019C00099AB04C0CAAEDDA6EDAAF9AA11E0641471
:1019D000750409F0B8CF27960FAD2797002309F4B7
:1019E00055C1C090520AD090530AE090540AF0902A
:1019F000550A2DEB37E346E855E3B601C7010E94CF
:101A000066F287FD43C19601A70169AD7EAD2196BF
:101A10008FAD219723969FAD23970E9466F287FD95
:101A200005C00C2D2D2C3E2C1F2D08C009AD2EAC51
:101A300021963FAC219723961FAD23979601A701CE
:101A4000602F722D832D912F0E947BF7A5966CAF8E
:101A50007DAF8EAF9FAFA59726E53AE062963FAF88
:101A60002EAF629780E090E0A0E8BFE32A968CAFAB
:101A70009DAFAEAFBFAF2A972B961FAE2B97629646
:101A8000AEADBFAD62976D917D918D919D91629646
:101A9000BFAFAEAF6297A5962CAD3DAD4EAD5FAD7D
:101AA000A5970E94CBF26B017C016696EEADFFAD6F
:101AB000669781909190A190B1906696FFAFEEAF3E
:101AC00066972B96FFAD2B97FF23B1F02A962CAD8E
:101AD0003DAD4EAD5FAD2A970E94CBF26B017C010C
:101AE0002A962CAD3DAD4EAD5FAD2A97C501B40130
:101AF0000E94CBF24B015C01A5019401C701B60124
:101B00000E94C5F820E030E0A90118162CF5C501A7
:101B1000B4010E94C5F818164CF020E030E0A9018D
:101B2000C701B6010E9466F287FF05C0A5019401B6
:101B3000C701B60124C02401350177FA709477F803
:101B40007094A3019201C701B6010E94C5F818164E
:101B50005CF52601370128C0C501B4010E9466F278
:101B600087FD09C020E030E0A901C701B6010E944D
:101B7000C5F818164CF4A7019601C501B4010E94DE
:101B80009EF62B013C0110C02601370177FA7094B4
:101B900077F87094A5019401C301B2010E94C5F8C1
:101BA000181614F024013501A196AEADBFADA19772
:101BB000CD90DD90ED90FD90A196BFAFAEAFA19717
:101BC000A7019601C301B2010E94C5F81816ECF4F2
:101BD000A3019201C701B6010E947BF79B01AC01F2
:101BE0002A966CAD7DAD8EAD9FAD2A970E94CBF24B
:101BF0002A966CAF7DAF8EAF9FAF2A972B96BFAD65
:101C00002B97BF5F2B96BFAF2B976296EEADFFADC4
